:109FD4000D0A0D0A0D0A092A2A2A2A2A2A2A2A2AB5
:109FE4002A2A2A2A2A2A2A2A2A2A2A2A2A2A2A2ACD
:109FF4002A2A2A2A2A2A2A2A2A2A2A2A2A2A2A0DDA
:10A004000A00092A20202020202020205472616B7D
:10A01400426F78202038303532202076332E363087
:10A02400612020202020202020202A0D0A00092A37
:10A03400202020284329204A414D5341542F4A418E
:10A044003646544C2020205365702E323220323054
:10A054003133202020202A0D0A00092A2A2A2A2AFC
:10A064002A2A2A2A2A2A2A2A2A2A2A2A2A2A2A2A4C
:10A074002A2A2A2A2A2A2A2A2A2A2A2A2A2A2A2A3C
:10A084002A2A2A0D0A0020205472616B426F78201C
:10A094003830353220200000202076657273696FD5
:10A0A4006E20332E3630612000002843294A414D6A
:10A0B4005341542F4A413646544C0000594F524F95
:10A0C4004E0031332F30312F30312030303A3030A0
:10A0D4003A3030000A0D07546F6F206F6C642065AE
:10A0E4006C656D656E74732E200D0A000A0D0700F1
:10A0F4000D0A092A2A2A2020547261636B696E674B
:10A10400206F626A65637420736174656C6C697432
:10A114006520202A2A2A0D0A000D0A0D0A092A2A76
:10A124002A202053656C656374206F626A656374CA
:10A1340020736174656C6C69746520202A2A2A0D69
:10A144000A0007000D0A094461746120696E2052F7
:10A15400414D20776173206C6F737420212120534B
:10A1640065742064656661756C7420706172616DDC
:10A1740065746572202120070D0A004E4F43414C3F
:10A184004C0000594F524F4E0000205B592F4E5D3A
:10A19400203F20000D0A093D3D3D3D204144432020
:10A1A40076616C756520616E6420616E74656E6E97
:10A1B4006120646972656374696F6E203D3D3D3D45
:10A1C400200D0A0D0A000D0A20092D2D2D2D2D2DEF
:10A1D400204D41494E204D454E55202D2D2D2D2DE0
:10A1E4002D0D0A0D0A0009312E205265616C746927
:10A1F4006D6520547261636B696E672E0D0A0009E8
:10A20400322E20446973706C6179205363686564ED
:10A21400756C652E0D0A0009332E20557064617427
:10A224006520536174656C6C69746520456C656D5B
:10A23400656E74732E0D0A0009342E205570646106
:10A2440074652053746174696F6E20456C656D6527
:10A254006E74732E0D0A0009352E205570646174D6
:10A2640065205265616C74696D6520436C6F636B26
:10A274002E0D0A0009362E20436F6E6669677572CB
:10A284006174696F6E2E0D0A0009372E20486F73B2
:10A2940074206D6F64652E0D0A0009382E20446900
:10A2A4007265637420416E74656E6E6120636F6EB7
:10A2B40074726F6C2E0D0A0D0A000D0953656C65DE
:10A2C4006374205B312D382C532C4D5D3A20000DE6
:10A2D4000A0D0A092020203D3D3D3D3D3D3D3D3DCB
:10A2E40020555044415445204D454E55203D3D3D5B
:10A2F4003D3D3D3D3D0D0A0009312E204544495464
:10A304003A202020566965772F456469742073616B
:10A3140074656C6C69746520456C656D656E7473E9
:10A324002062792068616E642E0D0A0009322E20A5
:10A3340053454C4543543A2053656C65637420532C
:10A344006174656C6C697465732066726F6D2074DA
:10A3540068652064617461626173652E0D0A000989
:10A36400332E2052454C4F41443A20436C65617270
:10A374002064617461626173652026207265616482
:10A3840020696E206E657720456C656D656E74730B
:10A394002E0D0A0009342E20415050454E443A20D7
:10A3A400417070656E64206E657720456C656D65DF
:06A3B4006E74732E0D0A09
:10A3BA000009352E204D554C544920545241434BE7
:10A3CA003A20436F6E666967757265206D756C74A5
:10A3DA006920747261636B696E67207361742E20E1
:10A3EA006E756D6265722E0D0A0D0A000D0909530C
:10A3FA00656C6563743A20000D0A092A2A2A20200E
:10A40A0053656C656374206F626A65637420736157
:10A41A0074656C6C69746520202A2A2A0D0A000763
:10A42A000D0A0953656C6563746564206C697374FD
:10A43A002077696C6C206265206C6F73742E2041E2
:10A44A00726520796F752073757265203F000D0A59
:10A45A000D0A09312E2053656C6563742020202073
:10A46A003A2053656C65637420736174732E20629D
:10A47A00792068616E642E0D0A0009322E20536518
:10A48A006C65637420416C6C3A2053656C65637427
:10A49A0020616C6C20736174732E20696E2074685D
:10A4AA00652064617461626173652E0D0A00093367
:10A4BA002E2055706C6F6164202020203A20557040
:10A4CA006C6F61642073656C656374696F6E206478
:10A4DA006174612066696C652E0D0A00070D0A0910
:10A4EA0053746F726564206461746120696E206DB3
:10A4FA00656D6F72792077696C6C206265206C6F6C
:10A50A0073742E2041726520796F75207375726598
:10A51A00203F00070D0A204E6F20726F6F6D206674
:10A52A006F7220617070656E6420210D0A000D0A39
:10A53A000946696C6520666F726D6174204E4153DD
:10A54A004120284E29203A2020000D0A09486F7719
:10A55A00206D616E7920736174656C6C69746573C2
:10A56A0020636F6E66696775726520666F72206D0B
:10A57A00756C746920747261636B696E67206D6FA4
:10A58A006465203F202832202D2035292020000D07
:10A59A000A094F7574206F662072616E6765202103
:10A5AA000700536F757468004E6F72746800203329
:10A5BA00303000313230300032343030003438300C
:10A5CA003000393630300031393230300020202026
:10A5DA0020202020202043616C6C7369676E002064
:10A5EA0020202020202020204C6174697475646525
:10A5FA000020202020202020204C6F6E676974756F
:10A60A00646500202020416E74656E6E6120686565
:10A61A006967687400526F746F7220737461727420
:10A62A002028532F4E290020202020434F4D2070F0
:10A63A006F72742062617564000D0A0D0A09202088
:10A64A00203D3D3D3D3D3D3D3D3D20537461746996
:10A65A006F6E2044617461203D3D3D3D3D3D3D3D71
:10A66A000D0A0009312E20454449543A202020562B
:10A67A006965772F456469742073746174696F6EB4
:10A68A0020656C656D656E74732062792068616EF1
:10A69A00642E0D0A0009322E2052454C4F41443A8D
:10A6AA0020436C6561722064617461626173652024
:10A6BA0026207265616420696E206E657720646168
:10A6CA0074612E0D0A0D0A000D0A0D0A093D3D3D61
:10A6DA003D3D3D3D3D3D2053746174696F6E20459B
:10A6EA006C656D656E7473203D3D3D3D3D3D3D3D60
:10A6FA000D0A0D0A00253135733A20202573090009
:10A70A00253135733A2020252B352E336600090072
:10A71A00253135733A202025352E3266002531350C
:10A72A00733A20202573092000253135733A2020F9
:10A73A002573000D0A09456E746572202759272072
:10A74A00666F72207A65726F207365632E2061646A
:10A75A006A7573746D656E74000D0A09456E7465C9
:10A76A00722027512720666F722065786974000D60
:10A77A000A09456E74657220275265742E27206671
:10A78A006F72205265616C2054696D6520436C6F4D
:06A79A00636B207365747F
:10A7A0000D0A0D0A000950726573656E74205469B4
:10A7B0006D653A55544320002534642F25303262AC
:10A7C000642F25303262642025303262643A2530AD
:10A7D0003262643A25303262640D000D0A0D0A09B6
:10A7E000536574207265616C74696D6520436C6F8C
:10A7F000636B2E0D0A0950726573656E742054697F
:10A800006D653A55544320002534642F253032625B
:10A81000642F25303262642025303262643A25305C
:10A820003262643A25303262640D0A0009456E7462
:10A830006572207769746820666F726D6174205B41
:10A8400059592F4D4D2F44442048483A4D4D3A53C5
:10A85000535D20000D0A095365742074696D653AD3
:10A860002025730D0A000D0A09202020454E54456D
:10A8700052207768656E2072656164792E000D0A3A
:10A8800007202120466F726D6174204572726F72CD
:10A8900020210043415420004D69632D636C69639E
:10A8A0006B20004E6F00596573002020202020206F
:10A8B00020536174656C6C69746520203A00202017
:10A8C0002045706F63682054696D652054302020E6
:10A8D0003A002020202045706F6368205265762062
:10A8E0004B3020203A00204D65616E20416E6F6D27
:10A8F000616C79204D3020203A0020204D65616E3A
:10A90000204D6F74696F6E204E3020203A00202059
:10A91000496E636C696E6174696F6E2049302020E6
:10A920003A0020456363656E7472696369747920C7
:10A93000453020203A0020204172672070657269FE
:10A9400067656520573020203A00202020202052C3
:10A950002E412E412E4E2E204F3020203A00202016
:10A960002020202020204465636179204E31202062
:10A970003A0020446F776E6C696E6B204672712EC0
:10A98000463120203A0020202055706C696E6B20E3
:10A990004672712E463220203A00202020446F77E4
:10A9A0006E6C696E6B206D6F646520203A0020200C
:10A9B00020202055706C696E6B206D6F64652020BF
:10A9C0003A0020202045706F63682059656172202D
:10A9D000593020203A00446F70706C657220636FAC
:10A9E00072726563742E20203A0020204C4344206C
:10A9F0004D4120646973706C617920203A002020F9
:10AA0000204F666673657420666F72204631202081
:10AA10003A002020204F666673657420666F7220AE
:10AA2000463220203A002020202020463120736C1E
:10AA3000657728487A2920203A006E6F6E65004CB1
:10AA40005342200055534220004357202000464DDA
:10AA50002020000D0A0D0A09093D3D3D3D3D3D20E8
:10AA6000536174656C6C6974652064617461203D28
:10AA70003D3D3D3D3D0D0A0009257320252D7309FF
:10AA800009000925732025640009090959303A0095
:10AA90000925732025362E356600090954303A0001
:10AAA0000925732025366C640009094B303A0009EA
:10AAB000094D303A0009094E303A00090949303A47
:10AAC00000090945303A00090957303A0009094F91
:10AAD000303A0009257320256500094E313A0009F6
:10AAE00025732025362E336600090946313A0009C0
:10AAF00025732025362E306600090946783A00096C
:10AB0000202046314F46465345543A0009257320CC
:10AB100025362E33662025362E33662025362E33F5
:10AB2000662025362E33660D0A09090920202020CB
:10AB30000025662025662025662025660009202040
:10AB400046324F46465345543A0009257320257333
:10AB500009092020200009257320257309090920EF
:10AB60002020000D0A0D0A093D3D3D3D3D3D3D20A3
:10AB7000436F6E66696775726174696F6E204D65AB
:06AB80006E7520203D3D32
:10AB86003D3D3D3D0D0A0009302E20446973706C31
:10AB9600617920616C6C20636F6E6669677572659A
:10ABA600642076616C7565730D0A0009312E2043A9
:10ABB600616C6962726174696F6E206F6620616E86
:10ABC60074656E6E61207370616E2076616C75655A
:10ABD6000D0A0009322E2053657420414443207328
:10ABE60070616E2076616C75650D0A0009332E2042
:10ABF60053657420446561642042616E6420616E11
:10AC06006420536B65772076616C75650D0A0009C3
:10AC1600342E2053657420616E74656E6E6120500B
:10AC260061726B696E6720616E64204C696D697430
:10AC360020706F736974696F6E0D0A0009352E20D6
:10AC46004D6F6E69746F72204144432076616C7556
:10AC560065202620416E74656E6E6120706F736983
:10AC660074696F6E0D0A0009362E20446972656399
:10AC76007420616E74656E6E6120636F6E74726FA0
:10AC86006C0D0A0009372E20526164696F2043411A
:10AC96005420706F727420636F6E66696775726197
:10ACA60074696F6E0D0A0009382E204D69632D6395
:10ACB6006C69636B20636F6E666967757261746930
:10ACC6006F6E0D0A0009392E20536574206465667F
:10ACD60061756C7420706172616D657465720D0AC0
:10ACE6000D0A000D0A09436F6E6669677572652065
:10ACF600796F75722073746174696F6E20656C6507
:10AD06006D656E7473203F205B592F4E5D202000C9
:10AD16000D0A0A0943415420526967204B454E5794
:10AD26004F4F442C59414553552C49434F4D205BB9
:10AD36004B2F592F495D203F2020000D0A094973EA
:10AD46002074686520434154205249472054532DAE
:10AD560037313120262054532D38313120636F6D21
:10AD660062696E6174696F6E203F205B592F4E5D7C
:10AD760020000D0A092020596F75206D7573742007
:10AD860075736520616C7465726E61746520434FDE
:10AD96004D20706F727420666F722055706C696EEC
:10ADA6006B20545258000D0A092020416C746572BC
:10ADB6006E61746520434F4D20706F727420697305
:10ADC60020383033312050312E352F434E332D3637
:10ADD60020000D0A0953656C65637420545258208F
:10ADE600313A46542D3733362020323A46542D38E0
:10ADF60034372020333A4F746865722020000D0ADC
:10AE06000953656C65637420464D4E206D6F64650D
:10AE1600203F205B592F4E5D20000D0A09456E74B8
:10AE260065722064657374696E6174696F6E204122
:10AE360064647265737320666F72205258202825E9
:10AE460042582920002568780009456E74657220ED
:10AE560064657374696E6174696F6E2041646472AF
:10AE660065737320666F722054582028254258292E
:10AE760020000953657061726174656420545258EC
:10AE8600203F205B592F4E5D2020000D0A09576197
:10AE960069742074696D6520666F7220636F6D6DCD
:10AEA600616E64205B25645D2000205B312D3235A8
:10AEB600355D20000D0A09506F7274206261756459
:10AEC6002072617465203F205B313230302F32347E
:10AED60030302F343830302F393630302F31393248
:10AEE60030305D20000D0A0955706C696E6B204488
:10AEF6006F70706C657220636F7272656374696FD0
:10AF06006E203F205B592F4E5D2020000D0A09441C
:10AF16006F776E6C696E6B20446F70706C65722013
:10AF2600636F7272656374696F6E203F205B592F81
:10AF36004E2F525D2020000D0A0953656C6563741F
:10AF46002046756C6C206F72626974206F722041A6
:10AF56004F532043415420636F6E74726F6C203FD1
:06AF6600205B462F415D57
:10AF6C002020000D0A0D0A0D0A09203D3D3D3D3DF6
:10AF7C003D3D3D3D3D205265616C74696D652054CD
:10AF8C007261636B696E67205B2534642F253032E8
:10AF9C0062642F25303262645D203D3D3D3D3D3D78
:10AFAC003D3D3D0D0A000D0A2020274527546F67B3
:10AFBC00676C6520726F746F7220636F6E74726F42
:10AFCC006C2020275027546F67676C65207072695E
:10AFDC006F7269747920747261636B2027512752E8
:10AFEC00657475726E20746F206D61696E206D656D
:10AFFC006E750D0A0D0A00202048483A4D4D3A5303
:10B00C00532020202000252D3133730020202D20AB
:10B01C00202020202020202020000D0A000D0A0DC9
:10B02C000A09203D3D3D3D3D3D3D3D3D3D205265A8
:10B03C00616C74696D6520547261636B696E672015
:10B04C005B2534642F25303262642F2530326264E4
:10B05C005D203D3D3D3D3D3D3D3D3D0D0A000D0A14
:10B06C00202027452720546F67676C6520726F740A
:10B07C006F7220636F6E74726F6C202027592720BB
:10B08C00525443207A65726F2061646A7573742020
:10B09C00202751272052657475726E20746F206DB5
:10B0AC0061696E206D656E75000D0A202027492799
:10B0BC0020496E697469616C697A652074686520D1
:10B0CC00545258202020202754272054756E652078
:10B0DC00545258202020275350432F4253272020CE
:10B0EC004E6578742F50726576696F75732E207368
:10B0FC0061742E000D0A202027312F322F332F346C
:10B10C00272055706C696E6B206368616E6E656C80
:10B11C002020272B2F2D2F302720446F70706C652B
:10B12C007220636F6D70656E736174696F6E202031
:10B13C00273F27206F626A2E207361742E000D0A40
:10B14C002020274E2720547261636B206E65787423
:10B15C0020736174656C6C697465202027502720FE
:10B16C00546F67676C65207072696F7269747920AF
:10B17C00747261636B696E670D0A0020205B53610A
:10B18C0074656C6C6974653A20252D39735D200DDE
:10B19C000A0020202020205554432020202020412C
:10B1AC007A696D2E202020456C65762E2020205249
:10B1BC00616E6765202020202020416C742E202099
:10B1CC00204C61742E2020204C6F6E672E20205056
:10B1DC0068617365202020446F70706C65720D0A75
:10B1EC0000202048483A4D4D3A53532020206465A6
:10B1FC006720202020206465672020202020204B01
:10B20C006D20202020202020204B6D20202020206D
:10B21C0064656720202020206465672020203C3254
:10B22C0035363E202020202020487A0D0A000D0AB9
:10B23C000D0A092A2A2A202053656C656374206F35
:10B24C00626A65637420736174656C6C69746520E3
:10B25C00666F72204C434420646973706C61792072
:10B26C002831202D2025626429202A2A2A0D0A0043
:10B27C00070D0A094F7574206F66206E756D626537
:10B28C00722021202831202D2025642920202331D3
:10B29C00207761732073656C656374656420666FD9
:10B2AC0072204C434420646973706C61790D0A0000
:10B2BC0025632025303262643A25303262643A25A7
:10B2CC0030326264200025352E31662F252D362E26
:10B2DC00316625362E31662F252D362E31662536D4
:10B2EC002E31662F252D362E316625362E31662FC2
:10B2FC00252D362E31660025362E31662F252D361E
:10B30C002E31660D0025303262643A25303262648B
:10B31C003A25303262642563252D377300415A205B
:10B32C0025332E316620454C25322E3166202020C7
:10B33C0020000D0A25730D0A00256320253032628A
:06B34C00643A2530326274
:10B35200643A25303262640025382E326625382E52
:10B36200326625392E316625392E316625372E3142
:10B372006625382E316625372E3166252B362E303E
:10B3820066002F252D352E3066200D0025303262C5
:10B39200643A25303262643A25303262642563258C
:10B3A2002D35732020004125332E3066204525326D
:10B3B2002E3066205025332E316620202020004179
:10B3C2005A2025332E316620454C25322E316620F7
:10B3D2002020202000070D0A0D0A20205B507269F0
:10B3E2006F7220536174656C6C69746520252D3908
:10B3F2007320697320414F535D0D0A00515258204A
:10B40200466C697020636865636B2E2E00070D0A17
:10B4120009526F7461746F72204572726F7220618B
:10B42200742025303262643A25303262643A253023
:10B432003262640D0A09436865636B20616E6420A1
:10B44200706F776572206F6E207265736574206607
:10B452006F722073797374656D207265636F7665A0
:10B4620072792E0D0A00526F7461746F72204572E8
:10B47200726F7220212000436865636B20746865D7
:10B482002073797374656D000709457869742066C5
:10B49200726F6D204572726F72206D6F64652061EC
:10B4A200742025303262643A25303262643A2530A3
:10B4B2003262640D0A0A000D0A665F6C6F732F66B2
:10B4C2005F616F732F665F646966662F70756C7358
:10B4D200653A256C642F256C642F256C642F256CCE
:10B4E200640D0A0055502070756C73653A0044571C
:10B4F2004E2070756C73653A002A005F0046422543
:10B502003031316C753B00002530394C6400002528
:10B512003031306C7500004641253031316C753B5D
:10B5220000004443303B004443313B004D4425621C
:10B53200643B0000464E303B00464E313B00414FDB
:10B542002D30370000534F2D33330000464F2D323C
:10B552003900000D0A0D0A0009312E446972656333
:10B562007420726F746F7220636F6E74726F6C20CE
:10B5720066726F6D206B657920626F6172642E0D49
:10B582000A0009322E456E74657220646972656321
:10B5920074696F6E2076616C75652E0D0A00093331
:10B5A2002E50726573657420436F6E74726F6C2EC9
:10B5B2000D0A0D0A000D0953656C6563745B312D2C
:10B5C200332C515D3A20000D0A0D0A094C65667450
:10B5D2002834292C2052696768742836292C205572
:10B5E200702838292C2044776E2832292C20537455
:10B5F2006F70283529206F72205265742E0D0A0D46
:10B602000A000D0A0D0A09417A696D7574683A20BB
:10B6120025322E3166000D0A09456C657661746922
:10B622006F6E3A2025322E3166000D0A0D0A09315D
:10B632003A25352E31662F252D342E316620323AA9
:10B6420025352E31662F252D342E316620333A25AD
:10B65200352E31662F252D342E316620343A25358C
:10B662002E31662F252D342E31660020353A2535B0
:10B672002E31662F252D342E3166000D0A0D0A0952
:10B6820053656C6563745B312D352C532C515D3AD7
:10B6920020000D0A0950726573657420706F73691A
:10B6A20074696F6E2025642020417A3A25352E3147
:10B6B2006600092020202020202020202020202079
:10B6C200202020202020456C3A25352E31660009A5
:10B6D200415A3D253464202F2025332E316664657E
:10B6E2006709454C3D253464202F2025332E3166D1
:10B6F2006465672E202020200D000D0A0D0A0954D2
:10B70200686973206D656E7520636F6E6669677513
:10B71200726573204144432076616C756520666FC3
:10B722007220746865206D69632D636C69636B2098
:06B73200636F6E74726F7C
:10B738006C0D0A000D0A09536574206E6577207632
:10B74800616C7565206F72204D6561737572652037
:10B758004144432076616C7565203F205B532F4D33
:10B768005D2020000D0A094D6F64656D206C6F63C4
:10B778006B65642063656E7465722041444320766E
:10B78800616C756520203A2025346400095265668D
:10B798006572656E6365204144432076616C75650A
:10B7A8002020202020202020203A20253464000D4D
:10B7B8000A0954756E652052582066726571756560
:10B7C8006E637920746F206D6F64656D206C6F6394
:10B7D8006B656420706F736974696F6E205B592F95
:10B7E8004E5D20000D0A095075736820446F776E0E
:10B7F800206D69632D636C69636B20627574746F67
:10B808006E2074776F2074696D6573205B592F4EB5
:10B818005D2020000D0A09456E7465722053746519
:10B8280070206672657175656E6379205B487A5D14
:10B838003A00094672657175656E6379207365749F
:10B848002043415420636F6D6D616E6420617420E4
:10B85800414F53203F205B592F4E5D20000D0A09B0
:10B868004175746F6D617469632075702070756CB3
:10B8780073652067656E65726174696F6E206174A7
:10B8880020414F53203F205B592F4E5D20000D0A69
:10B8980009506F726C6172697479206F66207374D5
:10B8A80065702070756C73652C204E6F726D616CBD
:10B8B8002F52657665727365203F205B4E2F525D6F
:10B8C800200009094144432076616C7565203D25B7
:10B8D80034642F313032332020200D000D0A0D0A38
:10B8E8002020414443207370616E2076616C756539
:10B8F800202020415A3A2025303464202D2025303C
:10B9080034642020454C3A2025303464202D2025ED
:10B918003034640D0A000D0A202053657420666CCB
:10B928006970206D6F6465206F7065726174696FEE
:10B938006E20666F7220656C65766174696F6E2023
:10B94800726F746F72000D0A2020526F74617465F3
:10B958002074686520616E74656E6E6120746F2056
:10B9680066756C6C792043435720616E6420456C82
:10B9780065766174696F6E206D696E696D756D208D
:10B98800706F736974696F6E000D0A2020526F74AE
:10B998006174652074686520616E74656E6E6120DF
:10B9A800746F2066756C6C7920435720616E642033
:10B9B800456C65766174696F6E206D6178696D7527
:10B9C8006D20706F736974696F6E000D0A094144C8
:10B9D80043207370616E2076616C7565202020416C
:10B9E8005A3A2025303464202D2025303464200034
:10B9F8000D0A09415A206D696E696D756D20766171
:10BA08006C7565203F203A20000D09415A206D6170
:10BA180078696D756D2076616C7565203F203A20D8
:10BA2800000D0A0953657420666C6970206D6F6497
:10BA380065206F7065726174696F6E20666F722021
:10BA4800656C65766174696F6E20726F746F7200D1
:10BA58000D0A09414443207370616E2076616C754C
:10BA680065202020454C3A2025303464202D20259F
:10BA780030346420000D0A09454C206D696D696DEC
:10BA8800756D2076616C7565203F203A20000D09A0
:10BA9800454C206D6178696D756D2076616C7565B2
:10BAA800203F203A20000D0A0D0A095365742041F1
:10BAB8006E74656E6E61205061726B696E6720707E
:10BAC8006F736974696F6E203F205B592F4E5D203C
:10BAD80020000D0A0D0A09417A696D7574682020E5
:10BAE8005061726B696E67202076616C7565203ACB
:10BAF8002025332E31660009456C65766174696FBF
:10BB08006E205061726B696E672076616C75652076
:06BB18003A2025332E3116
:10BB1E0066000D0A0953657420545258206D6F64E7
:10BB2E00652F667265712E20696E207061726B6969
:10BB3E006E67203F205B592F4E5D2020000D0A09B5
:10BB4E005258207061726B696E6720667265712043
:10BB5E003A2025362E336600095458207061726BD8
:10BB6E00696E672066726571203A2025362E33661F
:10BB7E0000095258207061726B696E67206D6F6498
:10BB8E00652028464D2F5553422F4C534229203ABB
:10BB9E002000095458207061726B696E67206D6FBA
:10BBAE0064652028464D2F5553422F4C5342292071
:10BBBE003A20000D0A0953657420416E74656E6E4D
:10BBCE006120726F746174696F6E206C696D697437
:10BBDE00203F205B592F4E5D2020000D0A0D0A09D3
:10BBEE00417A696D7574682020206D696E6D756D72
:10BBFE00202076616C7565203A2025332E31660043
:10BC0E0009417A696D75746820206D6178696D756A
:10BC1E006D202076616C7565203A2025332E3166B5
:10BC2E000009456C65766174696F6E20206D696ED2
:10BC3E006D756D2076616C7565203A2025332E3139
:10BC4E00660009456C65766174696F6E206D61786A
:10BC5E00696D756D2076616C7565203A2025332EE1
:10BC6E003166000D0A0953657420726F7461746F2A
:10BC7E007220736D6F6B652070726F74656374697B
:10BC8E006F6E203F205B592F4E5D2020000D0A095C
:10BC9E0054696D656F75742076616C756520666F7D
:10BCAE007220726F7461746F72206572726F72207F
:10BCBE005B7365635D203A20253364000D0A0941EC
:10BCCE0075746F207265636F766572792074696D15
:10BCDE00652066726F6D20726F7461746F7220656D
:10BCEE0072726F72205B312D36316D696E5D203A46
:10BCFE0020253364000D0A0D0A09417A696D7574A9
:10BD0E0068202020446561642042616E6420203AE0
:10BD1E002025322E31660009456C65766174696F97
:10BD2E006E20446561642042616E6420203A2025B5
:10BD3E00322E3166000D0A09417A696D75746820DC
:10BD4E002020536B65772076616C7565203A20252F
:10BD5E00322E31660009456C65766174696F6E200E
:10BD6E00536B65772076616C7565203A2025322EEF
:10BD7E003166004B454E574F4F4400594145535580
:10BD8E0020200049434F4D20006E6F6E65004C53CE
:10BD9E00420055534200435700464D00414F530059
:10BDAE0046756C6C000943616C6C7369676E3A2062
:10BDBE00257320204C61743A2025352E31662020C3
:10BDCE004C6F6E673A2025352E3166202048656906
:10BDDE006768743A2025352E31660D0A00094144F4
:10BDEE0043207370616E2076616C75652020202073
:10BDFE00415A3A20253564202D20253564202045D2
:10BE0E004C3A20253564202D202535642000284607
:10BE1E006C6970290009446561642062616E64205A
:10BE2E002020202020202020415A3A2025352E3156
:10BE3E006620202020202020202020454C3A20253E
:10BE4E00352E3166200D0A0009536B6577202020B0
:10BE5E002020202020202020202020415A3A20255A
:10BE6E00352E316620202020202020202020454CF9
:10BE7E003A2025352E3166200D0A0009416E746573
:10BE8E006E6E61207061726B696E67202020415A60
:10BE9E003A2025352E3166202020202020202020FB
:10BEAE0020454C3A2025352E3166200D0A000954C6
:10BEBE005258207061726B696E6720202052583A7A
:10BECE0025362E33662054583A25362E33662020DA
:10BEDE0020205258206D6F64653A257320545820E7
:10BEEE006D6F64653A25730D0A000954525820206F
:06BEFE007061726B696EB9
:10BF0400672020202020204F66660D0A0009416E1C
:10BF140074656E6E61207061726B696E672020209B
:10BF24004F66660D0A0009526F7461746F72206C5B
:10BF3400696D69742020202020415A3A2025352E2D
:10BF44003166202D2025352E31662020454C3A209F
:10BF540025352E3166202D2025352E3166200D0AFB
:10BF64000009526F7461746F72206C696D6974207A
:10BF7400202020204F66660D0A0009526F746174F8
:10BF84006F7220737461727420454C3A25352E31DA
:10BF94006620202050312E365F6F6E20454C3A25A6
:10BFA400352E316620202050312E365F6F66662094
:10BFB400454C3A25352E3166200D0A0009526F741E
:10BFC4006F7220736D6F6B652070726F746563742C
:10BFD400696F6E094F66660D0A000954696D656FD5
:10BFE40075742076616C756520666F7220726F744B
:10BFF40061746F72206572726F723A202533642007
:10C004007365630D0A00094175746F207265636F6F
:10C01400766572792074696D652066726F6D207221
:10C024006F7461746F72206572726F723A20253377
:10C0340064206D696E0D0A000943415420526967FA
:10C04400202020202020202020202025732025733C
:10C0540000202054533731312F383131002020460D
:10C06400542D37333600202046542D383437002FD2
:10C07400464D4E2D46696C74657200202028254279
:10C084005829282542582928773D25642900202548
:10C0940073000D0A095374657020636F6E74726FB8
:10C0A4006C204144432076616C7565202043656EA5
:10C0B4007465723A2535642020526566663A2535E2
:10C0C40064000D0A094672657175656E63792073A3
:10C0D40074657020202020256C64487A000D0A09BC
:10C0E400526F746F72207374617274202020202048
:10C0F40020202573000D0A09434F4D20706F727480
:10C10400202020202020202020202573204261751B
:10C114006420382D4E2D310D0A000D0A0909507284
:10C1240065737320616E79206B657920746F206369
:10C134006F6E74696E7565000D0A2534642F2530A1
:10C144003262642F25303262642025303262643AD0
:10C1540025303262643A25303262640D0A00537429
:10C16400617274696E67204461792F54696D65202A
:10C174003F205B59592F4D4D2F44442048483A4D98
:10C184004D3A53535D2000446179206F66207468F2
:10C19400652059656172205B545D203E2025352E53
:10C1A40035660D0A0054696D6520537465700D0A77
:10C1B40000094D696E205B315D3A200009536563C7
:10C1C400205B305D3A20002020253573202020207C
:10C1D4002535732020202020202025337320202F74
:10C1E4002533732020202020253573253130730D0D
:10C1F4000A00444154450054494D4500415A004504
:10C204004C00506861736500446F70706C65720017
:10C214002534642F25303262642F25303262642045
:10C2240025303262643A25303262643A2530326213
:10C23400642020202025352E31662F25342E3166AA
:10C2440025392E3166252B392E30660D0A002A2A0F
:10C254002A2A2A2A2A2A2A2A0A0D00092D2D2D20C3
:10C2640027512720666F722061626F7274202753F2
:10C274002720666F72207363726F6C6C202D2D2DD6
:10C28400000D0A0A0955706C6F6164204B65706576
:10C294006C6520646174612066696C652E20284594
:10C2A4004F463A6374726C2B5A290D0A00070D0A23
:10C2B400095253204275666665722046756C6C207F
:10C2C400210D0A004E4153413E2325336409257351
:10C2D4000D0A000D0A09536174656C6C697465205C
:06C2E400282573292073D8
:10C2EA00656C656374656420617320232562640D3F
:10C2FA000A002532642E2A252D3134732000253276
:10C30A00642E20252D31347320000D0A0953656CE3
:10C31A006563743A002532642E2563252D31347302
:10C32A00200020202020202020000D0A0907536128
:10C33A0074656C6C697465206973206E6F74206112
:10C34A007369676E65642E20476F20746F206D6570
:10C35A006E7520332D320D0A002000000D0A0A09DD
:10C36A0055706C6F616420667265712F6D6F6465BC
:10C37A0020646174612066696C652E2028454F46E9
:10C38A003A6374726C2B5A290D0A0025732025739F
:10C39A0020257320257320257320257320257320DB
:10C3AA00257300536174656C6C697465202825389F
:10C3BA007329207570646174656420616E642073EA
:10C3CA00656C656374656420617320232532626439
:10C3DA000D0A000D0A0D0A0955706C6F616420532D
:10C3EA00746174696F6E20696E666F2E2064617461
:10C3FA00612066696C652E2028454F463A6374723F
:10C40A006C2B5A290D0A00252A63202573202566DC
:10C41A0020256620256620257300252A63202564A9
:10C42A0020256420256420256420257300252A639D
:10C43A0020256620256620256620256600252A6394
:10C44A0020257320257320256878202568782025E3
:10C45A006420256400252A6320257320256620256B
:10C46A006620256620256620256600252A63202564
:10C47A0073202566202566202573202573202564D0
:10C48A0020256400252A6320257320256620256639
:10C49A00202566202566000D0A0953746174696FA8
:10C4AA006E20696E666F726D6174696F6E20757049
:10C4BA0064617465642E0D0A00070D0A09457272DB
:10C4CA006F72202120757064617465206E6F74200C
:10C4DA00636F6D706C657465642E0D0A000D0A0D2C
:10C4EA000A5472616B426F7820686F7374206D6FA3
:10C4FA0064652E000D0A436F6D6D616E643A4D5589
:10C50A007878782C4D447878782C46557878782C39
:10C51A0046447878782C415A7878785F454C787810
:10C52A002C537878782C5478782C512C3F412C3F16
:10C53A000D0A005472616B426F7820486F73746DF4
:10C54A006F64650000202020202020202020202049
:10C55A00202020202000000D0A5472616B426F785F
:10C56A003E3E200025732025730046555F2020207B
:10C57A0020202020202020202020000046445F2068
:10C58A002020202020202020202020200000467269
:10C59A0065712E20666F726D6174206572726F729A
:10C5AA002021202865782E204655313435393030FF
:10C5BA003030290D0A00465F666F726D617420651E
:10C5CA0072726F722000004D6F6465206572726F1F
:10C5DA0072202020202000004D6F64652065727251
:10C5EA006F72202865782E204D554C2F4D55552FAA
:10C5FA004D5546290D0A004D6F6465206572726FAC
:10C60A0072202865782E204D444C2F4D44552F4DCD
:10C61A004446290D0A004D6F646520466F726D61AC
:10C62A0074206572726F72202865782E204D554CE1
:10C63A0053422C4D44464D290D0A004D5F666F72D8
:10C64A006D6174206572726F72200000417A2F4505
:10C65A006C20666F726D6174206572726F72202829
:10C66A0065782E20417A30373520456C3135290DD1
:10C67A000A00415A5F666F726D6174206572726F4B
:10C68A0072200000547261636B2023204572726F1E
:10C69A007220210D0A000D0A436F6D6D616E643AB6
:10C6AA004D557878782C4D447878782C465578789A
:10C6BA00782C46447878782C415A7878785F454CBB
:06C6CA0078782C5378780B
:10C6D000782C5478782C3F412C3F2C510D0A004384
:10C6E0006F6D6D616E64206572726F72200D0A004D
:10C6F000436F6D6D616E64206572726F72202020D1
:10C700000000FF9FD4FFA006FFA032FFA05EFFA0A5
:10C710008AFFA09CFFA0AEFFA5ACFFA5B2FFA5B805
:10C72000FFA5BDFFA5C2FFA5C7FFA5CCFFA5D1FFF3
:10C73000A5D7FFA5E9FFA5FBFFA60DFFA61FFFA636
:10C7400031FFA893FFA898FFA8A3FFA8A6FFA8AA57
:10C75000FFA8BEFFA8D2FFA8E6FFA8FAFFA90EFF18
:10C76000A922FFA936FFA94AFFA95EFFA972FFA966
:10C7700086FFA99AFFA9AEFFA9C2FFA9D6FFA9EA21
:10C78000FFA9FEFFAA12FFAA26FFAA3AFFAA3FFFAF
:10C79000AA44FFAA49FFAA4EFFBD81FFBD89FFBD84
:10C7A00091FFA5ACFFA5B2FFBD97FFBD9CFFBDA04B
:10C7B000FFBDA4FFBDA7FFBDAAFFBDAEFFA5B8FF8B
:0EC7C000A5BDFFA5C2FFA5C7FFA5CCFFA5D153
:10C7CE0046002240D0E8F4FAFD45002840A0D0E80B
:10C7DE00F45A002F001F1C1F1E1F1E1F1F1E1F1E80
:10C7EE001F001F1D1F1E1F1E1F1F1E1F1E1F6078D6
:10C7FE0000493E8D06BC3E8CAFD53E8DBFCF3E8DE3
:10C80E0068E83E8D12023E8CBB1B3E8DCB143E8DD6
:10C81E00742E3E8D1D263E8CC63F3E8DD6393E8DE6
:10C82E007F523E8D286B3E8CD1853E8DE17E3E8DB6
:10C83E008A983E8D33B13E8CDCCA3E8DECA23E8D85
:10C84E0095BC3E8D3ED53E8CE7EF3E8DF7E83E8D96
:10C85E00A1013E8D4A1B3E8CF3343E8E032E3E8D3F
:0AC86E00AC263E8D553F3E8CFE586F
:10000300E4F5081201EF78857C677D017BFF7AA018
:1000130079C012D47AEF600F1202CA1201EF7BFF8C
:100023007AA079C6120A4E900007E030E30990E106
:1000330002E04450F0800790E102E054AFF07F30DB
:100043007E7512081A90C70E12D2931208957FC0BC
:100053001202A090C71412D29312089512083A7F85
:10006300007E007DC67C439065CE12D1DE12CBEEBE
:10007300600B40097BFF7AA079D8120877120850E9
:100083008F09E5096064900004E04401F0A3E0F007
:100093007BFF7AA079F012087790677912D2060075
:1000A30000000090E102E054F0F01208508F09E5DF
:1000B3000914FF906777F03395E0FE742D2FF582D6
:1000C300EE3417F583E0C3648094804004E509703F
:1000D300071208508F0980C1900004E0A330E105A6
:1000E3001223F380B412290A80AF900004E054FE77
:1000F300F012083A90E102E054F0F090677912D2DE
:100103000600000000900004E054FDF0900006E0BB
:100113004404F0A3E0F0900004E0A330E405750884
:10012300078005120AD08F08E50812D29F015201F9
:1001330001860201BA0301C00401C60501CC060110
:10014300D20701D80801DE6D015273000000F47B71
:10015300FF7AA079F41208771286E78E0A8F0BE5EF
:100163000BF47003E50AF46088906776E0FFC3E55B
:100173000B9F7480F8650A9840030200F412290A61
:100183000200F47BFF7AA1791D1208771286E78EAD
:100193000A8F0BE50BF47003E50AF470030200F415
:1001A300742D250BF582E43417F583E0FF3395E0D6
:1001B300FE1275A20200F4120C110200F4120DEDEE
:1001C3000200F41211320200F4121F410200F41271
:1001D30098CC0200F4125DAE0200F4900004E044F7
:0C01E30002F0A3E0F01223F30200F4226B
:1001EF0090E2017402F090E1037482F090E100E478
:1001FF00F0759852758922758850758780C28CC2A8
:10020F008EA3E020E705758DE8802890002DE0FF94
:10021F00C394004006EFD39405400B90002D740457
:10022F00F0758DFA800D74222FF582E43400F5837A
:10023F00E0F58D90002EE02428F582E43400F5835C
:10024F00E0F58CD28CD28E90E00FE0540464046001
:10025F001F7BFF7AA1794612087790E00F7407F0A1
:10026F007404F090E00DE054FEF090E00F7404F091
:10027F007F381202A07F381202A07F0C1202A07FDB
:10028F00061202A07F011202A090E00DE054FBF0D5
:01029F00223C
:1002A000C292C29190E100EFF07F0A7E0012081A1C
:0502B000D290C2902273
:1002B500D292C29190E100EFF07F0A7E0012081AF7
:0502C500D290C290225E
:1002CA007BFF7AA17948120877120583125AB0780F
:1002DA006A7C177D017BFF7AA1797F7E007F0712F6
:1002EA00CFF378857C677D017BFF7AA179877E00D1
:1002FA007F0612CFF390E101E020E705758DE880D3
:10030A000690002D7404F090002E7402F090E00F15
:10031A007407F07404F090E00DE054FEF090E00FE2
:10032A007404F090000A12D20641DB20C590000E38
:10033A0012D2064300A8317F007E007D007C009027
:10034A00000E12D1DE12CBEE600250197F007E0041
:10035A007D807CBF90000E12D1DE12CA4C90001232
:10036A0012D1FA801790000E12D1DE7F007E007D36
:10037A00B47C4312C95790001212D1FA9000161297
:10038A00D206424800009065EE12D2060000000034
:10039A009065F212D206000000009065F612D206AD
:1003AA00404000009065FA12D2063F800000906536
:1003BA00E6E4F0A37403F0A3F0A37445F0A3E4F019
:1003CA00A304F0A3F0A374CCF090660A12D206003C
:1003DA0000000090660E12D20600000000906649E6
:1003EA0012D2060000000090664512D206000000F4
:1003FA00009066587404F0906657F0906656F09034
:10040A006655F090661212D2060000000090661639
:10041A0012D20643B4000090661A12D206000000F7
:10042A000090661E12D20642B4000090662612D2CE
:10043A0006C000000090662A12D206C0A0000090F2
:10044A00662E12D206C0E00000E4906777F0A3742B
:10045A0003F090664112D206000000009066511225
:10046A00D2060000000AE4906632F0906635742ED7
:10047A00F0906637F0906636F0906638F090663302
:10048A00F0A3741EF0900000E4F0A37432F09067B9
:10049A008112D2060000006490001A7401F0A304CD
:1004AA00F0A3F0A37426F0A37402F0A37430F090C2
:1004BA006771E4F0A37478F0A3E4F0A3743DF090BC
:1004CA0000047468F0A37440F0A3740DF0A374835D
:0C04DA00F0900009E04402F01204E62259
:1004E6009065E6E0FEA3E0FFC39065E9E09FFF901C
:1004F60065E8E09EFE12E917AC06AD07EC12CC717A
:100506007B007A0079B4784312CB559065E212D11C
:10051600FA900006E0A330E6329065EAE0FEA3E03A
:10052600FFC39065EDE09FFF9065ECE09EFE12E94B
:1005360017AC06AD07EC12CC717B007A00793478E3
:100546004312CB559065DE12D1FA229065EAE0FEA1
:10055600A3E0FFC39065EDE09FFF9065ECE09EFE93
:1005660012E917AC06AD07EC12CC717B007A007964
:0D057600B4784212CB559065DE12D1FA2206
:10058300E4F50CE50CC3943C4003020798E50C2505
:10059300E025E0245DF582E43414F58312D20600ED
:1005A300000000E50C25E025E0246DF582E434131A
:1005B300F58312D20600000000E50C25E025E024B7
:1005C3004DF582E43415F58312D206000000007560
:1005D300F010E50C900F7D12D23712D20600000006
:1005E3000075F010E50C900F7912D23712D2060085
:1005F30000000075F010E50C900F7512D23712D27F
:10060300060000000075F010E50C900F7112D23750
:1006130012D206000000007431250CF582E4341375
:10062300F583E4F0E50C25E025E02481F582E4344C
:100633000EF58312D20600000000E50C25E025E04C
:100643002491F582E4340DF58312D20600000000F4
:10065300E50C25E025E024A1F582E4340CF58312B2
:10066300D20600000000E50C25E025E024B1F58268
:10067300E4340BF58312D20600000000E50C25E0FC
:1006830025E024D1F582E43409F58312D206000073
:100693000000E50C25E025E024E1F582E43408F5CB
:1006A3008312D20600000000E50C25E025E024F1CA
:1006B300F582E43407F58312D20600000000E50C4E
:1006C30025E025E02401F582E43407F58312D20600
:1006D30000000000E50C25E02499F582E43405F5DB
:1006E30083E4F0A3F0E50C25E025E02411F582E492
:1006F3003406F58312D2063F800000E50C25E02581
:10070300E024C1F582E4340AF58312D20600000026
:10071300017479250CF582E43416F583E4F0743D15
:10072300250CF582E43416F583E4F0E50C25E0248A
:10073300B6F582E43416F583E054FBF0E50C25E0CE
:1007430024B6F582E43416F583E054FEF0E50C2577
:10075300E024B6F582E43416F583E054FDF0E50CAD
:1007630025E024B6F582E43416F583E054EFF07EF9
:10077300007F14C006C0077D00E50C75F014A424A7
:10078300E9F9740035F0FA7B01D007D00612D58061
:10079300050C020586E4900020F0A3F0F50CE50CAF
:1007A300C3943C5012742D250CF582E43417F58361
:1007B30074FFF0050C80E7E4F50CE50CC3940550D9
:1007C30030E50C25E025E024D5F582E43400F583FB
:1007D30012D20600000000E50C25E025E024C1F557
:1007E30082E43400F58312D20600000000050C8079
:0207F300C92219
:1007F500900020E0FEA3E0FFC3EF9420EE944E505E
:1008050013747E2FF582EE3417F583E4F00FEF7045
:05081500010E80E42249
:10081A00E4F522F523EF2401FDE43EFCC3E5239D24
:10082A00E5229C500A0523E5237002052280E62270
:10083A001241D390676512D1C290676D12D1FA90B6
:06084A00676912D1FA22D9
:10085000900006E0A320E40990E101E0F4540FFFCA
:10086000227F02120A8AE529AE287806CEC313CE6B
:0708700013D8F9540FFF2219
:100877008B0C8A0D890E780CE475F00112D24312A5
:0E088700D01CF50F6007AF0F12E8BF80E9220A
:100895008B0C8A0D890E780CE475F00112D2431287
:0E08A500D01CF50F6007AF0F1202B580E922DC
:1008B3008B0C8A0D890E780CE475F00112D2431269
:1008C300D01CF50F6009AF0FE4FD12C87980E72251
:1008D30090690412D28A906904E475F00112D25C23
:0F08E30012D01CF5246007AF2412C8D980E82278
:1008F20090690812D28AE490690BF0A3F012E8E63C
:10090200EF640D604CEF640A6047EF6408600EEF1D
:10091200B47F2490690BE07002A3E0601A9069082A
:1009220074FFF5F012D25CE412D06290690B74FF8E
:10093200F5F012D0BE80C6906908E475F00112D2BB
:100942005CEF12D06290690BE475F00112D0BE80A8
:10095200AC906908E475F00112D25CE412D06290A6
:08096200690BE0FEA3E0FF2297
:10096A001208777B017A6879331208F2906830129C
:10097A00D253E4F5F012D0EA7B017A68793312E9AE
:10098A00D490683012D253EE8FF012D0EA7B017AFB
:07099A0068793312EB132210
:1009A1001208777B017A6879B81208F29068B5125B
:1009B100D253E4F5F012D0EA7B017A6879B812E9F2
:1009C100D49068B512D253EE8FF012D0EA7B017A3F
:0709D1006879B812DE8122F3
:1009D8001208777BFF7AA1798E12087712E8E6AEC3
:1009E80007EE4420FDB479037F0122EDB46E037F46
:0509F80000227FFF2238
:1009FD0090E00DE04401F0E030E11090E00DE054A6
:0C0A0D00FEF07F0A7E0012081A80E5222D
:100A19001209FDE4FFEFC3940C501FEFFDC3740BE3
:100A29009DFD74E09400FC8D82F583E0540F443001
:100A3900FE74352FF8A6060F80DBE4F54190E00D32
:050A4900E054FEF02264
:100A4E008B0C8A0D890E7F10E4FEFDEDC3940C50C5
:100A5E002AAB0CAA0DA90E8F8275830012D03524F5
:100A6E00D0FCE42DF582E434E0F583ECF01F0EEEBD
:0C0A7E00C3940240031FE4FE0D80D02250
:100A8A00EF540790E200F07F1E7E0012081AA3E0DE
:100A9A00FF90E200E0FDEF7F00FEEDFFE4EF780655
:100AAA00CEC313CE13D8F9FFEE5403F5288F2922AB
:100ABA007BFF7AA1799812087730980412E8E62227
:060ACA0012616480F422B9
:100AD00090C70212D29312087790C70512D29312D0
:100AE000087790C70812D29312087790C70B12D2DA
:100AF000931208777F801202A090C70E12D2931231
:100B000008957FC01202A090C71112D293120895C7
:100B10007BFF7AA179CA1208777BFF7AA179EA1262
:100B200008777BFF7AA279031208777BFF7AA27994
:100B30001B1208777BFF7AA2793C1208777BFF7A39
:100B4000A2795B1208777BFF7AA279781208777B0B
:100B5000FF7AA2798D1208777BFF7AA2799E12081C
:100B6000777BFF7AA279BE12087730983012E8E6D8
:100B7000AE07EEC39430400BEED394385005EE240C
:100B8000D0FF22EE4420FDB473037F7322EDB46DD9
:100B9000037F6D227BFF7AA279BE12087790000452
:100BA000E0FEA3E0FF30E4C230E2BF7F01129EBC52
:030BB00080B822E8
:100BB3007BFF7AA279D31208777BFF7AA279FC12A2
:100BC30008777BFF7AA379301208777BFF7AA379C2
:100BD300631208777BFF7AA379981208777BFF7AF1
:100BE300A379BB1208777BFF7AA379F612087712F1
:100BF300E8E6AE07EEC39431400BEED394355005CF
:0E0C0300EE24D0FF22EE4420B471DB7F71227C
:100C1100120BB39067D8EFF024FE604C14700302FE
:100C21000D29147003020D29147003020DA62494DA
:100C31007003020DEC247070D77BFF7AA479021245
:100C410008771286E79067D5EFF0F460C3E0FF33D1
:100C510095E0FE742D2FF582EE3417F583E0FF3316
:100C610095E0FE12125E80A87BFF7AA47929120911
:100C7100D89067D6EFF0D3648094804093E4906776
:100C8100D7F09067D7E0FFC3943C5018EF25E024DC
:100C9100B6F582E43416F583E054EFF09067D7E0BF
:100CA10004F080DE7BFF7AA479581208777BFF7A03
:100CB100A479841208777BFF7AA479B81208777B2C
:100CC100FF7AA379F612087712E8E6EF24CE6010D6
:100CD10014604F24026003020C111284D4020C111F
:100CE100E49067D7F0906775E0FF9067D7E0C39F06
:100CF100502AE0FF242DF582E43417F583EFF0EF5D
:100D010025E024B6F582E43416F583E04410F09032
:100D110067D7E004F0E0906776F080C91288650239
:100D21000C111288F4020C119067D8E0B403217BF6
:100D3100FF7AA479E61209D89067D6EFF0D36480E0
:100D410094805003020C11E4900020F0A3F0801C69
:100D51009067D8E0B40415906775E0C3943C400CEB
:100D61007BFF7AA5791D120877020C117BFF7AA50A
:100D7100793812087712E8E6E49067D7F09067D7E0
:100D8100E0FFC3943C5018EF25E024B6F582E4342B
:100D910016F583E054EFF09067D7E004F080DE129F
:100DA1007DA6020C117B017A6779D990683012D245
:100DB1008A7BFF7AA5795412096A9067D8EFF0C34C
:100DC10094024011E0FFD39405500A906775E0FE4C
:100DD100EFD39E400B7BFF7AA5799912087780C5E6
:0C0DE1009067D8E0906778F0020C1122B7
:100DED0078E87C677D017BFF7AC779177E007F06E7
:100DFD0012CFF378EE7C677D017BFF7AC7791D7E7C
:100E0D00007F1212CFF378007C687D017BFF7AC7DB
:100E1D00792F7E007F1212CFF37BFF7AA6794312D2
:100E2D0008777BFF7AA6796D1208777BFF7AA67912
:100E3D009F1208777BFF7AA379F612087712E8E6FE
:100E4D009067D7EFF06431600DE0FF64326007EF1B
:100E5D004420B471DF229067D7E0B4320412904F72
:100E6D00229067D7E0643160030211317F1A12E8D6
:100E7D00BF7BFF7AA679D212087790680012D25301
:100E8D0090679212D28A7B017A17796A90679512D0
:100E9D00D28A7BFF7AA679FF12D7537B017A6779C5
:100EAD00D81208F2EF4E600F786A7C177D017B0136
:100EBD007A6779D812D56390680312D253906792EE
:100ECD0012D28A90000A12D1C290679512D1FA7B84
:100EDD00FF7AA7790A12D7537B017A6779D5906883
:100EED00B512D28A7BFF7AA779181209A19067E211
:100EFD0012D1FA9067D5E07002A3E0600C9067E222
:100F0D0012D1C290000A12D1FA90680612D25390F3
:100F1D00679212D28A90000E12D1C290679512D1AB
:100F2D00FA7BFF7AA7790A12D7537B017A6779D5B5
:100F3D009068B512D28A7BFF7AA779181209A19011
:100F4D0067E212D1FA9067D5E07002A3E0600C90D1
:100F5D0067E212D1C290000E12D1FA7F007E007DA1
:100F6D00007C0090000E12D1DE12CBEE50197F00E6
:100F7D007E007D807CBF90000E12D1DE12CA4C9097
:100F8D00001212D1FA802A7F007E007D007C009035
:100F9D00000E12D1DE12CBEE401790000E12D1DEF4
:100FAD007F007E007DB47C4312C95790001212D190
:100FBD00FA90680912D25390679212D28A90001655
:100FCD0012D1C290679512D1FA7BFF7AA7791A12C6
:100FDD00D7537B017A6779D59068B512D28A7BFF9A
:100FED007AA779181209A19067E212D1FA9067D504
:100FFD00E07002A3E0600C9067E212D1C29000167F
:10100D0012D1FA900004E0FFA3E09067E6CFF0A3C1
:10101D00EFF090680C12D25390679212D28AE4FED0
:10102D009067E7E054087803CEC313CE13D8F99038
:10103D0067E875F00312D237EE75F003A42583F53A
:10104D008312D25390679512D28A7BFF7AA77927A4
:10105D0012D7537B017A6779D81208F29067D8E0DE
:10106D004420FFB46E09900005E04408F0800BEFBA
:10107D00B47307900005E054F7F09067D9E0442071
:10108D00B4610C900006E04410F0A3E0F0800790EE
:10109D000006E054EFF090680F12D2539067921251
:1010AD00D28A90002DE075F003A424EEF582E4348D
:1010BD0067F58312D25390679512D28A7BFF7AA778
:1010CD00793312D7537B017A6779D590683012D274
:1010DD008A7BFF7AA7791812096AEF8EF012D2C5B2
:1010ED001109012C110F04B011160960111D12C048
:1010FD0011242580112B4B0000001131E490002D9F
:10110D00F02290002D7401F02290002D7402F02237
:10111D0090002D7403F02290002D7404F0229000A5
:05112D002D7405F02205
:101132007BFF7AA7793D1208777BFF7AA779631242
:1011420008777BFF7AA779791208771241D37BFF60
:101152007AA779A51208777BFF7AA779B890679268
:10116200E52EF0A3E52FF0A3E530F0A3E531F0A3DF
:10117200E532F0A3E533F0A3E534F012D75330980B
:10118200CA12E8E69067F3EFF04420FFB4790890C2
:10119200E00DE04408F022EF6471700302125D1268
:1011A20041D37BFF7AA779DB1208777BFF7AA87994
:1011B20008906792E52EF0A3E52FF0A3E530F0A3A7
:1011C200E531F0A3E532F0A3E533F0A3E534F01204
:1011D200D7537BFF7AA8792C120877E49067DAF06C
:1011E2009067D7F07B017A6779D51208F29067DAB7
:1011F200E0FF9067D7E04F642F70549067E3E0FF01
:101202009067E0E04F643A704690E00F7407F07424
:1012120004F090E00DE054FEF090E00F7404F07BD7
:10122200017A6779D590679212D28A7BFF7AA87980
:101232005412D7537BFF7AA8796612087712E8E630
:101242009067F3EFF07B017A6779D5120A4E227B21
:0C125200FF7AA8797E1208771211322270
:10125E009067DBEEF0A3EFF0785B7C687D017BFF9F
:10126E007AC779417E007F0612CFF378617C687D64
:10127E00017BFF7AC779477E007F0612CFF378672E
:10128E007C687D017BFF7AC7794D7E007F3C12CF53
:10129E00F378A37C687D017BFF7AC779897E007F16
:1012AE000F12CFF37BFF7AAA7953120877906867F3
:1012BE0012D25390679212D28A9067DBE0FEA3E0BF
:1012CE00FF7C007D1412D07474E92FF974003EFA7D
:1012DE007B0190679512D28A7BFF7AAA797812D712
:1012EE00537B017A6879431208F2EF4E60249067BF
:1012FE00DBE0FEA3E0FF7C007D1412D07474E92FB6
:10130E00F974003EA801FC7D017B017A68794312D5
:10131E00D56390689112D25390679212D28A9067D9
:10132E00DCE025E0FF9067DBE033FE74992FF58259
:10133E00EE3405F583E0FFA3E0906795CFF0A3EFC1
:10134E00F07BFF7AAA798212D7537B017A6779DD17
:10135E009068B512D28A7BFF7AAA79891209A112F6
:10136E00CCAA9067DDE07002A3E06020AC06AD076A
:10137E009067DCE025E0FF9067DBE033FE74992F89
:10138E00F582EE3405F583ECF0A3EDF090686A1269
:10139E00D25390679212D28A9067DBE0FEA3E07878
:1013AE0002C333CE33CED8F92411F582EE3406F5CE
:1013BE008312D1C290679512D1FA7BFF7AAA7990E7
:1013CE0012D7537B017A6779DD9068B512D28A7B8A
:1013DE00FF7AAA799A1209A190685712D1FA9067EA
:1013EE00DDE07002A3E0603290685712D1C2C004F3
:1013FE00C005C006C0079067DBE0FEA3E07802C31D
:10140E0033CE33CED8F92411F582EE3406F583D0DF
:10141E0007D006D005D00412D1FA90686D12D253BF
:10142E0090679212D28A9067DBE0FEA3E07802C347
:10143E0033CE33CED8F924C1F582EE340AF58312B9
:10144E00D1C290679512D1FA7BFF7AAA79A012D7F2
:10145E00537B017A6779DD9068B512D28A7BFF7A69
:10146E00AA79A91209A190685712D1FA9067DDE006
:10147E007002A3E0603590685712D1C212CCAAC098
:10148E0004C005C006C0079067DBE0FEA3E078024B
:10149E00C333CE33CED8F924C1F582EE340AF583A8
:1014AE00D007D006D005D00412D1FA90687012D2AF
:1014BE005390679212D28A9067DBE0FEA3E0780227
:1014CE00C333CE33CED8F92401F582EE3407F5833B
:0F14DE0012D1C290679512D1FA7BFF7AAA79904A
:1014ED0012D7537B017A6779DD9068B512D28A7B6A
:1014FD00FF7AAA79AF1209A190685712D1FA9067B5
:10150D00DDE07002A3E0603290685712D1C2C004D2
:10151D00C005C006C0079067DBE0FEA3E07802C3FC
:10152D0033CE33CED8F92401F582EE3407F583D0CE
:10153D0007D006D005D00412D1FA90687312D25399
:10154D0090679212D28A9067DBE0FEA3E07802C327
:10155D0033CE33CED8F924F1F582EE3407F583126C
:10156D00D1C290679512D1FA7BFF7AAA799012D7E2
:10157D00537B017A6779DD9068B512D28A7BFF7A49
:10158D00AA79B51209A190685712D1FA9067DDE0DA
:10159D007002A3E0603290685712D1C2C004C0053A
:1015AD00C006C0079067DBE0FEA3E07802C333CE30
:1015BD0033CED8F924F1F582EE3407F583D007D078
:1015CD0006D005D00412D1FA90687612D2539067E6
:1015DD009212D28A9067DBE0FEA3E07802C333CE8D
:1015ED0033CED8F924E1F582EE3408F58312D1C259
:1015FD0090679512D1FA7BFF7AAA799012D7537B17
:10160D00017A6779DD9068B512D28A7BFF7AAA7963
:10161D00BB1209A190685712D1FA9067DDE07002F4
:10162D00A3E0603290685712D1C2C004C005C00655
:10163D00C0079067DBE0FEA3E07802C333CE33CE64
:10164D00D8F924E1F582EE3408F583D007D006D021
:10165D0005D00412D1FA90687912D2539067921284
:10166D00D28A9067DBE0FEA3E07802C333CE33CE9F
:10167D00D8F924D1F582EE3409F58312D1C29067E1
:10168D009512D1FA7BFF7AAA799012D7537B017A02
:10169D006779DD9068B512D28A7BFF7AAA79C1127B
:1016AD0009A190685712D1FA9067DDE07002A3E0AE
:1016BD00603290685712D1C2C004C005C006C00781
:1016CD009067DBE0FEA3E07802C333CE33CED8F9CA
:1016DD0024D1F582EE3409F583D007D006D005D09C
:1016ED000412D1FA90687C12D25390679212D28A6A
:1016FD009067DBE0FEA3E07802C333CE33CED8F99A
:10170D0024B1F582EE340BF58312D1C29067951298
:10171D00D1FA7BFF7AAA799012D7537B017A677938
:10172D00DD9068B512D28A7BFF7AAA79C71209A11A
:10173D0090685712D1FA9067DDE07002A3E0603235
:10174D0090685712D1C2C004C005C006C00790678B
:10175D00DBE0FEA3E07802C333CE33CED8F924B15B
:10176D00F582EE340BF583D007D006D005D00412E8
:10177D00D1FA90687F12D25390679212D28A9067F5
:10178D00DBE0FEA3E07802C333CE33CED8F924A13B
:10179D00F582EE340CF58312D1C290679512D1FA11
:1017AD007BFF7AAA799012D7537B017A6779DD9006
:1017BD0068B512D28A7BFF7AAA79CD1209A19068F9
:1017CD005712D1FA9067DDE07002A3E060329068A5
:1017DD005712D1C2C004C005C006C0079067DBE038
:1017ED00FEA3E07802C333CE33CED8F924A1F5821F
:1017FD00EE340CF583D007D006D005D00412D1FA03
:10180D0090688212D25390679212D28A9067DBE071
:10181D00FEA3E07802C333CE33CED8F92491F582FE
:10182D00EE340DF58312D1C290679512D1FA7BFF7C
:10183D007AAA79D312D7537B017A6779DD9068B58F
:10184D0012D28A7BFF7AAA79DA1209A1906857120F
:10185D00D1FA9067DDE07002A3E060329068571214
:10186D00D1C2C004C005C006C0079067DBE0FEA36F
:10187D00E07802C333CE33CED8F92491F582EE341D
:10188D000DF583D007D006D005D00412D1FA90689B
:10189D008512D25390679212D28A9067DBE0FEA335
:1018AD00E07802C333CE33CED8F92481F582EE34FD
:1018BD000EF58312D1C290679512D1FA7BFF7AAAE9
:1018CD0079DF12D7537B017A6779DD9068B512D233
:1018DD008A7BFF7AAA79E91209A190685712D1FA89
:1018ED009067DDE07002A3E0603290685712D1C2BC
:1018FD00C004C005C006C0079067DBE0FEA3E0781A
:10190D0002C333CE33CED8F92481F582EE340EF5F1
:10191D0083D007D006D005D00412D1FA9068A0125A
:10192D00D25390679212D28A9067DBE0FEA3E078E3
:10193D0002C333CE33CED8F9244DF582EE3415F5EE
:10194D008312D1C290679512D1FA7BFF7AAA79EFF3
:10195D0012D7537B017A6779DD9068B512D28A7BF5
:10196D00FF7AAA79F91209A190685712D1FA9067F6
:10197D00DDE07002A3E0603290685712D1C2C0045E
:10198D00C005C006C0079067DBE0FEA3E07802C388
:10199D0033CE33CED8F9244DF582EE3415F583D000
:1019AD0007D006D005D00412D1FA90689A12D253FE
:1019BD0090679212D28A9067DBE0FEA3E07802C3B3
:1019CD0033CE33CED8F9246DF582EE3413F5831270
:1019DD00D1C290679512D1FA7BFF7AAA79DF12D71F
:1019ED00537B017A6779DD9068B512D28A7BFF7AD5
:1019FD00AA79FF1209A190685712D1FA9067DDE01C
:101A0D007002A3E0603290685712D1C2C004C005C5
:101A1D00C006C0079067DBE0FEA3E07802C333CEBB
:101A2D0033CED8F9246DF582EE3413F583D007D07B
:101A3D0006D005D00412D1FA90688812D25390675F
:101A4D009212D28A9067DCE0C4F8540FC868FB90FC
:101A5D0067DBE0C454F048FA74712BF582EA340F59
:101A6D00F58312D1C290679512D1FA74752BF58258
:101A7D00EA340FF58312D1C290679912D1FA9067AB
:101A8D00DCE0C4F8540FC868FB9067DBE0C454F089
:101A9D0048FA74792BF582EA340FF58312D1C2908E
:101AAD00679D12D1FA747D2BF582EA340FF58312FE
:101ABD00D1C29067A112D1FA7BFF7AAB790C12D704
:101ACD00537B017A6779DF1208F2EF4E7003021B28
:101ADD007B7BFF7AAB79319067C212D28A9067DC3B
:101AED00E0C4F8540FC868FF9067DBE0C454F048B9
:101AFD00FE74712FF9740F3EFA7B019067C512D2F7
:101B0D008A9067DCE0C4F8540FC868FF9067DBE08B
:101B1D00C454F048FE74752FF9740F3EFA9067C8DF
:101B2D0012D28A9067DCE0C4F8540FC868FF906742
:101B3D00DBE0C454F048FE74792FF9740F3EFA902F
:101B4D0067CB12D28A9067DCE0C4F8540FC868FFE7
:101B5D009067DBE0C454F048FE747D2FF9740F3E9E
:101B6D00FA9067CE12D28A7A6779DF12DBE190683C
:101B7D009D12D25390679212D28A9067DBE0FEA33A
:101B8D00E07802C333CE33CED8F9245DF582EE343E
:101B9D0014F58312D1C290679512D1FA7BFF7AAA00
:101BAD0079DF12D7537B017A6779DD9068B512D250
:101BBD008A7BFF7AAB793D1209A190685712D1FA51
:101BCD009067DDE07002A3E0603290685712D1C2D9
:101BDD00C004C005C006C0079067DBE0FEA3E07837
:101BED0002C333CE33CED8F9245DF582EE3414F52D
:101BFD0083D007D006D005D00412D1FA90688B128D
:101C0D00D25390679212D28A9067DCE02479F582E4
:101C1D00E43416F583E075F003A424A3F582E434CF
:101C2D0068F58312D25390679512D28A7BFF7AABF7
:101C3D00794A12D7537B017A6879431208F2EF4E35
:101C4D006071906843E04420249D603424FD60421F
:101C5D0024F8605024F96016240970579067DCE071
:101C6D002479F582E43416F5837401F0804590678C
:101C7D00DCE02479F582E43416F5837402F08033C8
:101C8D009067DCE02479F582E43416F5837403F073
:101C9D0080219067DCE02479F582E43416F58374B5
:101CAD0004F0800F9067DCE02479F582E43416F5BA
:101CBD0083E4F090688E12D25390679212D28A907C
:101CCD0067DCE0243DF582E43416F583E075F0031E
:101CDD00A424A3F582E43468F58312D2539067955A
:101CED0012D28A7BFF7AAB794A12D7537B017A687D
:101CFD0079431208F2EF4E6071906843E04420245E
:101D0D009D603424FD604224F8605024F96016244F
:0E1D1D000970579067DCE0243DF582E434162F
:101D2B00F5837401F080459067DCE0243DF582E497
:101D3B003416F5837402F080339067DCE0243DF5B4
:101D4B0082E43416F5837403F080219067DCE02481
:101D5B003DF582E43416F5837404F0800F9067DC54
:101D6B00E0243DF582E43416F583E4F09068941298
:101D7B00D25390679212D28A9067DCE025E0FF90F5
:101D8B0067DBE033FE74B52FF582EE3416F583E492
:101D9B00A3E0540190685B75F00312D237E475F041
:101DAB0003A42583F58312D25390679512D28A7BB5
:101DBB00FF7AAB794A12D7537B017A6879431208C1
:101DCB00F2EF4E6046906843E04420FDB4631D90F3
:101DDB0067DCE025E0FF9067DBE033FE74B62FF5A0
:101DEB0082EE3416F583E054FEF0801FEDB46D1BCC
:101DFB009067DCE025E0FF9067DBE033FE74B62FE5
:101E0B00F582EE3416F583E04401F090689712D218
:101E1B005390679212D28A9067DCE025E0FF9067BF
:101E2B00DBE033FE74B52FF582EE3416F583E4A3B5
:101E3B00E05402FFE4C313FEEF1390686175F003E7
:101E4B0012D237EE75F003A42583F58312D253908B
:101E5B00679512D28A7BFF7AAB795612D7537B01E7
:101E6B007A6879431208F2EF4E6045906843E0447C
:101E7B0020FDB4791C9067DCE025E0FF9067DBE088
:101E8B0033FE74B62FF582EE3416F583E04402F080
:101E9B0022EDB46E1B9067DCE025E0FF9067DBE082
:101EAB0033FE74B62FF582EE3416F583E054FDF055
:011EBB002204
:101EBC007BFF7AAB79631208777BFF7AAB798D1253
:101ECC0008777BFF7AAB79B11208777BFF7AAB7915
:101EDC00D91208777BFF7AAB79F21208777BFF7AFD
:101EEC00AC79151208777BFF7AAC79421208777BB4
:101EFC00FF7AAC796D1208777BFF7AAC798A12087D
:101F0C00777BFF7AAC79AD1208777BFF7AAC79CB13
:101F1C001208777BFF7AA379F612087712E8E6AEFF
:101F2C0007EED394395005EE24D0FF22EE4420B4B2
:051F3C0071E17F71223C
:101F4100121EBCEF442064717003021FD3EF12D242
:101F51009F1F74001F79011F7E021F83031F8804C6
:101F61001F8D051F92061F97071F9C081FA10900BF
:101F7100001F4112716080C8126A0E80C3126AEF9D
:101F810080BE12704780B9126C3C80B4120ABA80CC
:101F9100AF125DAE80AA121FD480A51262C180A0CB
:101FA1007BFF7AA479E612087712E8E6EF44206411
:101FB10079708D1202CA7BFF7AAC79E91208771227
:101FC100E8E6EF442064796003021F4112904F025A
:031FD1001F41228B
:101FD400E49067EAF0A3F07BFF7AAD7916120877F4
:101FE40012E8E69067D5EFF04420646B7040906689
:101FF40032F07BFF7AAD794112087712E8E69067F8
:10200400D5EFF04420B4791C7BFF7AAD79781208BF
:10201400777BFF7AAD79AC120877900007E0442013
:10202400F00221AE900007E054DFF00221AE906789
:10203400D5E04420647960030220C690663204F03F
:102044007BFF7AAD79D812087712E8E6EF24CE60E8
:102054001D14603024027040906633742EF0A37413
:102064001EF0900009E04402F054FBF0802A9066D0
:10207400337421F0A37411F0900009E04404F05487
:10208400FDF080149066347401F0906633F0900093
:1020940009E054FDF054FBF07BFF7AAE790412089A
:1020A4007712E8E69067D5EFF04420B4790A9000FF
:1020B40005E04440F00221AE900005E054BFF00278
:1020C40021AE9067D5E04420646960030221AE909C
:1020D40066327402F07BFF7AAE7920906635E09028
:1020E4006792F012D7537B017A6779D61208F2EF20
:1020F4004E601F7BFF7AAE794B9067C212D28A7B07
:10210400017A6679359067C512D28A7A6779D612D0
:10211400DBE17BFF7AAE794F906636E0906792F010
:1021240012D7537B017A6779D61208F2EF4E601FFB
:102134007BFF7AAE794B9067C212D28A7B017A66B2
:1021440079369067C512D28A7A6779D612DBE17B39
:10215400FF7AAE797812D75312E8E6EF4420B479C7
:1021640009900009E04410F08007900009E054EF62
:10217400F07BFF7AAE7991900000E0FFA3E09067D6
:1021840092CFF0A3EFF012D7537B017A6779EC90EA
:10219400683012D28A7BFF7AAE79B012096AEF4EA8
:1021A4006008900000EEF0A3EFF07B017A6779EC11
:1021B40090683012D28A7BFF7AAE79BA12096A909B
:1021C40067EAEEF0A3EFF08EF012D2C5220004B05D
:1021D4002207096021E812C021F0258021F84B0074
:1021E4000000220D90002E7402F0801D90002E74C9
:1021F40003F0801590002E7404F0800DE490002EFE
:10220400F0800690002E7401F0C28C90002EE02421
:1022140028F582E43400F583E0F58CD28C7BFF7AD8
:10222400AE79EB12087712E8E6EF442024926010AE
:1022340024F57013900004E04420F0A3E0F080073C
:10224400900004E054DFF07BFF7AAF791212087734
:1022540012E8E6EF44202492602E24F56017240748
:102264007034900004E04440F0A3E0F0900007E0F4
:102274004410F08021900004E04440F0A3E0F0908A
:0B2284000007E054EFF0800E90000413
:10228F00E054BFF0900007E054EFF07BFF7AAF7996
:10229F003D12087712E8E6EF4420249F600C24FBE0
:1022AF00700F900005E04480F022900005E0547F0D
:0222BF00F0220B
:1022C1007BFF7AAF796F906792E52EF0A3E52FF04F
:1022D100A3E530F0A3E531F012D7537BFF7AAF7954
:1022E100B21208777BFF7AB07903120877E4F525FB
:1022F100906778E0FFE525C39F5035742D2525F5BE
:1023010082E43417F583E0FF3395E0FE7C007D1411
:1023110012D07474E92FF974003EFA7B0190679230
:1023210012D28A7BFF7AB0791212D753052580C069
:10233100906778E0F525E525C39405500D7BFF7A7C
:10234100B07918120877052580EC7BFF7AB07926E1
:0423510012087722D5
:102355007BFF7AB07929906792E52EF0A3E52FF0FF
:10236500A3E530F0A3E531F012D7537BFF7AB079BE
:102375006A1208777BFF7AB079B51208777BFF7A06
:10238500B17900120877900004E0A330E10B7BFFE0
:102395007AB1794A12087780097BFF7AB0792612DB
:1023A5000877906777E0FF3395E0FE742D2FF5826F
:1023B500EE3417F583E0FF3395E0FE7C007D1412C3
:1023C500D07474E92FF974003EFA7B01906792127C
:1023D500D28A7BFF7AB1798712D7537BFF7AB1799D
:0E23E5009E12D7537BFF7AB179ED12D75322A7
:1023F3009067F77420F0E4F526F527C3E5279405E5
:10240300E5269400503BE527AE267802C333CE334E
:10241300CED8F9FBAA062414F582EA3468F58312B0
:10242300D2060000000074002BF582EA3468F583BD
:1024330012D206000000000527E52770020526805A
:10244300BAE49067D6F09067D5F0900006E04404B4
:10245300F0A3E0F0900004E0A330E02F120850EF67
:10246300149067D6F0C3648094804018906778E036
:10247300FF9067D6E0FD3395E0FCC3ED9F7480F8D1
:102483006C984070E49067D6F080697BFF7AB279EC
:102493003A906778E0906792F012D7531286E790EC
:1024A3006777E0FFF47003022909EFFD3395E0FC41
:1024B300742D2DF582EC3417F583E0C3648094808A
:1024C3004014906778E0FDEF3395E0FEC3EF9D7411
:1024D30080F86E9840167BFF7AB2797C906778E03B
:1024E300906792F012D753E4906777F0906777E0A4
:1024F3009067D6F0906775E0FF906778E0D39F40D0
:1025030002EFF09067D6E0FF3395E0FE742D2FF5D0
:1025130082EE3417F583E09067D7F012083A12225F
:10252300C190E102E054F0F0900004E0FEA3E0FF6C
:1025330030E214EE30E3089067F77426F0800E90D3
:1025430067F77421F080069067F77420F0E4F526AE
:10255300F527906778E0FFC3E5279FE526940050B1
:10256300C7742D2527F582E43417F583E09067D5EA
:10257300F0C36480948040DAE0FFD3648094BC505D
:10258300D11243C91241D39067D5E0FF124963903A
:10259300674912D1C2C004C005C006C007E527AE13
:1025A300267802C333CE33CED8F92400F582EE3435
:1025B30068F583D007D006D005D00412D1FA90670E
:1025C3004112D1C2C004C005C006C007E527AE262C
:1025D3007802C333CE33CED8F92414F582EE3468AF
:1025E300F583D007D006D005D00412D1FA9067D76F
:1025F300E0FF9067D5E0B5071890674912D1C29004
:1026030067F812D1FA90674112D1C29067FC12D1D8
:10261300FAE59020E4061261640227587BFF7AB240
:1026230079BC9067F7E0906792F0A3E532F0A3E5F9
:1026330033F0A3E534F012D7537BFF7AB279D2900B
:10264300680012D1C290679212D1FA90681412D125
:10265300C290679612D1FA90680412D1C290679A19
:1026630012D1FA90681812D1C290679E12D1FA90D3
:10267300680812D1C29067A212D1FA90681C12D1D5
:10268300C29067A612D1FA90680C12D1C29067AAC1
:1026930012D1FA90682012D1C29067AE12D1FA1209
:1026A300D7537BFF7AB3790390681012D1C2906736
:0126B3009294
:1026B40012D1FA90682412D1C290679612D1FA12FC
:1026C400D7537F801202A07BFF7AB379119067926F
:1026D40012D28A906795E532F0A3E533F0A3E5348E
:1026E400F09067F7E0906798F09067D7E0FF339534
:1026F400E0FE7C007D1412D07474E92FF974003E5E
:10270400FA7B0190679912D28A7A6779D912D74DE8
:102714007B017A6779D91208957FC01202A07BFFEA
:102724007AB3792990679212D28A9067F812D1C24B
:1027340090679512D1FA9067FC12D1C290679912F2
:10274400D1FA7B017A6779D912D74D7B017A6779FF
:10275400D9120895900004E0A330E0751208509057
:1027640067D8EFF07008900004E054FDF022906701
:10277400D8E014F0906778E0FF9067D8E0FDFB3371
:1027840095E0FAC3EB9F7480F86A98400A90172D7D
:10279400E09067D7F08020EDFF3395E0FE742D2F95
:1027A400F582EE3417F583E0FF9067D7E0FEEF6E15
:1027B4006005EFF002252B90E101E0F430E409908C
:1027C4000005E04404F08064900005E054FBF080D0
:1027D4005B30985812E8E6EF4420249B600F24F500
:1027E400602014704790E102E054DFF0229000056D
:1027F400E030E20554FBF08033900005E04404F03F
:10280400802A900004E0FEA3E0FFEE30E30E900087
:102814000454F7F09067F77421F08010EE440890A8
:102824000004F0EFA3F09067F77426F090662A1284
:10283400D1C290674112D1DE12CBEE602B402990B9
:102844000005E030E222906777E527F07BFF7AA16C
:102854007946120877900004E054FBF012290A909C
:102864000004E0A330E256227F007E007D407CC05D
:1028740090674112D1DE12CBEE401990E000E030B7
:10288400E00990E102E04420F0803290E102E0545B
:10289400DFF0802990E102E054DFF0900004E0FED4
:1028A400A3E0FF30E40D30E20A9067D5E0FF129E0A
:1028B400BC800A90E102E054F0F012083A9000075C
:1028C400E030E636906777E0FF3395E0FEEF78027C
:1028D400C333CE33CED8F92414F582EE3468F583AD
:1028E40012D1C290662E12D1DE12CBEE600C400AD9
:1028F400439040900007E054BFF00527E52770029D
:0629040005260225552204
:10290A009068AE7420F0A3742AF0900004E0FEA34D
:10291A00E0FFEE30E11A90E00E740AF0EE30E308C0
:10292A009068AF7426F080159068AF7421F0800D1E
:10293A009068AF742AF090E00EE04401F090E10252
:10294A00E054DFF0900004E0FEA3E0FFEE30E01B6D
:10295A0020E118120850EF14906777F0C36480944E
:10296A008040E1E0D3648094BC50D9900006E044F2
:10297A0005F0A3E04481F0900006E0545FF090E097
:10298A000DE054FBF0906777E0FF90688EF0339586
:10299A00E0FE742D2FF582EE3417F583E0FFC36451
:1029AA00809480409F90688CEFF01243C9906641F2
:1029BA0012D20600000000906632E06401706FFFD8
:1029CA00FD1239F5900009E030E14E7FC97D04120D
:1029DA00C8797F607D0412C879E4FF7D0412C87942
:1029EA00E4FF7D0412C879906634E0FF7D0412C8C2
:1029FA00797F057D0412C8797F107D0412C879E4B5
:102A0A00FF7D0412C879E4FF7D0412C87990663408
:102A1A00E0FF7D0412C879800E900009E030E207D9
:102A2A00E4FF7D4E1239F5E4FF7D801239F5906698
:102A3A005912D1C290663912D1FA90665D12D1C28A
:102A4A0090663D12D1FA90688CE0FF123F477FCD25
:102A5A007ECC7DCC7C3D9065CA12D1DE12CBEE6075
:102A6A000A400890688CE0FF123CAA7FCD7ECC7D9C
:102A7A00CC7C3D9065C612D1DE12CBEE600A4008CE
:102A8A0090688CE0FF123A3E90665112D20600001E
:102A9A00000A906656E0B4040A90665112D2060003
:102AAA000000C812083A12235590E102E054F0F0EF
:102ABA00900004E0FEA3E0FF30E20A9068AFE090E5
:102ACA0068ADF080069068AD7420F0EE30E07A12BE
:102ADA00085090688DEFF0900004E0FEA3E0FFEE4E
:102AEA0020E12C90688DE0700BEE4402900004F017
:102AFA00EFA3F02290688DE014F0906777E0FF90E2
:102B0A00688DE0FE6F6016906777EEF002294E90AE
:102B1A00688DE07008900004E054FDF02290E10115
:102B2A00E0F430E412900005E04404F09068AFE06D
:102B3A009068ADF0022E1B900005E054FBF09068FF
:102B4A00AEE09068ADF0022E1B209803022E1B12F5
:102B5A00E8E6EF442012D29F2C98202CBD282D6F36
:102B6A002B2D8B2D2DAA302B99312BD8322C1833A3
:102B7A002C58342DB63F2D3B652E03692CF16E2D52
:102B8A0007702CD4712DF1742D627900002E1B90E0
:102B9A00688CE0FFFD3395E0FC74312DF582EC344E
:102BAA0013F583E4F0EF3395E0FEEFC4F8540FC851
:102BBA0068FFEEC454F048FE74712FF582EE340FAC
:102BCA00F58312D1C29065CA12D1FA022E1B9068FF
:102BDA008CE0FFFD3395E0FC74312DF582EC341363
:102BEA00F5837401F0EF3395E0FEEFC4F8540FC893
:102BFA0068FFEEC454F048FE74752FF582EE340F68
:102C0A00F58312D1C29065CA12D1FA022E1B9068BE
:102C1A008CE0FFFD3395E0FC74312DF582EC341322
:102C2A00F5837402F0EF3395E0FEEFC4F8540FC851
:102C3A0068FFEEC454F048FE74792FF582EE340F23
:102C4A00F58312D1C29065CA12D1FA022E1B90687E
:102C5A008CE0FFFD3395E0FC74312DF582EC3413E2
:102C6A00F5837403F0EF3395E0FEEFC4F8540FC810
:102C7A0068FFEEC454F048FE747D2FF582EE340FDF
:0B2C8A00F58312D1C29065CA12D1FA86
:102C9500022E1B906777E004F0906776E0FFA3E0D3
:102CA500FD3395E0FCC3ED9F7480F86C98500302EA
:102CB5002E1BE014F0022E1B906777E014F0E0C3A2
:102CC500648094804003022E1BE004F0022E1B90CA
:102CD500E102E054F0F0E054DFF0900006E054DF4C
:102CE500F0900004E04404F0A3E0F022900004E03A
:102CF500A320E103022E1B90E102E054DFF0122233
:102D0500C122900004E0FEA3E0FFEE20E103022EC5
:102D15001B30E30F90000454F7F09068AF7421F076
:102D2500022E1BEE4408900004F0EFA3F09068AF6C
:102D35007426F0022E1B900005E020E20E4404F0FC
:102D45009068AFE09068ADF0022E1B900005E0544E
:102D5500FBF09068AEE09068ADF0022E1B12083AC9
:102D650090E00DE04408F0022E1B90664112D1C29E
:102D7500EF2464FFE43EFEE43DFDE43CFC90664147
:102D850012D1FA022E1B90664112D1C2C3EF946490
:102D9500FFEE9400FEED9400FDEC9400FC9066417E
:102DA50012D1FA807190664112D2060000000080AF
:102DB50065906777E0FF3395E0FE742D2FF582EE81
:102DC5003417F583E0FF3395E0FE7C007D1412D0C7
:102DD5007474E92FF974003EFA7B0190679212D260
:102DE5008A7BFF7AB3793E12D753802A90688CE0AC
:102DF500FF123CAA90688CE0FF123A3E801890685A
:102E05008CE0FF123F4790688CE0FF123CAA906867
:102E15008CE0FF123A3E906777E0FF90688EE06F96
:102E250060030229751241D390688CE0FF12496353
:102E350090674912D1C290660212D1FA9067411289
:102E4500D1C290660612D1FA90688CE0FF3395E006
:102E5500FE126497E59020E40612616402301A7B45
:102E6500FF7AB379459068ADE0906792F0A3E532BB
:102E7500F0A3E533F0A3E534F012D7539067491278
:102E8500D1C290679212D1FA90674112D1C2906770
:102E95009612D1FA90672D12D1C290679A12D1FA83
:102EA5007F487E517DC77CC59066CD12D1DE12C9A3
:102EB5005B90679E12D1FA90674D12D1C29067A2BE
:102EC50012D1FA90675112D1C29067A612D1FA9029
:102ED50066B512D1C29067AA12D1FA90675912D17C
:102EE500C29067AE12D1FA7BFF7AB3795A12D753E3
:102EF50090664112D1C2EC12CC6C90679212D1FA55
:102F05007BFF7AB3798412D7537F801202A07BFFAF
:102F15007AB3798E90679212D28A906795E532F0EE
:0B2F2500A3E533F0A3E534F09068ADA5
:102F3000E0906798F0906777E0FF3395E0FE742D9E
:102F40002FF582EE3417F583E0FF3395E0FE7C0029
:102F50007D1412D07474E92FF974003EFA7B01904D
:102F6000679912D28A7A68798F12D74D7B017A6875
:102F7000798F1208957FC01202A0906777E0FF3327
:102F800095E0FE742D2FF582EE3417F583E0FF33C4
:102F900095E0FEEF25E0FFEE33FE74B52FF582EEEF
:102FA0003416F583A3E030E13B7BFF7AB379A89038
:102FB000679212D28A90674912D1C290679512D156
:102FC000FA90674112D1C290679912D1FA9066B512
:102FD00012D1C290679D12D1FA7B017A68798F1263
:102FE000D74D802D7BFF7AB379C190679212D28A38
:102FF00090674912D1C290679512D1FA9067411239
:10300000D1C290679912D1FA7B017A68798F12D771
:103010004D7B017A68798F12089590662A12D1C289
:1030200090674112D1DE12CBEE402B5390BF90003F
:1030300007E04440F0900006E0FEA3E0FFEE30E63B
:1030400075900005E030E26EEE20E76A90688CE053
:10305000FF12342A8060900004E0A330E12590E163
:1030600002E054F0F01222C17BFF7AA179461208E7
:1030700077900006E04404F0A3E0F0900006E054EE
:10308000DFF022900007E030E62C90662E12D1C2CD
:1030900090674112D1DE12CBEE600250194390408E
:1030A00090664112D20600000000900006E0545FD6
:1030B000F0A3E054BFF0900007E030E72C7F007EE3
:1030C000007D007C0090660612D1DE12CBEE601906
:1030D000401790688CE0FF123F4790688CE0FF1229
:1030E0003CAA900007E0547FF0900005E030E00B30
:1030F00090688CE0FF1236BF02318D900005E02011
:10310000E7157F007E007D407CC090660612D1DE10
:1031100012CBEE6078407690663D12D1C290665D2B
:1031200012D1DE12D11612E9297B2C7A01790078AE
:1031300000C312D181501C900004E0A330E514902C
:10314000665D12D1C290663D12D1FA90688CE0FFA4
:10315000123CAA90663912D1C290665912D1DE1281
:10316000D11612E92990665112D1DEC312D19750BF
:103170001C900004E0A330E61490665912D1C2906E
:10318000663912D1FA90688CE0FF123A3E90E10164
:10319000E020E56AE020E63890688CE0FF3395E0B7
:1031A000FEEF7802C333CE33CED8F9244DF582EE4C
:1031B0003415F583C083C08212D1C27B007A0079B6
:1031C00048784212C95BD082D08312D1FA02325DB4
:1031D00090E101E020E70C90664112D20600000069
:1031E00000807A90664112D1C2EF2432FFE43EFEA5
:0931F000E43DFDE43CFC90664165
:1031F90012D1FA805F90E101E020E758E020E6373C
:1032090090688CE0FF3395E0FEEF7802C333CE334C
:10321900CED8F9244DF582EE3415F583C083C082EA
:1032290012D1C27B007A007948784212C957D082FC
:10323900D08312D1FA801D90664112D1C2C3EF9496
:1032490032FFEE9400FEED9400FDEC9400FC9066D4
:103259004112D1FA906771E0FEA3E0FFE4FCFDC0E2
:1032690004C005C006C00790676912D1DE90676582
:1032790012D1C212D116A804A905AA06AB07D00714
:10328900D006D005D004D312D1975038906771E099
:10329900FEA3E0FFE4FCFDC004C005C006C0079022
:1032A900676D12D1DE90676512D1C212D116A804DA
:1032B900A905AA06AB07D007D006D005D004D312BA
:1032C900D19740031235F6900007E030E30990E109
:1032D90002E04450F0800790E102E054AFF090E042
:1032E9000DE020E20302341A900004E0FEA3E0FF9F
:1032F900EE20E30302341A20E10302341A90E00DB0
:10330900E054FBF0E4906889F0A3F0906778E0FF5F
:10331900C390688AE09F906889E094004003023472
:1033290012A3E0242DF582E43417F583E090688B2D
:10333900F0C3648094805003023405E0FFD36480B5
:1033490094BC40030234051243C91241D390688BDF
:10335900E0FF1249637F007E007D007CC0906741D9
:1033690012D1DE12CBEE600250030234059067776A
:10337900E0FF3395E0FEC390688AE09F906889E09A
:103389009E503EA3E0FF906777F03395E0FE742DE1
:103399002FF582EE3417F583E0FF3395E0FE7C00CC
:1033A9007D1412D07474E92FF974003EFA7B0190F0
:1033B900679212D28A7BFF7AB379D712D75302293F
:1033C90075906777E0FF3395E0FED390688AE09FB8
:1033D900906889E09E40327F007E007D007C0090ED
:1033E900660612D1DE12CBEE501F900007E020E7EF
:1033F9001890688AE0906777F0022975906889E4E7
:1034090075F00112D0BE02331490688CE0FF1243AC
:10341900C990688CE0FF3395E0FE126497022ABADE
:013429002280
:10342A009068B0EFF090674912D1C29068B112D19A
:10343A00FA90E102E054F0F07F007E007D207C41AA
:10344A009065B612D1DE12CBEE40199065CE12D13C
:10345A00C27B607A0B79B6783A12C95B9065CE1254
:10346A00D1FA80179065CE12D1C27B2F7A8E7963FA
:10347A00783C12C95B9065CE12D1FA9068B0E0FF31
:10348A001249637FC01202A07BFF7AB379FE120849
:10349A0095900005E030E3030235337F007E007D1E
:1034AA00B47C429068B112D1DE12CBEE602A402879
:1034BA007F007E007D347C439068B112D1DE12CB4E
:1034CA00EE50157F007E007D347C4390674912D10F
:1034DA00DE12CBEE600250447F007E007D877C4383
:1034EA009068B112D1DE12CBEE40030235B77F00ED
:1034FA007E007D347C439068B112D1DE12CBEE603F
:10350A000250030235B77F007E007D347C4390670A
:10351A004912D1DE12CBEE40030235B7900006E025
:10352A004420F0A3E0F00235E07F007E007D877C36
:10353A00439068B112D1DE12CBEE602840267F009C
:10354A007E007DB47C439068B112D1DE12CBEE507E
:10355A00137F007E007DB47C4290674912D1DE124F
:10356A00CBEE403D7F007E007DB47C429068B11274
:10357A00D1DE12CBEE50367F007E007D007C0090BB
:10358A0068B112D1DE12CBEE602340217F007E00AB
:10359A007D877C4390674912D1DE12CBEE600E40E4
:1035AA000C900006E04420F0A3E0F0802990662AFF
:1035BA0012D1C290674112D1DE12CBEE50099000AF
:1035CA0006E054DFF0800F90674912D1C29068B1CB
:1035DA0012D1FA023442900006E04480F0A3E0F0EF
:0C35EA001241D39068B0E0FF1249632248
:1035F600900006E0A330E3030236BE90E102E054F9
:10360600F0F07BFF7AB4790F906792E532F0A3E58C
:1036160033F0A3E534F012D7537F801202A07BFF6C
:103626007AB479681208957FC01202A07BFF7AB43B
:1036360079791208959068B3E4F0A3E533F0A3E432
:10364600F0A3E534F090E000E030E00990E102E01C
:103656004420F0800790E102E054DFF01241D3905D
:1036660068B3E0FCA3E0FDC3E5339DE49CC364803E
:1036760094805006743C2533F5339068B5E0FAA380
:10368600E0B534C1E4B502BDC3E5339DFFE49CFE5D
:10369600906773E0FCA3E0B507ABEEB504A77BFF2C
:1036A6007AB4798A906792E532F0A3E533F0A3E520
:0936B60034F012D75312083A2235
:1036BF009068B0EFF090001CE0FEA3E0FFC3900015
:1036CF001FE09F9068B4F090001EE09E9068B3F0EA
:1036DF0090001AE0FF7E007C037DE812D0749068A2
:1036EF00B5EEF0A3EFF07F007E007D007C009066CA
:1036FF000612D1DE12CBEE50030238017F03120AFD
:10370F008A90001CE0FEA3E0FFC3E5299F9068B2FA
:10371F00F0E5289E9068B1F09068B3E0FEA3E0FF5B
:10372F0012E917C006C0079068B1E0FEA3E0FF12D0
:10373F00E917AC06AD07D007D006C3ED9FEE648046
:10374F00F8EC6480985003023801C39068B3E064CA
:10375F008094805043D39068B2E094009068B1E0B9
:10376F00648094804019900007E030E30990E102F3
:10377F00E054BFF0806390E102E04440F0805A9043
:10378F000007E030E30990E102E054EFF0804A9047
:10379F00E102E04410F08041D39068B2E0940090D1
:1037AF0068B1E0648094804019900007E030E3092D
:1037BF0090E102E054EFF0802090E102E04410F03D
:1037CF008017900007E030E30990E102E054BFF06A
:1037DF00800790E102E04440F0E4FFFE9068B5E01E
:1037EF00FCA3E0FDC3EF9DEE9C50070FEF70010EA1
:0337FF0080EA223B
:1038020090001AE0FF7E007C037DE812D07490687D
:10381200B6EEF0A3EFF090001BE0FF7E0012D07432
:103822009068B8EEF0A3EFF090677D12D1DE90665B
:103832005912D1C212D1169068BA12D1FA90678188
:1038420012D1DE9068BA12D1C212E87B12E9299035
:1038520068BE12D1FA7BFF7AB479B990677D12D132
:10386200C290679212D1FA90665912D1C2906796AD
:1038720012D1FA9068BA12D1C290679A12D1FA9014
:1038820068BE12D1C290679E12D1FA12D7537F003E
:103892007E007D007C009068BA12D1DED312D18105
:1038A200400B7BFF7AB479E6120877801D7F007E99
:1038B200007D007C009068BA12D1DEC312D1815023
:1038C200097BFF7AB479F0120877E49068B2F0A32A
:1038D200F09068B2E0FEA3E0FFE4FCFD9068BE1247
:1038E200D1DED312D19750030239E47F007E007DEE
:1038F200007C009068BA12D1DED312D181401990B7
:103902000007E030E30990E102E054EFF0802090FC
:10391200E102E04410F08017900007E030E30990E4
:10392200E102E054BFF0800790E102E04440F07B06
:10393200FF7AB479FB120877E49068B4F0A3F090B0
:1039420068B6E0FEA3E0FFC39068B5E09F9068B45C
:10395200E09E500C9068B4E475F00112D0BE80DF96
:103962007F007E007D007C009068BA12D1DED31207
:10397200D1814019900007E030E30990E102E04470
:1039820010F0802090E102E054EFF08017900007E1
:10399200E030E30990E102E04440F0800790E10268
:1039A200E054BFF07BFF7AB479FD120877E49068A7
:1039B200B4F0A3F09068B8E0FEA3E0FFC39068B54E
:1039C200E09F9068B4E09E500C9068B4E475F001FA
:1039D20012D0BE80DF9068B2E475F00112D0BE0250
:1039E20038D37BFF7AB07926120877900007E0542B
:0339F200FEF022C2
:1039F5008D0C7D0412C879E4FF7D0412C879E4FFBB
:103A05007D0412C879E4FF7D0412C879AF0C7D04EA
:043A150012C8792238
:103A1900906904EFF07FFEE4FD12C8797FFEE4FDB2
:103A290012C879906904E0FFE4FD12C8797F02E4C5
:053A3900FD12C8792216
:103A3E009068B3EFF0906632E0705B7BFF7AB479FA
:103A4E00FF90679212D28A90665912D1C2906795F2
:103A5E0012D1FA7B017A6879BC12D74D900007E03B
:103A6E0030E5299068B3E0FF3395E0FEEF25E0FFE7
:103A7E00EE33FE74B52FF582EE3416F583A3E030E7
:103A8E00E30A7B017A6879BC1208D3227B017A683B
:103A9E0079BC1208B322906632E064016003023BE7
:103AAE00C7FFFD1239F57B0A7A007900780090661F
:103ABE005912D1C212E87B9068B812D1FA7BFF7A04
:103ACE00B5790A90679212D28A9068B812D1C290D4
:103ADE00679512D1FA7B017A6879BC12D74DE490C2
:103AEE0068B7F09068B6F09068BCE0B4311DA3E002
:103AFE00B43218A3E024D0540F9068B6F044C0FF3F
:103B0E009068B5F07D0412C87980319068BCE0648D
:103B1E00307029A3E024D0540FFF9068B7F090685E
:103B2E00BEE024D0540FFE9068B6F0EFC454F054AB
:103B3E00F04EFF9068B5F07D0412C8799068B474A9
:103B4E0003F09068B4E0C364809488505AE490689F
:103B5E00B7F09068B6F09068B4E0FFFD3395E0FCE6
:103B6E0074BC2DF582EC3468F583E024D0540FFE3E
:103B7E009068B7F0EF3395E0FC74BD2DF582EC3410
:103B8E0068F583E024D0540FFF9068B6F0EEC4546D
:103B9E00F054F04FFF9068B5F07D0412C87990682C
:103BAE00B4E02402F0809B906634E0FF7D0412C8DE
:103BBE0079E4FF7D801239F522906632E06402606E
:103BCE0003023CA990665912D1C29068B812D1FA7C
:103BDE007BFF7AB5791190679212D28A9068B812EB
:103BEE00D1C290679512D1FA7B017A6879BC12D74F
:103BFE004D900009E020E425906637E0FF123A1957
:103C0E007F07E4FD12C8797FD1E4FD12C8797FFDEC
:103C1E00E4FD12C879900001E0FF12C945906637A5
:103C2E00E0FF123A19E4FFFD12C8799068B47409E6
:103C3E00F09068B4E0FFD364809480404FE49068C5
:103C4E00B7F09068B6F0EF3395E0FE74BC2FF582B6
:103C5E00EE3468F583E024D0540FFD9068B6F0740E
:103C6E00BB2FF582EE3468F583E024D0540FFF901D
:103C7E0068B7F0C454F054F04DFF9068B5F0E4FD11
:103C8E0012C8799068B4E024FEF080A57FFDE4FDB3
:0C3C9E0012C879900001E0FF12C9452215
:103CAA009068B3EFF0906632E06003023D417BFF1B
:103CBA007AB5791990679212D28A90665D12D1C24A
:103CCA0090679512D1FA7B017A6879B812D74D902C
:103CDA000007E030E5459068B3E0FF3395E0FEEF7A
:103CEA0025E0FFEE33FE74B52FF582EE3416F58328
:103CFA00A3E030E3137BFF7AB579241208B37B0182
:103D0A007A6879B81208B3227BFF7AB57924120847
:103D1A00D37B017A6879B81208D3227BFF7AB57906
:103D2A00241208B37B017A6879B81208B37BFF7A48
:103D3A00B579291208B322906632E0640160030261
:103D4A003E64FFFD1239F57B0A7A0079007800900B
:103D5A00665D12D1C212E87B9068E012D1FA7BFF4D
:103D6A007AB5790A90679212D28A9068E012D1C223
:103D7A0090679512D1FA7B017A6879B812D74DE427
:103D8A009068B7F09068B6F09068B8E0B4311DA3B7
:103D9A00E0B43218A3E024D0540F9068B6F044C0BF
:103DAA00FF9068B5F07D0412C87980319068B8E058
:103DBA0064307029A3E024D0540FFF9068B7F090C4
:103DCA0068BAE024D0540FFE9068B6F0EFC454F0FD
:103DDA0054F04EFF9068B5F07D0412C8799068B42B
:103DEA007403F09068B4E0C364809488505AE490F5
:103DFA0068B7F09068B6F09068B4E0FFFD3395E0DC
:103E0A00FC74B82DF582EC3468F583E024D0540FA5
:103E1A00FE9068B7F0EF3395E0FC74B92DF582ECAB
:103E2A003468F583E024D0540FFF9068B6F0EEC4EE
:103E3A0054F054F04FFF9068B5F07D0412C87990A1
:103E4A0068B4E02402F0809B906633E0FF7D0412A0
:103E5A00C879E4FF7D801239F522906632E0640267
:103E6A006003023F4690665D12D1C29068E012D1AB
:103E7A00FA7BFF7AB5791190679212D28A9068E03C
:103E8A0012D1C290679512D1FA7B017A6879B81279
:103E9A00D74D900009E020E425906638E0FF123AF9
:103EAA00197F07E4FD12C8797FD0E4FD12C8797F33
:103EBA00FDE4FD12C879900001E0FF12C945906641
:103ECA0038E0FF123A19E4FFFD12C8799068B47419
:103EDA0009F09068B4E0FFD364809480404FE49086
:103EEA0068B7F09068B6F0EF3395E0FE74B82FF536
:103EFA0082EE3468F583E024D0540FFD9068B6F062
:103F0A0074B72FF582EE3468F583E024D0540FFF9E
:103F1A009068B7F0C454F054F04DFF9068B5F0E4DF
:103F2A00FD12C8799068B4E024FEF080A57FFDE414
:0D3F3A00FD12C879900001E0FF12C9452278
:103F47009068B3EFF0906632E060030240527BFF67
:103F57007AB5792E90679212D28A906655E090676B
:103F670095F07B017A6879B412D74D7BFF7AB579E2
:103F77002E90679212D28A906656E0906795F07BF2
:103F8700017A6879DC12D74D900007E020E503023B
:103F9700401B9068B3E025E024B5F582E43416F5BC
:103FA70083A3E030E3377BFF7AB579241208B37B2C
:103FB700FF7AB579361208B37B017A6879B41208AB
:103FC700B37BFF7AB579291208D37BFF7AB5793BA2
:103FD7001208D37B017A6879DC1208D3227BFF7A37
:103FE700B579241208D37BFF7AB579361208D37BCB
:103FF700017A6879B41208D37BFF7AB57929120858
:10400700B37BFF7AB5793B1208B37B017A6879DC19
:104017001208B3227BFF7AB579241208B37BFF7AA3
:10402700B579361208B37B017A6879B41208B37B85
:10403700FF7AB579291208B37BFF7AB5793B120865
:10404700B37B017A6879DC1208B322906632E064A8
:10405700017073FFFD1239F5906655E0FF60262465
:10406700FE600A04700FE4900002F0800E900002D8
:104077007401F080069000027408F0900002E0FFDF
:104087007D271239F5906656E024FE600A04700F0A
:10409700E4900002F0801D9000027401F0801590FA
:1040A7000005E030E6089000027488F08006900072
:1040B700027408F0900002E0FF7D171239F5E4FF63
:1040C7007D801239F522906632E064026003024176
:1040D700D2900009E020E425906638E0FF123A19F3
:1040E7007F07E4FD12C8797FD0E4FD12C8797FFD10
:1040F700E4FD12C879900001E0FF12C945906638C7
:10410700E0FF123A197F01E4FD12C879906655E085
:1041170024FE601214601814601E24037021E4FF4B
:10412700FD12C87980197F01E4FD12C87980107FDC
:1041370003E4FD12C87980077F05E4FD12C8797F83
:10414700FDE4FD12C879900001E0FF12C945900017
:1041570009E020E425906637E0FF123A197F07E46B
:10416700FD12C8797FD1E4FD12C8797FFDE4FD1205
:10417700C879900001E0FF12C945906637E0FF1249
:104187003A197F01E4FD12C879906656E024FE6073
:104197001214601814601E24037021E4FFFD12C876
:1041A7007980197F01E4FD12C87980107F03E4FD4F
:1041B70012C87980077F05E4FD12C8797FFDE4FD09
:0C41C70012C879900001E0FF12C94522E7
:1041D300120A19E53575F00AA4FF7C002536FFECB9
:1041E30035F0CF245CF52FEF3405F52EE535643932
:1041F300600B7464252FF52FE4352EF52EE5372457
:10420300D075F00AA4FFE53824D02FF530E5392422
:10421300D075F00AA4FFE53A24D02FF531E53B240D
:10422300D075F00AA4FFE53C24D02FF532E53D24F8
:10423300D075F00AA4FFE53E24D02FF533E53F24E3
:10424300D075F00AA4FFE54024D02FF534AF2FAE8C
:104253002EAD30AB31124386AC06AD07E412CC7100
:104263009065D612D1FAAF32E4FCFDFE7B107A0ED4
:10427300F9F812D124EC12CC6CC004C005C006C0FE
:10428300077F007EC07DA87C479065D612D1DE12E1
:10429300CA4CD003D002D001D00012C95BC004C005
:1042A30005C006C007AF33E4FCFDFE7B3CFAF9F81A
:1042B30012D124EC12CC6CD003D002D001D0001266
:1042C300C95BC004C005C006C007AF34E4FCFDFEF3
:1042D30012CC6CD003D002D001D00012C95B12CC37
:1042E300AA90676512D1FA90676512D1C2E412CC25
:1042F3006C7B007AC079A8784712CB559065CE12B3
:10430300D1FAAC2EAD2FE412CC719065DA12D1DE66
:1043130012C95712CCAA8E0C8F0DEF4E6064750E26
:1043230000750F01D3E50F950DE50E950C5053E580
:104333002F24FFFFE52E34FFEF540370199065CE51
:1043430012D1C27B007A0079B7784312C95B9065BA
:10435300CE12D1FA80179065CE12D1C27B007A803B
:1043630079B6784312C95B9065CE12D1FAD3E50FC3
:104373009405E50E9400500A050FE50F7002050E33
:0343830080A222F3
:104386009068B7EEF0A3EFF0AF037E00E4E05403CD
:1043960070047C0180027C00A9047C01ECC39D5062
:1043A60021E975F00DA4242FF582E43400F583E5A8
:1043B600822CF582E43583F583E02FFFE43EFE0C84
:0343C60080DA2278
:1043C9009068B3EFF0E0FFC3648094805003024922
:1043D90062EF3395E0FEEF25E0FFEE33FE74992F8F
:1043E900F582EE3405F583E0FEA3E0246CFDEE349E
:1043F90007FCE412CC719065DA12D1FA9068B3E047
:10440900FF3395E0FEEF25E0FFEE33FE74992FF5BB
:1044190082EE3405F583E0FEA3E0C3945AEE9400DE
:1044290050179065DA12D1C27B007A0079C87842B8
:1044390012C95B9065DA12D1FA7F007EE07DF87CC3
:10444900C49065DA12D1DE12C95B12CCAA9068B4A5
:10445900EEF0A3EFF0C3EE64809480400ED3E094B5
:104469001D9068B4E06480948040099068B4E4F0D9
:10447900A3741DF09068B3E0FF3395E0FEEF780276
:10448900C333CE33CED8F9FBAA062411F582EA3418
:1044990006F58312D1C29065BE12D1FA74C12BF50B
:1044A90082EA340AF58312D1C2E412CC6C9065BA5F
:1044B90012D1FA9068B3E0F9FF3395E0FEEF780284
:1044C900C333CE33CED8F9FBAA062401F582EA34E8
:1044D90007F58312D1C29065B212D1FA74F12BF5A6
:1044E90082EA3407F58312D1C29065B612D1FAE98E
:1044F900FF3395E0FEEF7802C333CE33CED8F9FB14
:10450900AA0624E1F582EA3408F58312D1C290653E
:10451900A212D1FA74D12BF582EA3409F58312D1AA
:10452900C29065AA12D1FAE9FF3395E0FEEF78024D
:10453900C333CE33CED8F9FBAA0624B1F582EA34C7
:104549000BF58312D1C29065AE12D1FA74A12BF585
:1045590082EA340CF58312D1C29065A612D1FAE928
:10456900FF3395E0FEEF7802C333CE33CED8F9FBA3
:10457900AA062491F582EA340DF58312D1C2906519
:10458900C212D1FA74812BF582EA340EF58312D165
:10459900C29065C612D1FAE9FF3395E0FEEFC4F87F
:1045A900540FC868FFEEC454F048FE74712FF582A9
:1045B900EE340FF583C083C0829068B3E0FF339572
:1045C900E0FE74312FF582EE3413F583E0D082D00A
:1045D9008375F00412D23712D1C29065CA12D1FA8A
:1045E9007F007E007D007C0090677912D1DEC312C6
:1045F900D1977019FF7E247D747C499065C612D1CC
:10460900DE12CA4C12CCAA90677D12D1FA9068B317
:10461900E0F9FF3395E0FE743D2FF582EE3416F58F
:1046290083E0906655F074792FF582EE3416F583A0
:10463900E0906656F0E93395E0FEEF25E0FFEE33B2
:10464900FE74B52FF582EE3416F583E0FEA3E0FF84
:1046590030E009900005E04401F08007900005E092
:1046690054FEF0EF30E210906636E0A3F090663524
:10467900E0906638F08010906635E0906637F090EB
:104689006636E0906638F07F007E247D747C499020
:1046990065C612D1DE12CA4C12CCAA90665912D143
:1046A900FA90665912D1DEC000C001C002C0039061
:1046B90068B3E0FF3395E0FEEF7802C333CE33CE23
:1046C900D8F9246DF582EE3413F58312D1C27B003B
:1046D9007A247974784912CA4C12CCAAD003D00230
:1046E900D001D00012D10990665912D1FA7F007E0B
:1046F900247D747C499065CA12D1DE12CA4C12CC51
:10470900AA90665D12D1FA90665D12D1DEC000C032
:1047190001C002C0039068B3E0FF3395E0FEEF7873
:1047290002C333CE33CED8F9245DF582EE3414F5C5
:104739008312D1C27B007A247974784912CA4C1247
:0D474900CCAAD003D002D001D00012D109BB
:1047560090665D12D1FA9068B4E0FEA3E07802C3D9
:1047660033CE33CED8F92449F582EE3400F58312E0
:10477600D1C290659E12D1FA7F357EFA7D8E7C3C41
:104786009065A212D1DE12CA4C12DFD49066A11235
:10479600D1FA7F357EFA7D8E7C3C9065A212D1DE01
:1047A60012CA4C12DFBE9066A512D1FA7F357EFA88
:1047B6007D8E7C3C90000A12D1DE12CA4C906715A1
:1047C60012D1FA90671512D1C212DFD4906719126E
:1047D600D1FA90671512D1C212DFBE90671D12D1B1
:1047E600FA7F357EFA7D8E7CBC90001212D1DE12E5
:1047F600CA4C12DFD490672112D1FA7F357EFA7D3A
:104806008E7C3C90001212D1DE12CA4C12DFBE9092
:10481600672512D1FA7F007E007D007C40906715E7
:1048260012D1DE12CA4C12DFBE7B297ABC79DB7844
:104836003A12CA4C7B227A92797F783F12C95B7B07
:10484600487A5179C7784512CA4CC004C005C006DB
:10485600C0077B007A00797A784490001612D1C29C
:1048660012CB55D003D002D001D00012C95B90669E
:10487600D112D1FA7F447E497D7E7C3F9067191222
:10488600D1DE12CA4C90671D12D1DE12CB5512E151
:104896001E90671512D1FA90671512D1C212DFD495
:1048A6009066D112D1DE12CA4C90670112D1FA90ED
:1048B600671512D1C212DFBE9066D112D1DE12CABE
:1048C6004C90672512D1DE12CA4C9066DD12D1FAE1
:1048D60090671512D1C212DFBE9066D112D1DE12D8
:1048E600CA4C90672112D1DE12CA4C9066ED12D1E5
:1048F600FA90671512D1C212DFBEC004C005C00609
:10490600C0079066D112D1C212CC5BD003D002D0C0
:1049160001D00012CA4C90672112D1DE12CA4C7B1C
:10492600407AED7998783812CA4C90675D12D1FAC0
:1049360090671512D1C212DFBE9066D112D1DE1277
:10494600CA4C90672512D1DE12CA4C7B407AED79AB
:0D49560098783812CA4C90676112D1FA228D
:104963009068B5EFF09065BE12D1DE9065CE12D19E
:10497300C212C95790690212D1FA7F007E007D00EE
:104983007C4090690212D1DE12CA4C9065C212D1EA
:10499300DE12CA4C9065B612D1DE12C95B9068B6BE
:1049A30012D1FA9068B612D1C2A804A905AA06AB1F
:1049B3000712CA4CA804A905AA06AB077FCB7E1829
:1049C3007D897C5612CB55C004C005C006C0079034
:1049D300692612D2063EAAAAABD007D006D005D0CC
:1049E3000412E40790669512D1FA9068B612D1C208
:1049F30090669512D1DE12CA4C7B5B7A82799878E5
:104A03003812CA4C9068BA12D1FA9065AA12D1C270
:104A1300A804A905AA06AB0712CA4CA804A905AAAB
:104A230006AB077F007E007D807C3F12C9579068EC
:104A3300EA12D1FA9068EA12D1C212DECE90669DD4
:104A430012D1FA7B007A0079B478439065B212D11F
:104A5300C212CB559065BA12D1DE12C95B90690AB6
:104A630012D1FA90669512D1DE7F487E517DC77CC4
:104A73004512CB55C004C005C006C0079069261275
:104A8300D20640600000D007D006D005D00412E45F
:104A9300077B337A33791F784112CA4CC004C005AF
:104AA300C006C0079068EA12D1C2A804A905AA06E5
:104AB300AB0712CA4CA804A905AA06AB07D007D0B6
:104AC30006D005D00412CB559068EE12D1FA906847
:104AD300EE12D1C290690212D1DE12CA4C9066A5C1
:104AE30012D1DE12CA4CA804A905AA06AB07906529
:104AF300A612D1C212C9579066A912D1FA7F357E88
:104B0300FA7D8E7C3C9066A912D1DE12CA4C12DF6C
:104B1300D49068E612D1FA7F357EFA7D8E7C3C9084
:104B230066A912D1DE12CA4C12DFBE9068E212D11E
:104B3300FA9066A512D1C2A804A905AA06AB07126A
:104B4300CA4C7B007A007920784012CA4C7B007AE9
:104B530000790078BF12C95BC004C005C006C00756
:104B63009068EE12D1C290690212D1DE12CA4CD003
:104B730003D002D001D00012CA4C9065AE12D1DE30
:104B830012C95B9066AD12D1FA7F357EFA7D8E7CB9
:104B93003C9066AD12D1DE12CA4C12DFD49068F697
:104BA30012D1FA7F357EFA7D8E7C3C9066AD12D1B0
:104BB300DE12CA4C12DFBE9068F212D1FA9068E698
:104BC30012D1C29068F612D1DE12CA4C9066A512B9
:104BD300D1DE12CA4CC004C005C006C0079068E20B
:104BE30012D1C29068F212D1DE12CA4CD003D002A5
:104BF300D001D00012C95790667912D1FA9068E6B5
:0F4C030012D1C29068F212D1DE12CA4C9066A58F
:104C120012D1DE12CA4CC004C005C006C00790689B
:104C2200E212D1C29068F612D1DE12CA4C7B007A2F
:104C320000798078BF12CA4CD003D002D001D000D4
:104C420012C95790668912D1FA9068E212D1C290C5
:104C520068F612D1DE12CA4C9066A512D1DE12CAD3
:104C62004CC004C005C006C0079068E612D1C290CD
:104C720068F212D1DE12CA4CD003D002D001D000A9
:104C820012C95B90667D12D1FA9068E212D1C2908D
:104C920068F212D1DE12CA4C9066A512D1DE12CA97
:104CA2004CC004C005C006C0079068E612D1C2908D
:104CB20068F612D1DE12CA4C7B007A00798078BF86
:104CC20012CA4CD003D002D001D00012C95B906648
:104CD2008D12D1FA9066A112D1C29068F612D1DE7D
:104CE20012CA4C90668112D1FA9066A112D1C2907A
:104CF20068F212D1DE12CA4C90669112D1FA906912
:104D02002612D2064000000090690212D1C212E4BB
:104D1200079065C212D1DE12CA4CC004C005C0069B
:104D2200C00790690212D1C29065B612D1DE12CAD2
:104D32004C90690A12D1DE12C95BD003D002D001B5
:104D4200D00012C95B90690612D1FA7FBD7E377D11
:104D5200867C3590690612D1DE12C95B12E314908B
:104D620068FA12D1FA9068FA12D1DE90690612D16D
:104D7200C212C9577BBD7A377986783512C95B7BF7
:104D8200007A007980784312CA4C9066B512D1FA43
:104D92009068FA12D1DE90690612D1C212C9577B0D
:104DA200DB7A0F79C9784012CA4C9066B912D1FAEF
:104DB2007F007E007D007C409066B912D1DE12CA6F
:104DC2004C12DFD4C004C005C006C0079065AA1209
:104DD200D1C2A804A905AA06AB0712CA4C7B007A65
:104DE200007900783F12CA4CD003D002D001D00023
:104DF20012CA4CC004C005C006C0079066B912D1E1
:104E0200C212DFD49065AA12D1DE12CA4C9066B9E2
:104E120012D1DE12C95BD003D002D001D00012C978
:104E22005B90669912D1FA90669912D1C212DFD4C0
:104E32009066BD12D1FA90669912D1C212DFBE906D
:104E420066C112D1FA9066C112D1C29065AA12D17E
:104E5200DE12CA4CA804A905AA06AB077F007E0091
:104E62007D807C3F12C9579066C512D1FA9066BD0B
:094E720012D1C29065AA12D1DE32
:104E7B0012CA4CA804A905AA06AB0790669912D1D1
:104E8B00C212C9579066C912D1FA9066B912D1DE17
:104E9B009066C912D1C212C9579068DE12D1FA902E
:104EAB0068DE12D1C212DE747BBD7A377986783513
:104EBB0012CBEE6002503990669912D1C2C004C079
:104ECB0005C006C0079066C512D1DE9068DE12D110
:104EDB00C212CB55A804A905AA06AB07D007D0066A
:104EEB00D005D00412C95790669912D1FA024E29F7
:104EFB009065AA12D1DE9066C112D1C212C9579029
:104F0B00669512D1DE12CA4C9066D912D1FA906610
:104F1B009D12D1C290669512D1DE12CA4C9066BD1D
:104F2B0012D1DE12CA4C9066E912D1FA9066C51204
:104F3B00D1C290669512D1DE12CA4C9066CD12D1B9
:104F4B00FA9068BA12D1C212CC5B9066BD12D1DE58
:104F5B0012CA4C9066C512D1DE12CB5590690E1257
:104F6B00D1FA90669D12D1C29068BA12D1DE12CAE4
:104F7B004C9066C112D1DE12CA4C9066C512D1DEBE
:104F8B0012CB5590691212D1FA90668912D1C29048
:104F9B0066E912D1DE12CA4CC004C005C006C007B8
:104FAB0090667912D1C29066D912D1DE12CA4CD05A
:104FBB0003D002D001D00012C95B9068CA12D1FA9B
:104FCB0090668D12D1C29066E912D1DE12CA4CC026
:104FDB0004C005C006C00790667D12D1C29066D989
:104FEB0012D1DE12CA4CD003D002D001D00012C9AC
:104FFB005B9068CE12D1FA90669112D1C29066E99D
:10500B0012D1DE12CA4CC004C005C006C0079066A0
:10501B008112D1C29066D912D1DE12CA4CD003D004
:10502B0002D001D00012C95B9066FD12D1FA9066D6
:10503B008912D1C290691212D1DE12CA4CC004C0BF
:10504B0005C006C00790667912D1C290690E12D1C5
:10505B00DE12CA4CD003D002D001D00012C95B9033
:10506B0068D212D1FA90668D12D1C290691212D108
:10507B00DE12CA4CC004C005C006C00790667D1284
:10508B00D1C290690E12D1DE12CA4CD003D002D01D
:09509B0001D00012C95B9068D637
:1050A40012D1FA90669112D1C290691212D1DE1215
:1050B400CA4CC004C005C006C00790668112D1C2A4
:1050C40090690E12D1DE12CA4CD003D002D001D0A6
:1050D4000012C95B9068DA12D1FA7FB77E597D80DD
:1050E4007C3F9065CE12D1DE12CA4C90659E12D1DF
:1050F400DE12C95B90670912D1FA90670912D1C216
:1051040012E314A804A905AA06AB0790670912D1F3
:10511400C212C9577BDB7A0F79C9784012CA4C9006
:10512400670912D1FA90670912D1C212DFD47B0049
:105134007A00798078BF12CA4C90670D12D1FA9028
:10514400670912D1C212DFBE90671112D1FA9067BB
:105154000D12D1C29068CE12D1DE12CA4CC004C066
:1051640005C006C00790671112D1C29068CA12D157
:10517400DE12CA4CD003D002D001D00012C957901D
:1051840066D512D1FA90671112D1C29068CE12D1AD
:10519400DE12CA4CC004C005C006C00790670D12D9
:1051A400D1C29068CA12D1DE12CA4CD003D002D048
:1051B40001D00012C95B9066E512D1FA9066FD1227
:1051C400D1C29066F512D1FA90670D12D1C29068DF
:1051D400D612D1DE12CA4CC004C005C006C0079066
:1051E400671112D1C29068D212D1DE12CA4CD00318
:1051F400D002D001D00012C9579068BE12D1FA90E3
:10520400671112D1C29068D612D1DE12CA4CC00402
:10521400C005C006C00790670D12D1C29068D212B3
:10522400D1DE12CA4CD003D002D001D00012C95B27
:105234009068C212D1FA9068DA12D1C29068C6128C
:10524400D1FA9066DD12D1DE9066D512D1C212C9B0
:10525400579066E112D1FA9066ED12D1DE9066E5C0
:1052640012D1C212C9579066F112D1FA9067011295
:10527400D1DE9066F512D1C212C95790670512D1DA
:10528400FA9066F112D1C29066F112D1DE12CA4CC4
:10529400C004C005C006C0079066E112D1C2906682
:1052A400E112D1DE12CA4CD003D002D001D00012D8
:1052B400C95BC004C005C006C00790670512D1C20F
:1052C40090670512D1DE12CA4CD003D002D001D0AF
:0D52D4000012C95B12DECE90672D12D1FAD8
:1052E10090672112D1C29066F112D1DE12CA4C90A0
:1052F100671D12D1DE12CA4CC004C005C006C0072A
:1053010090672512D1C29066E112D1DE12CA4C908B
:10531100671D12D1DE12CA4CD003D002D001D000D9
:1053210012C95BC004C005C006C00790671912D13D
:10533100C290670512D1DE12CA4CD003D002D0014F
:10534100D00012C95B90673112D1FA90672512D152
:10535100C29066E112D1DE12CA4C90671912D1DEF9
:1053610012CA4C7B007A00798078BF12CA4CC00403
:10537100C005C006C00790672112D1C29066F11224
:10538100D1DE12CA4C90671912D1DE12CA4CA804A0
:10539100A905AA06AB07D007D006D005D00412C9CB
:1053A10057C004C005C006C00790671D12D1C29046
:1053B100670512D1DE12CA4CD003D002D001D00051
:1053C10012C95B90673512D1FA90672112D1C29050
:1053D10066E112D1DE12CA4CC004C005C006C00786
:1053E10090672512D1C29066F112D1DE12CA4CD05B
:1053F10003D002D001D00012C95790673912D1FAF7
:1054010090672D12D1DE90673112D1C212CB559027
:10541100672912D1FA90672912D1C290672912D156
:10542100DE12CA4CA804A905AA06AB077F007E00BC
:105431007D807C3F12C95712DECE90673D12D1FAB2
:1054410090673D12D1DE90672912D1C212CB55125D
:10545100E11E7B357AFA798E783C12CB5590674103
:1054610012D1FA90673512D1DE90673912D1C2128A
:10547100CB5512E11E7B357AFA798E783C12CB55E9
:1054810090674912D1FA9066CD12D1DE9066F5127D
:10549100D1C212CB5590674512D1FA90674512D10E
:1054A100C290674512D1DE12CA4CA804A905AA060A
:1054B100AB077F007E007D807C3F12C95712DECE94
:1054C100A804A905AA06AB0790674512D1C212CB61
:1054D1005512E11E7B337A337965784212CA4C90BA
:1054E100674D12D1FA9066D512D1DE9066E512D1E0
:1054F100C212CB5512E11E7B337A337965784212A1
:10550100CA4C90675112D1FA7F007E007D007C0069
:105511009066D512D1DE12CBEE501A90675112D19E
:10552100DE7F007E007D347C4312C95790675112A3
:10553100D1FA0256157F007E007D007C009066D571
:1055410012D1DE12CBEE602F402D7F007E007D0058
:0B5551007C009066E512D1DE12CBEE6C
:10555C00501A90675112D1C27B007A00798078BFC3
:10556C0012CA4C90675112D1FA0256157F007E0078
:10557C007D007C009066D512D1DE12CBEE603040FF
:10558C002E7F007E007D007C009066E512D1DE123D
:10559C00CBEE601B401990675112D1DE7F007E006C
:1055AC007DB47C4312C95790675112D1FA805A7F4F
:1055BC00007E007D007C009066D512D1DE12CBEE11
:1055CC00701BFFFEFDFC9066E512D1DE12CBEE40A7
:1055DC000C90675112D20643870000802C7F007E0E
:1055EC00007D007C009066D512D1DE12CBEE7019D6
:1055FC00FFFEFDFC9066E512D1DE12CBEE500A9058
:10560C00675112D20642B400007F007E007D347CCC
:10561C004390675112D1DE12CBEE501990675112A4
:10562C00D1C27B007A00798078BF12CA4C90675146
:10563C0012D1FA802A7F007E007D347C4390675122
:10564C0012D1DE12CBEE401790675112D1DE7F00E3
:10565C007E007DB47C4312C95790675112D1FA7FFA
:10566C00007E007D007C0090673512D1DE12CBEEFF
:10567C00501A90674912D1C27B007A007934784372
:10568C0012C95B90674912D1FA0257337F007E0032
:10569C007D007C0090673512D1DE12CBEE602E407F
:1056AC002C7F007E007D007C0090673912D1DE12C9
:1056BC00CBEE50197F007E007DB47C43906749127D
:1056CC00D1DE12C95B90674912D1FA805A7F007EF5
:1056DC00007D007C0090673512D1DE12CBEE701B82
:1056EC00FFFEFDFC90673912D1DE12CBEE400C9020
:1056FC00674912D20642B40000802C7F007E007DE8
:10570C00007C0090673512D1DE12CBEE7019FFFED3
:10571C00FDFC90673912D1DE12CBEE500A9067492E
:10572C0012D2064387000090676112D1DE9068C2E6
:10573C0012D1C212C9579066F112D1DE12CA4CC0F6
:10574C0004C005C006C00790675D12D1DE9068BE2C
:10575C0012D1C212C9579066E112D1DE12CA4CD0D6
:10576C0003D002D001D00012C95BC004C005C00632
:10577C00C00790670512D1C29068C612D1DE12CA5A
:10578C004CD003D002D001D00012C95B90672D120F
:10579C00D1DE12CB559068FE12D1FA7F007E007DCF
:1057AC00807CBF9065C612D1DE12CA4C9068FE1286
:1057BC00D1DE12CA4C7B207A7B7955784012CA4CC8
:1057CC0090675912D1FA900007E020E4030258D1F7
:1057DC007B007A40791C784690675912D1C212CB63
:1057EC005512CCAA90691612D1FA90675912D1C2EF
:1057FC0012CCAA7B107A277900780012E87BAC00D7
:10580C00AD01AE02AF0390691A12D1FA7F107E2758
:10581C007D007C0090691612D1DE12D12490691E95
:10582C0012D1FA7FC47E097D007C0090691A12D1D6
:01583C00DE8D
:10583D00C312D181501290691E12D1C2EC12CC6CE0
:10584D0090675912D1FA80507F4C7E1D7D007C00EF
:10585D0090691A12D1DEC312D181401F90691E12B8
:10586D00D1C2EF2410FFEE3427FEE43DFDE43CFCF5
:10587D0012CC6C90675912D1FA801D90691E12D10D
:10588D00C2EF2488FFEE3413FEE43DFDE43CFC1230
:10589D00CC6C90675912D1FA7F007E007D007C00A0
:1058AD009068FE12D1DE12CBEE6019401790675949
:1058BD0012D1C27B007A00798078BF12CA4C9067F2
:1058CD005912D1FA7F007E247D747C499065C612F1
:1058DD00D1DE12CA4C12CCAAC004C005C006C00746
:1058ED0090675912D1C212CCAAD003D002D001D0E8
:1058FD000012D10990664112D1DE12D1099066597C
:10590D0012D1FA90665912D1DEC000C001C002C09A
:10591D00039068B5E0FF3395E0FEEF7802C333CE18
:10592D0033CED8F9246DF582EE3413F58312D1C23E
:10593D007B007A247974784912CA4C12CCAAD00310
:10594D00D002D001D00012D10990665912D1FA902F
:10595D00665912D1DEC000C001C002C0039068B507
:10596D00E0FF3395E0FEEF7802C333CE33CED8F9A6
:10597D00244DF582EE3415F58312D1C212CCAAD086
:10598D0003D002D001D00012D10990665912D1FA7C
:10599D007F007E007D807CBF9065CA12D1DE12CA69
:1059AD004C9068FE12D1DE12CA4C7B207A7B795561
:1059BD00784012CA4C90675512D1FA7F007E247D33
:1059CD00747C499065CA12D1DE12CA4C12CCAAC0A1
:1059DD0004C005C006C00790675512D1C212CCAAEB
:1059ED00A804A905AA06AB07D007D006D005D00498
:1059FD0012D11690665D12D1FA90665D12D1DEC09D
:105A0D0000C001C002C0039068B5E0FF3395E0FE11
:105A1D00EF7802C333CE33CED8F9245DF582EE3460
:105A2D0014F58312D1C27B007A247974784912CA95
:105A3D004C12CCAAD003D002D001D00012D10990C3
:105A4D00665D12D1FA9065D612D1C212E220C00461
:105A5D00C005C006C0079065CE12D1C212E220A8C3
:105A6D0004A905AA06AB07D007D006D005D00412AD
:105A7D00CBEE602E9065D212D1C27B007A00798078
:105A8D00783F12C95B9065D212D1FA9065D612D1CA
:105A9D00C27B007A007980783F12C95B9065D6127F
:035AAD00D1FA2209
:105AB000900599E4F0A3740DF090061112D20643FC
:105AC0007F8412900AC112D20600012F689007014C
:105AD00012D206421DE9449007F112D206414893C2
:105AE000619008E112D20642CAE17C9009D112D23B
:105AF000063AA170FE900BB112D20642E8998C9042
:105B00000CA112D2064371E0AA900D9112D206B4F4
:105B10009652E8900E8112D20643D98F5C900F7195
:105B200012D2064311E666900F7512D2064311F9A0
:105B30009A900F7912D2064311E666900F7D12D229
:105B4000064311E6669016797404F090163DF090C5
:105B500016B6E054FEF054FDFFF0FB90145D12D237
:105B6000060000000090136D12D20600000000EB4A
:105B700044109016B6F078E97C007D017BFF7AB581
:105B800079407E007F0612CFF390059BE4F0A3746A
:105B90000DF090061512D206437E8AC4900AC512F3
:105BA000D20600012F9D90070512D20643A1E9C736
:105BB0009007F512D2064164A8C59008E512D206F6
:105BC00041FB78A19009D512D2063D0FDDA9900BBB
:105BD000B512D2064341FB3D900CA512D206439567
:105BE00055B5900D9512D20636A5C247900E851276
:105BF000D20643D99666900F8112D2064311D99AE4
:105C0000900F8512D2064311E666900F8912D206D4
:105C10004311E666900F8D12D2064311E666901688
:105C20007A7404F090163EF09016B8E054FEF054EA
:105C3000FDF04410F090146112D2060000000090B4
:105C4000137112D2060000000078FD7C007D017BFC
:105C5000FF7AB579477E007F0612CFF390059DE469
:105C6000F0A3740DF090061912D206437EBE349054
:105C70000AC912D2060001494D90070912D2064303
:105C80002A3E229007F912D20641587B179008E964
:105C900012D20642C517669009D912D2063D0F27C7
:105CA000A0900BB912D2064395F3EB900CA912D237
:105CB000064396D8BE900D9912D20633D6BF959062
:105CC0000E8912D20643D9F47B900F9112D206436B
:105CD00011DEB8900F9512D2064311D99A900F9900
:105CE00012D2064311E3D7900F9D12D2064311E85A
:105CF000F690167B7404F090163FF09016BAE054BC
:105D0000FEF054FDFFF0FB90146512D20600000077
:105D10000090137512D20600000000EB441090169C
:105D2000BAF078117C017D017BFF7AB5794E7E0057
:105D30007F0612CFF3E490172DF0A304F0A304F034
:105D40007F03EFC3943C500F742D2FF582E434177A
:105D5000F583EFF00F80EB906776743CF0906775F9
:025D6000F0222F
:105D62007BFF7AB579551208777BFF7AB5795A129B
:105D720008777BFF7AB579841208777BFF7AB57949
:105D8200A01208777BFF7AB579B712087712E8E696
:105D9200AE07EEC39431400BEED394335005EE249C
:0C5DA200D0FF22EE4420B471DB7F7122A0
:105DAE00125D62EF24FE7003025E55147003025EF4
:105DBE00E724927003025EED247070E47BFF7AB5E7
:105DCE0079C912087790E102E04480F0E49067DB35
:105DDE00F030986512E8E6EF24CE603324FD603B88
:105DEE0014601424FE601C2404703D1269C890E1F6
:105DFE0002E04420F080421269BE90E102E04420AD
:105E0E00F080361269E690E102E04420F0802A121A
:105E1E0069F090E102E04420F0801E90E102E0542F
:105E2E00F0F0E054DFF0801190E102E054F0F0E089
:105E3E0054DFF09067DB7401F09067DBE0600302E3
:105E4E005DAE126164808A7BFF7AB6790490660239
:105E5E0012D1C290679212D1FA12D7537B017A6790
:105E6E0079D59068B512D28A7BFF7AA77918120974
:105E7E00A19067D712D1FA9067D5E07002A3E060C7
:105E8E000C9067D712D1C290660212D1FA7BFF7ABC
:105E9E00B6791890660612D1C290679212D1FA1294
:105EAE00D7537B017A6779D59068B512D28A7BFF7A
:105EBE007AA779181209A19067D712D1FA9067D5EF
:105ECE00E07002A3E0600C9067D712D1C290660614
:105EDE0012D1FA125EEE025DAE125F35025DAE2297
:105EEE00900005E04404F090E102E04420F07BFFD6
:105EFE007AB0792612087712670690E102E0540F05
:105F0E00601230980A12E8E6906889EFF080051268
:105F1E00616480E3900005E054FBF090E102E054F0
:075F2E00DFF0E054F0F02267
:105F35007BFF7AB6792C9000C112D1C2906792127C
:105F4500D1FA9000D512D1C290679612D1FA90007D
:105F5500C512D1C290679A12D1FA9000D912D1C256
:105F650090679E12D1FA9000C912D1C29067A21211
:105F7500D1FA9000DD12D1C29067A612D1FA900035
:105F8500CD12D1C29067AA12D1FA9000E112D1C206
:105F95009067AE12D1FA12D7537BFF7AB6796D901E
:105FA50000D112D1C290679212D1FA9000E512D1B8
:105FB500C290679612D1FA12D7537BFF7AB6797DD4
:105FC50012087712E8E69067DCEFF0C394314040A1
:105FD500E0FFD394355039EF24CFF0E0FB25E025E1
:105FE500E024C1F582E43400F58312D1C290660243
:105FF50012D1FAEB25E025E024D5F582E43400F54D
:106005008312D1C290660612D1FA125EEE025F3596
:106015009067DCE04420647360030261569067E397
:10602500F0A3F0C39067E4E094059067E3E0940083
:106035004003025F357BFF7AB67994E0FEA3E0FF6B
:106045002401906793F0E43E906792F0EF7802C3E5
:1060550033CE33CED8F924C1F582EE3400F5831260
:10606500D1C290679412D1FA12D7537B017A67791E
:10607500E19068B512D28A7BFF7AA779181209A137
:106085009067DD12D1FA9067E1E07002A3E060321B
:106095009067DD12D1C2C004C005C006C007906775
:1060A500E3E0FEA3E07802C333CE33CED8F924C1B2
:1060B500F582EE3400F583D007D006D005D0041262
:1060C500D1FA7BFF7AB679B49067E3E0FEA3E07876
:1060D50002C333CE33CED8F924D5F582EE3400F59C
:1060E5008312D1C290679212D1FA12D7537B017AEB
:1060F5006779E19068B512D28A7BFF7AA779181281
:1061050009A19067DD12D1FA9067E1E07002A3E082
:1061150060329067DD12D1C2C004C005C006C00759
:106125009067E3E0FEA3E07802C333CE33CED8F91F
:1061350024D5F582EE3400F583D007D006D005D0FE
:106145000412D1FA9067E3E475F00112D0BE026043
:0F615500289067DCE0442064716003025F35220C
:10616400E4FF120A8A9065E6E0FEA3E0FFC3E52996
:106174009FFFE5289EFEEF252BF52BEE352AF52A09
:10618400A2E713F52AE52B13F52B9068D6E528F042
:10619400A3E529F07F01120A8A9065EAE0FEA3E0F4
:1061A400FFC3E5299FFFE5289EFEEF252DF52DEE83
:1061B400352CF52CA2E713F52CE52D13F52D90685D
:1061C400D8E528F0A3E529F0AC2AAD2BEC12CC716C
:1061D4009065E212D1DE12CB559068CE12D1FAACA2
:1061E4002CAD2DEC12CC719065DE12D1DE12CB55A4
:1061F4009068D212D1FA900005E020E3457F007E3A
:10620400007D347C439068CE12D1DE12CBEE601B4D
:1062140040199068CE12D1C27B007A007934784359
:1062240012C9579068CE12D1FA80179068CE12D155
:10623400C27B007A007934784312C95B9068CE122D
:10624400D1FA7BFF7AB679D19068D6E0FFA3E090CB
:106254006792CFF0A3EFF09068CE12D1C29067940A
:1062640012D1FA9068D8E0FFA3E0906798CFF0A32A
:10627400EFF09068D212D1C290679A12D1FA12D775
:10628400537BFF7AB3792990679212D28A9068CEB1
:1062940012D1C290679512D1FA9068D212D1C290ED
:1062A400679912D1FA7B017A6879B012D74D7FC011
:0D62B4001202A07B017A6879B012089522D1
:1062C1007BFF7AB679FC1208777BFF7AB7793C12AB
:1062D100087712E8E69067D5EFF044206473600315
:1062E1000263827BFF7AB7796C90001CE0FFA3E028
:1062F100906792CFF0A3EFF012D7537B017A6779C1
:10630100D69068B512D28A7BFF7AA779181209A1B3
:106311009067D812D1FA9067D6E07002A3E06011BD
:106321009067D812D1C212CCAA90001CEEF0A3EF54
:10633100F07BFF7AB7799490001EE0FFA3E09067AD
:1063410092CFF0A3EFF012D7537B017A6779D69001
:1063510068B512D28A7BFF7AA779181209A19067D2
:10636100D812D1FA9067D6E07002A3E0605D906721
:10637100D812D1C212CCAA90001EEEF0A3EFF08089
:106381004A9067D5E04420646D70407BFF7AB7790D
:10639100B71208777BFF7AB0792612087730980F09
:1063A10012E8E6EF44202492700302647D8000121B
:1063B100647E80E930980F12E8E6EF442024927061
:1063C1000302647D800012647E80E97B017A677933
:1063D100D690683012D28A7BFF7AB8791C12096A8A
:1063E1009067D6E07002A3E0600CEE3395E0FDFC0F
:1063F10090678112D1FA7BFF7AB8793A1208771245
:10640100E8E69067D5EFF04420FFB47909900007E2
:10641100E04402F0800BEFB46E07900007E054FDFA
:10642100F07BFF7AB8796512087712E8E6EF44202D
:106431002492600D24F57010900007E04405F0806F
:1064410007900007E054FBF07BFF7AB879961208B9
:106451007712E8E6EF44202492601324FC701D902B
:106461000007E04408F090E102E04450F02290007F
:0D64710007E054F7F090E102E054AFF02294
:10647E007F03120A8A7BFF7AB879CA906792E52861
:09648E00F0A3E529F012D7532216
:106497009068B0EEF0A3EFF0900005E020E23C90AA
:1064A700E102E054F0F012083A90662612D1C29049
:1064B700660612D1DE12CBEE6019401790E000E0BD
:1064C70030E00890E102E04420F02290E102E0543D
:1064D700DFF02290E102E054DFF02290662612D12D
:1064E700C290660612D1DE12CBEE400302658A7FA8
:1064F700007E007D407CC090660612D1DE12CBEE96
:10650700401790E000E030E00990E102E04420F01D
:10651700800790E102E054DFF07F007E007D407C41
:10652700C090660612D1DE12CBEE502190E102E058
:1065370054DFF0900007E020E01390677912D1C292
:1065470090677D12D1FA900007E04401F0900005B2
:10655700E030E42490662A12D1C290660612D1DE9A
:1065670012CBEE50139068B1E0FF129EBC90660606
:1065770012D206C17000002212083A90E102E054DC
:10658700F0F022900005E030E042A3E0A330E02BDA
:106597007FCD7ECC7DCC7C3D9065C612D1DE12CB03
:1065A700EE60184016900007E030E10F9068B1E008
:1065B700FF123A3E900006E054FEF0900006E0FE1F
:1065C700A3E0FF30E20630E003123802906659126A
:1065D700D1C290677D12D1FA90677912D1FA90E112
:1065E70002E04420F0900005E020E50302670290F6
:1065F700661E12D1C290660612D1DE12CBEE601073
:10660700400E90661E12D1C290660612D1FA801D06
:1066170090661A12D1C290660612D1DE12CBEE50E6
:106627000C90661A12D1C290660612D1FA906612C1
:1066370012D1C290661612D1DE12CBEE60464044EC
:1066470090661612D1C290660212D1DE12CBEE60AE
:1066570011400F90661612D1C290660212D1FA024B
:10666700670290661212D1C290660212D1DE12CB77
:10667700EE400302670290661212D1C290660212C0
:10668700D1FA807790661212D1C290661612D1DEC7
:1066970012CBEE506690661212D1C290660212D1EA
:1066A700DE12CBEE50237F007E007D347C43906664
:1066B7000212D1DE12CBEE6010400E90661212D19C
:1066C700C290660212D1FA803290661612D1C29039
:1066D700660212D1DE12CBEE6021401F7F007E00E2
:1066E7007D347C4390660212D1DE12CBEE500C90C3
:0F66F700661612D1C290660212D1FA12670622FD
:10670600E4FF120A8A9065E6E0FEA3E0FFC3E529EE
:106716009FFFE5289EFEEF252BF52BEE352AF52A61
:10672600A2E713F52AE52B13F52B7F01120A8A90AF
:1067360065EAE0FEA3E0FFC3E5299FFFE5289EFE8C
:10674600EF252DF52DEE352CF52CA2E713F52CE5CE
:106756002D13F52DAC2AAD2BEC12CC719065E212FF
:10676600D1DE12CB559068B312D1FAAC2CAD2DEC1C
:1067760012CC719065DE12D1DE12CB559068B7123D
:10678600D1FA900005E020E3457F007E007D347C51
:106796004390660212D1DE12CBEE50197F007E00C6
:1067A6007D347C4390660212D1DE12C95B9068BBD1
:1067B60012D1FA80257F007E007D347CC39066026C
:1067C60012D1DE12C95B9068BB12D1FA800C9066BA
:1067D6000212D1C29068BB12D1FA90660612D1C2DB
:1067E6009068BF12D1FA9068BB12D1C29065EE12C2
:1067F600D1DE12C95B9068BB12D1FA9068BF12D184
:10680600C29065F212D1DE12C95B9068BF12D1FA4E
:10681600900006E0A330E52E9068BB12D1C27B0043
:106826007A007934784312C95B9068BB12D1FA902A
:1068360068BF12D1DE7F007E007D347C4312C957CB
:106846009068BF12D1FA7F007E007DB47C439068C9
:10685600BB12D1DE12CBEE601B40199068BB12D181
:10686600C27B007A0079B4784312C9579068BB128C
:10687600D1FA802A7F007E007D007C009068BB12E2
:10688600D1DE12CBEE50179068BB12D1C27B007AD4
:106896000079B4784312C95B9068BB12D1FA7F00C5
:1068A6007E007D347C439068BF12D1DE12CBEE4071
:1068B6000C9068BF12D20643340000801F7F007E12
:1068C600007D007C009068BF12D1DE12CBEE600224
:1068D600500A9068BF12D206000000009068BB12F2
:1068E600D1DE9068B312D1C212C95712DE74C00449
:1068F600C005C006C0077F007E007D407C409065D5
:10690600F612D1DE12CA4CA804A905AA06AB07D016
:1069160007D006D005D00412CBEE500990E102E074
:106926004480F0800790E102E0547FF09068BB124B
:10693600D1DE9068B312D1C212C95712DE749065C7
:10694600F612D1DE12CBEE501D9068B312D1C29072
:1069560068BB12D1DE12CBEE600740051269BE801D
:10696600081269C880031269D29068BF12D1DE90FE
:0869760068B712D1C212C95723
:10697E0012DE749065FA12D1DE12CBEE502E9068B4
:10698E00B712D1C29068BF12D1DE12CBEE600640B4
:10699E00041269E6227F007E007D007C009068BFB5
:1069AE0012D1DE12CBEE40071269F0221269FA22E2
:0A69BE0090E102E054FC4402F022D4
:0A69C80090E102E054FC4401F022CB
:1069D20090676512D1C290676912D1FA90E102E024
:0469E20054FCF0224F
:0A69E60090E102E054F34408F022AF
:0A69F00090E102E054F34404F022A9
:1069FA0090676512D1C290676D12D1FA90E102E0F8
:046A0A0054F3F0222F
:106A0E007BFF7AB879E49065E6E0FFA3E0906792A9
:106A1E00CFF0A3EFF09065E8E0FFA3E0906794CF8E
:106A2E00F0A3EFF09065EAE0FFA3E0906796CFF059
:106A3E00A3EFF09065ECE0FFA3E0906798CFF0A392
:106A4E00EFF012D7537BFF7AB9791E1209D89067EF
:106A5E00D5EFF0B4010C900006E04440F0A3E0F056
:106A6E00800D9067D5E07007900006E054BFF07B74
:106A7E00FF7AB9794E1209D89067D5EFF0640160AC
:106A8E00079067D5E070E822E4FF120A8A9065E667
:106A9E00E528F0A3E529F07F01120A8A9065EAE560
:106AAE0028F0A3E529F07BFF7AB979911209D890E5
:106ABE0067D5EFF0640160079067D5E070E822E4D7
:106ACE00FF120A8A9065E8E528F0A3E529F07F0118
:106ADE00120A8A9065ECE528F0A3E529F01204E687
:016AEE002285
:106AEF007BFF7AB979D39065E6E0FFA3E0906792D8
:106AFF00CFF0A3EFF09065E8E0FFA3E0906794CFAD
:106B0F00F0A3EFF012D7537B017A6779D59068B570
:106B1F0012D28A7BFF7AB979F81209A19067D7123E
:106B2F00D1FA9067D5E07002A3E060119067D71299
:106B3F00D1C212CCAA9065E6EEF0A3EFF07B017AFA
:106B4F006779D59068B512D28A7BFF7ABA7911121C
:106B5F0009A19067D712D1FA9067D5E07002A3E030
:106B6F0060119067D712D1C212CCAA9065E8EEF0EF
:106B7F00A3EFF07BFF7ABA79291209D8EFB4010C91
:106B8F00900006E04440F0A3E0F0800AEF70079019
:106B9F000006E054BFF07BFF7ABA79589065EAE0BF
:106BAF00FFA3E0906792CFF0A3EFF09065ECE0FFCA
:106BBF00A3E0906794CFF0A3EFF012D7537B017A45
:106BCF006779D59068B512D28A7BFF7ABA797D1230
:106BDF0009A19067D712D1FA9067D5E07002A3E0B0
:106BEF0060119067D712D1C212CCAA9065EAEEF06D
:106BFF00A3EFF07B017A6779D59068B512D28A7BC3
:106C0F00FF7ABA79961209A19067D712D1FA9067D5
:106C1F00D5E07002A3E060119067D712D1C212CCF9
:0D6C2F00AA9065ECEEF0A3EFF01204E6224F
:106C3C007BFF7ABA79AE12087712E8E6EF4420901F
:106C4C0067DDF064796003026E20900005E044106B
:106C5C00F07BFF7ABA79DA90660A12D1C290679209
:106C6C0012D1FA12D7537B017A6779D59068B51295
:106C7C00D28A7BFF7AA779181209A19067D912D111
:106C8C00FA9067D5E07002A3E0600C9067D912D13E
:106C9C00C290660A12D1FA7BFF7ABA79FF90660E1F
:106CAC0012D1C290679212D1FA12D7537B017A6734
:106CBC0079D59068B512D28A7BFF7AA77918120918
:106CCC00A19067D912D1FA9067D5E07002A3E06069
:106CDC000C9067D912D1C290660E12D1FA7BFF7A52
:106CEC00BB792012087712E8E6EF44209067DDF0BC
:106CFC0064796003026E17900006E04402F0A3E092
:106D0C00F07BFF7ABB794B90664512D1C2906792AB
:106D1C0012D1FA12D7537B017A6779D59068B512E4
:106D2C00D28A7BFF7AA779181209A19067D912D160
:106D3C00FA9067D5E07002A3E0600C9067D912D18D
:106D4C00C290664512D1FA7BFF7ABB796690664990
:106D5C0012D1C290679212D1FA12D7537B017A6783
:106D6C0079D59068B512D28A7BFF7AA77918120967
:106D7C00A19067D912D1FA9067D5E07002A3E060B8
:106D8C000C9067D912D1C290664912D1FA7BFF7A66
:106D9C00BB797F12D7537B017A6779DE1208F2EF49
:106DAC004E60289067DEE04420249A601824F1603D
:106DBC000C240970169066587401F0800E90665879
:106DCC007402F080069066587404F07BFF7ABB79ED
:106DDC00A012D7537B017A6779DE1208F2EF4E606E
:106DEC00419067DEE04420249A601824F1600C2462
:106DFC0009702F9066577401F080279066577402C3
:106E0C00F0801F9066577404F08017900006E054D1
:106E1C00FDF0800E9067DDE0B46E07900005E05445
:106E2C00EFF07BFF7ABB79C112087712E8E6EF44EA
:106E3C00209067DDF064796003026F69900005E0D3
:106E4C004420F07BFF7ABB79E990661212D1C29094
:106E5C00679212D1FA12D7537B017A6779D5906871
:106E6C00B512D28A7BFF7AA779181209A19067D93B
:106E7C0012D1FA9067D5E07002A3E0600C9067D94C
:106E8C0012D1C290661212D1FA7BFF7ABC790E90A5
:106E9C00661612D1C290679212D1FA12D7537B01A7
:106EAC007A6779D59068B512D28A7BFF7AA7791860
:106EBC001209A19067D912D1FA9067D5E07002A39C
:106ECC00E0600C9067D912D1C290661612D1FA7B91
:106EDC00FF7ABC792F90661A12D1C290679212D1A8
:106EEC00FA12D7537B017A6779D59068B512D28A9A
:106EFC007BFF7AA779181209A19067D912D1FA9061
:106F0C0067D5E07002A3E0600C9067D912D1C290F3
:106F1C00661A12D1FA7BFF7ABC795090661E12D198
:106F2C00C290679212D1FA12D7537B017A6779D546
:106F3C009068B512D28A7BFF7AA779181209A190B2
:106F4C0067D912D1FA9067D5E07002A3E0601C906B
:106F5C0067D912D1C290661E12D1FA800E9067DDED
:106F6C00E0B46E07900005E054DFF07BFF7ABC794B
:106F7C007112087712E8E6EF44209067DDF064792F
:106F8C006003027035900006E054F7F07BFF7ABC8A
:106F9C00799B906771E0FFA3E0906792CFF0A3EF2D
:106FAC00F012D7537B017A6779D590683012D28A68
:106FBC007BFF7AA7791812096A9067D7EEF0A3EFD6
:106FCC00F09067D5E07002A3E0600F9067D7E0FF08
:106FDC00A3E0906771CFF0A3EFF07BFF7ABC79CA86
:106FEC00906773E0FFA3E0906792CFF0A3EFF012ED
:106FFC00D7537B017A6779D590683012D28A7BFFA0
:10700C007AA7791812096A9067D7EEF0A3EFF0907F
:10701C0067D5E07002A3E060219067D7E0FFA3E0A2
:10702C00906773CFF0A3EFF0229067DDE0B46E0AA7
:0B703C00900006E04408F0A3E0F02202
:107047007BFF7ABD79039065F612D1C290679212E1
:10705700D1FA12D7537B017A6779D59068B512D2E6
:107067008A7BFF7AA779181209A19067D712D1FAFC
:107077009067D5E07002A3E0600C9067D712D1C289
:107087009065F612D1FA7BFF7ABD79259065FA12E1
:10709700D1C290679212D1FA12D7537B017A6779DE
:1070A700D59068B512D28A7BFF7AA779181209A101
:1070B7009067D712D1FA9067D5E07002A3E0600C11
:1070C7009067D712D1C29065FA12D1FA7BFF7ABDC9
:1070D70079439065EE12D1C290679212D1FA12D716
:1070E700537B017A6779D59068B512D28A7BFF7A8C
:1070F700A779181209A19067D712D1FA9067D5E03E
:107107007002A3E0600C9067D712D1C29065EE12AF
:10711700D1FA7BFF7ABD79639065F212D1C290678D
:107127009212D1FA12D7537B017A6779D59068B555
:1071370012D28A7BFF7AA779181209A19067D71212
:10714700D1FA9067D5E07002A3E0600C9067D71280
:09715700D1C29065F212D1FA22B6
:1071600078D57C677D017BFF7AC779987E007F099F
:1071700012CFF378DE7C677D017BFF7AC779A17E31
:10718000007F0612CFF378E47C677D017BFF7AC72E
:1071900079A77E007F0F12CFF378F37C677D017BA8
:1071A000FF7AC779B67E007F0612CFF378F97C6745
:1071B0007D017BFF7AC779BC7E007F1212CFF390EE
:1071C0000004E0FFA3E090680BCFF0A3EFF07BFF9B
:1071D0007AB579551208777B017A17796A906792A8
:1071E00012D28A90000A12D1C290679512D1FA90F9
:1071F000000E12D1C290679912D1FA90001612D1E6
:10720000C290679D12D1FA7BFF7ABD79B312D75332
:107210007BFF7ABD79EB9065E6E0FFA3E090679293
:10722000CFF0A3EFF09065E8E0FFA3E0906794CF84
:10723000F0A3EFF09065EAE0FFA3E0906796CFF04F
:10724000A3EFF09065ECE0FFA3E0906798CFF0A388
:10725000EFF012D753900006E0A330E6097BFF7AE7
:10726000BE791C12D7537BFF7AB0792612D7537B95
:10727000FF7ABE79239065F612D1C290679212D13F
:10728000FA9065FA12D1C290679612D1FA12D753CA
:107290007BFF7ABE79569065EE12D1C2906792124A
:1072A000D1FA9065F212D1C290679612D1FA12D734
:1072B00053900005E020E4030273467BFF7ABE7919
:1072C0008990660A12D1C290679212D1FA90660E26
:1072D00012D1C290679612D1FA12D753900006E0ED
:1072E000A330E15790664512D1C290679212D1FA4D
:1072F00090664912D1C290679612D1FA906658E012
:1073000075F003A424E4F582E43467F58312D253C4
:1073100090679A12D28A906657E075F003A424E42D
:10732000F582E43467F58312D25390679D12D28AB6
:107330007BFF7ABE79BC12D75380147BFF7ABE796B
:10734000F812087780097BFF7ABF791112D7539022
:107350000005E030E53B7BFF7ABF792A9066121288
:10736000D1C290679212D1FA90661612D1C290677C
:047370009612D1FAA6
:1073740090661A12D1C290679A12D1FA90661E12C0
:10738400D1C290679E12D1FA12D75380097BFF7A3B
:10739400BF796512D7537BFF7ABF797E9066261238
:1073A400D1C290679212D1FA90662A12D1C2906724
:1073B4009612D1FA90662E12D1C290679A12D1FA1F
:1073C40012D753900006E0A330E30B7BFF7ABF791A
:1073D400C012087780397BFF7ABF79DE906771E04D
:1073E400FFA3E0906792CFF0A3EFF012D75390671A
:1073F40073E0FEA3E0FFC3943DEE940050117BFFC5
:107404007AC0790A906792EEF0A3EFF012D7539006
:107414006632E075F003A424D5F582E43467F5837D
:1074240012D25390679212D28AE4FE90680CE05410
:10743400807807CEC313CE13D8F99067F375F003A1
:1074440012D237EE75F003A42583F58312D253903C
:10745400679512D28A7BFF7AC0793C12D753906623
:1074640032E014601914604A2402706E900007E040
:1074740030E5677BFF7AC07955120877805C90000D
:1074840009E030E10B7BFF7AC07961120877801044
:10749400900009E030E2097BFF7AC0796A1208772C
:1074A400900005E030E6337BFF7AC07973120877E9
:1074B40080287BFF7AC0797F906635E0906792F0F0
:1074C400906636E0906793F0900000E0FFA3E090B0
:1074D4006794CFF0A3EFF012D75390002EE075F02D
:1074E40003A424FCF582E43467F58312D253906735
:1074F4009212D28A7BFF7AC0799212D7537BFF7A99
:10750400C0799690001CE0FFA3E0906792CFF0A3AF
:10751400EFF090001EE0FFA3E0906794CFF0A3EF9C
:10752400F012D7537BFF7AC079C690678112D1C21B
:1075340090679212D1FA12D753E4FE90680CE0548B
:10754400087803CEC313CE13D8F99067DE75F00321
:1075540012D237EE75F003A42583F58312D253902B
:10756400679212D28A7BFF7AC079E112D7539000D6
:107574002DE075F003A424F9F582E43467F5831251
:10758400D25390679212D28A7BFF7AC079F912D7CC
:0E759400537BFF7AC1791E12D75312E8E6220C
:1075A2009067D5EEF0A3EFF0E490680CF0A3F090B2
:1075B200681512D2063F80000090681912D20600A8
:1075C2000000009067D6E0FF1243C91241D37BFF4F
:1075D2007AC1793C906792E52EF0A3E52FF0A3E5FE
:1075E20030F0A3E531F0A3E532F0A3E533F0A3E5F3
:1075F20034F012D7537BFF7AC17962120877E49094
:1076020067E9F09067E6F07B017A6779E41208F2A5
:107612009067E9E0FF9067E6E04F642F600302762F
:10762200C79067F2E0FF9067EFE04F643A600302B1
:1076320076C79067E4E0FB75F00AA4FFA3E07C0044
:107642002FFFEC35F0CF245C9067DCF0EF3405902F
:1076520067DBF0EB64396007E475F06412D0BE902A
:1076620067E7E024D075F00AA4FFA3E024D02F90AE
:1076720067DDF09067EAE024D075F00AA4FFA3E08A
:1076820024D02F9067DEF09067EDE024D075F00AE9
:10769200A4FFA3E024D02F9067DFF09067F0E024EE
:1076A200D075F00AA4FFA3E024D02F9067E0F090F9
:1076B20067F3E024D075F00AA4FFA3E024D02F9052
:1076C20067E1F0801E9067DBE52EF0A3E52FF0A3C3
:1076D200E530F0A3E531F0A3E532F0A3E533F0A302
:1076E200E534F09067DBE0FEA3E0FFA3E0FDA3E05A
:1076F200FBA3E0906835F09067E0E0906836F09088
:1077020067E1E0906837F0127A357BFF7AC1798BB6
:107712009065CE12D1C290679212D1FA12D7537BE2
:10772200FF7AC179A91208777B017A68790E90688D
:10773200B512D28A7BFF7AC179B51209A190682568
:1077420012D1FA90680EE07002A3E0600C906825F6
:1077520012D1C290681512D1FA7B017A68790E9023
:1077620068B512D28A7BFF7AC179C01209A19068EA
:107772002912D1FA90680EE07002A3E0600C9068C2
:107782002912D1C290681912D1FA90681512D1C289
:107792007B5E7A0B7936783A12CA4C90681512D110
:1077A200FA90681912D1C27B417A2E794278371247
:1077B200CA4C90681912D1FA90681912D1C2906815
:1077C2001512D1DE12C95B90681D12D1FA7BFF7AC5
:1077D200C179F690679212D28A7AC179FB90679545
:1077E20012D28A7AC2790090679812D28A7AC279C2
:1077F2000390679B12D28A7AC2790690679E12D250
:0D7802008A7AC2790C9067A112D28A7AC1ED
:10780F0079CB12D753E49067E3F09067E3E0C3942A
:10781F001640030279FA30980B12E8E6E490680DEF
:10782F00F00279FA9067D6E0FF1249639065CE12A5
:10783F00D1C212CCAAAC06AD079067D9ECF0A3ED7C
:10784F00F0EC12CC71A804A905AA06AB079065CE7F
:10785F0012D1C212C95790682112D1FA7B017A68EE
:10786F00791090683812D28A7A680990683B12D2E0
:10787F008A7A6779D79067D9E0FCA3E0FDA3E0FE91
:10788F00A3E0FF127B9F7B017A687913906838120F
:10789F00D28A7A680990683B12D28A7A68791290F4
:1078AF00682112D1C2127CA87F007E007D807CBF30
:1078BF0090674112D1DE12CBEE6002500302798243
:1078CF007BFF7AC279149067D7E0FFA3E0906792AD
:1078DF00CFF0A3EFF0906810E0906794F0906811EC
:1078EF00E0906795F0906812E0906796F0906813BB
:1078FF00E0906797F0906814E0906798F090674970
:10790F0012D1C290679912D1FA90674112D1C290E9
:10791F00679D12D1FA9066B512D1C29067A112D1AC
:10792F00FA90675912D1C29067A512D1FA12D753A4
:10793F0090682D12D1C290674112D1DE12CBEE604A
:10794F0008400690680C7401F09067E3E004F09033
:10795F0065CE12D1C290681D12D1DE12C95B90653F
:10796F00CE12D1FA90674112D1C290682D12D1FA7E
:10797F0002781990682D12D1C290674112D1DE1290
:10798F00CBEE501590680CE0B4010E7BFF7AC279F4
:10799F0052120877E490680CF07F147E0B7D367CD2
:1079AF003A90681D12D1DE12CBEE60194017906528
:1079BF00CE12D1C290681D12D1DE12C95B9065CE76
:1079CF0012D1FA80179065CE12D1C27B147A0B793F
:1079DF0036783A12C95B9065CE12D1FA9067411290
:1079EF00D1C290682D12D1FA02781990680DE0601B
:1079FF00030277CF7BFF7AC2795F12087712E8E62E
:107A0F009067E2EFF04420FF64716019EF647360D8
:107A1F00030277CF90680D04F07BFF7AB0792612BE
:067A2F0008770277CF2268
:107A3500906831EEF0A3EFF0906831E0FEA3E0FF2F
:107A4500124386AC06AD07E412CC719065D612D10F
:107A5500FA906835E0FCE412CC767B007A0079C0B8
:107A6500784112CB5590683C12D1FA906836E0FC0B
:107A7500E412CC767B007A0079B4784412CB559029
:107A8500684012D1FA906837E0FCE412CC767B00AE
:107A95007AC079A8784712CB5590684412D1FA90EC
:107AA5006831E0FCA3E0FDE412CC719065DA12D1F7
:107AB500DE12C95712CCAA906838EEF0A3EFF04E4B
:107AC5006076A3E4F0A304F0906838E0FEA3E0FF3D
:107AD500A3E0FCA3E0FDD39FEC9E505CC39068320D
:107AE500E09DFF906831E09CEF540370199065D6D6
:107AF50012D1C27B007A0079B7784312C95B9065D1
:107B0500D612D1FA80179065D612D1C27B007A8041
:107B150079B6784312C95B9065D612D1FAD39068CD
:107B25003BE0940590683AE09400500C90683AE484
:107B350075F00112D0BE80907F007E807DC67C43AB
:107B45009065D612D1DE12CBEE600B40097BFF7A31
:107B5500A079D81208779065D612D1C29065CE1259
:107B6500D1FA9065CE12D1DEC000C001C002C003BB
:107B750090684012D1C290683C12D1DE12C95B9068
:107B8500684412D1DE12C95BD003D002D001D00007
:0A7B950012C95B9065CE12D1FA22EE
:107B9F00906831EEF0A3EFF0A3ECF0A3EDF0A31299
:107BAF00D28A9068427401F09065DA12D1C212CC79
:107BBF00AA90683EEEF0A3EFF0E490683FE0540324
:107BCF0070047F0180027F00906842EFF09068336D
:107BDF00E0FFA3E0906840CFF0A3EFF0906843740C
:107BEF0001F0906843E0FF906842E0F975F00DA452
:107BFF00242FF582E43400F583E5822FF582E435F6
:107C0F0083F583E0FEFD906840E0FAA3E0FBD39D8F
:107C1F00EA9400401EEFD3940C5018EEFFC3EB9F75
:107C2F00906841F0EA9400906840F0906843E00457
:107C3F00F080AF906843E0FFD3940C402EEFD394C5
:107C4F000C4099E9600D90683374FE75F09212D074
:107C5F00BE800B90683374FE75F09312D0BE90689F
:107C6F003EE475F00112D0BE027BC890683812D284
:107C7F0053EF12D062906841E0FF90683B12D253ED
:107C8F00EF12D06290683EE0FEA3E0FF90683512DD
:097C9F00D253EE8FF012D0EA225C
:107CA80090683112D1FA90683512D28A7F007E002E
:107CB8007DC07C4190683112D1DE12CA4C90683E7A
:107CC80012D1FA90683E12D1C212CCAA906842EE44
:107CD800F0A3EFF090683E12D1C2C004C005C00600
:107CE800C007906842E0FCA3E0FDEC12CC71A80448
:107CF800A905AA06AB07D007D006D005D00412C93B
:107D08005790683E12D1FA7F007E007D707C4290C9
:107D1800683E12D1DE12CA4C12CCAA906844EEF02A
:107D2800A3EFF090683E12D1C2C004C005C006C0DF
:107D380007906844E0FCA3E0FDEC12CC717B007A6C
:107D4800007970784212CB55A804A905AA06AB079A
:107D5800D007D006D005D00412C95790683E12D17A
:107D6800FA7F007E007D617C4590683E12D1DE126C
:107D7800CA4C12CCAA906843E0FD90683512D253E1
:107D8800ED12D062906845E0FD90683812D253ED4C
:0E7D980012D06290683B12D253EF12D06222DA
:107DA600E49067DDF0A3F01207F57BFF7AC27985D0
:107DB600120877900020E0FFA3E09067DBCFF0A3E6
:107DC600EFF0C39067DCE0941F9067DBE0944E50C1
:107DD6002A12E8E69067E0EFF09067DBE0FCA3E0AC
:107DE600247EF582EC3417F583EFF0641A600C906C
:107DF60067DBE475F00112D0BE80C79067DBE0FE5A
:107E0600A3E0FF900020EEF0A3EFF0C3941EEE94E3
:107E16004E40097BFF7AC279B11208777BFF7AB0B0
:107E26007926120877E49067DBF0A3F0E49067DF29
:107E3600F09067DFE0FFC3944F50409067DBE47536
:107E4600F00112D0D4FC747E25F0F582EC3417F5DF
:107E560083E09067E0F0E0FE641A601FEE640D6058
:107E66001AEE640A60159067DFE0FD04F074312DA8
:107E7600F582E43468F583EEF080B69067E0E0645E
:107E86001A70030284D074312FF582E43468F583C6
:107E9600E4F0906831E0FF64206091EF608E7E0030
:107EA6007F14C006C0077F00C0079067DDE0FEA311
:107EB600E0FF7C007D1412D07474E92FF974003E43
:107EC600FA7B01D005D007D00612D5809067DDE099
:107ED600FEA3E0FF7C007D1412D07474E92FF974C0
:107EE600003EA801FC7D017B017A6879317E007F26
:107EF6000F12CFF3E49067DFF09067DFE0C3944F93
:107F060050409067DBE475F00112D0D4FE747E25F4
:107F1600F0F582EE3417F583E09067E0F0E0FF6459
:107F26001A601FEF640D601AEF640A60159067DF30
:107F3600E0FE04F074E12EF582E43467F583EFF099
:107F460080B79067E1E064316003027E329067E3B8
:107F5600E064417003027E329067F3E024D075F04E
:107F66000AA4FFA3E0FD24D0FDE434FFCD2FCD35D8
:107F7600F0FC9067DEE025E0FF9067DDE033FE74FD
:107F8600992FF582EE3405F583ECF0A3EDF0E4903D
:107F960067DFF09067DFE0FFC3940C5021E0FE241A
:107FA600F5F582E43467F583E0FD74312EF582E45D
:107FB6003468F583EDF09067DFE004F080D5743126
:107FC6002FF582E43468F583E4F07B017A68793131
:107FD60012DE81C004C005C006C0079067DDE0FE62
:107FE600A3E07802C333CE33CED8F92411F582EE5E
:107FF6003406F583D007D006D005D00412D1FAE4B2
:108006009067DFF09067DFE0FFC3940A5021E0FE3F
:108016002402F582E43468F583E0FD74312EF5829E
:10802600E43468F583EDF09067DFE004F080D57402
:10803600312FF582E43468F583E4F07B017A6879C0
:108046003112DE81C004C005C006C0079067DDE0BE
:10805600FEA3E07802C333CE33CED8F92491F5825D
:10806600EE340DF583D007D006D005D00412D1FA30
:10807600E49067DFF09067DFE0C3944F504090676D
:10808600DBE475F00112D0D4FE747E25F0F582EEA5
:108096003417F583E09067E0F0E0FF641A601FEFA5
:1080A600640D601AEF640A60159067DFE0FE04F065
:1080B60074E12EF582E43467F583EFF080B79067BC
:1080C600E1E064326003027E32E49067DFF090679D
:1080D600DFE0FFC394085021E0FE24E9F582E43492
:1080E60067F583E0FD74312EF582E43468F583ED9F
:1080F600F09067DFE004F080D574312FF582E43428
:1081060068F583E4F07B017A68793112DE81C00478
:10811600C005C006C0079067DDE0FEA3E07802C395
:1081260033CE33CED8F924E1F582EE3408F583D088
:1081360007D006D005D00412D1FAE49067DFF0909C
:1081460067DFE0FFC394085021E0FE24F2F582E4E5
:108156003467F583E0FD74312EF582E43468F583E7
:10816600EDF09067DFE004F080D574312FF582E4FE
:0F8176003468F583E4F07B017A68793112DE8199
:10818500C004C005C006C0079067DDE0FEA3E07827
:1081950002C333CE33CED8F924A1F582EE340CF5E3
:1081A50083D007D006D005D00412D1FA9067DF74CA
:1081B50002F09067DFE0FFC394075021E0FE24F949
:1081C500F582E43467F583E0FD74312EF582E434FD
:1081D50068F583EDF09067DFE004F080D574312F0A
:1081E500F582E43468F583E4F09068317430F0A3E7
:1081F500742EF07B017A68793112DE81C004C005E6
:10820500C006C0079067DDE0FEA3E07802C333CE69
:1082150033CED8F924D1F582EE3409F583D007D0D1
:1082250006D005D00412D1FAE49067DFF09067DF3D
:10823500E0FFC394085021E0FE2403F582E434688E
:10824500F583E0FD74312EF582E43468F583EDF0B5
:108255009067DFE004F080D574312FF582E434684F
:10826500F583E4F07B017A68793112DE81C004C0C0
:1082750005C006C0079067DDE0FEA3E07802C333C2
:10828500CE33CED8F924B1F582EE340BF583D00781
:10829500D006D005D00412D1FAE49067DFF09067DC
:1082A500DFE0FFC394085021E0FE240CF582E4349E
:1082B50068F583E0FD74312EF582E43468F583EDCD
:1082C500F09067DFE004F080D574312FF582E43457
:1082D50068F583E4F07B017A68793112DE81C004A8
:1082E500C005C006C0079067DDE0FEA3E07802C3C5
:1082F50033CE33CED8F92401F582EE3407F583D099
:1083050007D006D005D00412D1FAE49067DFF090CB
:1083150067DFE0FFC3940B5021E0FE2415F582E4EE
:108325003468F583E0FD74312EF582E43468F58315
:10833500EDF09067DFE004F080D574312FF582E42D
:108345003468F583E4F07B017A68793112DE81C007
:1083550004C005C006C0079067DDE0FEA3E0780213
:10836500C333CE33CED8F924F1F582EE3407F58345
:10837500D007D006D005D00412D1FAE49067DFF01B
:108385009067DFE0FFC394055021E0FE2420F582CD
:10839500E43468F583E0FD74312EF582E43468F544
:1083A50083EDF09067DFE004F080D574312FF5821E
:1083B500E43468F583E4F07B017A68793112EA05E3
:1083C500C004C005C006C0079067DDE0FEA3E078E5
:1083D50002C333CE33CED8F9FBAA0624C1F582EA0F
:1083E500340AF583D007D006D005D00412D1FA742B
:1083F500812BF582EA340EF58312D20600000000C7
:108405009067DEE0C4F8540FC868FB9067DDE0C4F0
:1084150054F048FA747D2BF582EA340FF58312D2B5
:10842500060000000074792BF582EA340FF58312FB
:10843500D206000000009067DEE0C4F8540FC8685B
:10844500FB9067DDE0C454F048FA74752BF582EAB9
:10845500340FF58312D2060000000074712BF582EB
:10846500EA340FF58312D206000000009067DDE0C4
:10847500FEA3E0FF2401906793F0E43E906792F03D
:108485007C007D1412D07474E92FF974003EFA7BD8
:108495000190679412D28A7BFF7AC279C812D753AA
:1084A5009067DDE475F00112D0BE9067DEE090675D
:1084B50075F0C39067DE943C9067DDE09400500B47
:0F84C5009067E0E0641A6003027E321288F422AE
:1084D4007BFF7AB07926120877E49067DCF0906726
:1084E400DBF09067DBE0FFC3943C5015742D2FF54F
:1084F40082E43417F58374FFF09067DBE004F080C6
:10850400E1E49067DBF09067DBE0C3943C506512D4
:108514008584C3EE64809480500B9067DCE0D39430
:10852400004049804F9067DBE0242DF582E4341746
:10853400F583EFF07C007D1412D07474E92FF97484
:10854400003EFA7B0190679212D28A9067DCE004C5
:10855400906795F07BFF7AC279D712D7539067DC86
:10856400E004F09067DCE0C3943C50089067DBE0E3
:1085740004F080929067DCE0906776F012886522C0
:10858400E49067DFF0A3F07BFF7AB07926120877D6
:10859400E49067DDF0A3F09067DDE0FEA3E0FFC3A5
:1085A400943CEE64809480400302867B906775E07F
:1085B400FDC3EF9D7480F8EE648098400302867BCF
:1085C400EF4E601C9067DDE0FEA3E0FF7C007D04BD
:1085D40012D088ED4C70097BFF7AB07926120877A7
:1085E4009067DDE0FCA3E0FD25E0FFEC33FE74B50D
:1085F4002FF582EE3416F583A3E030E42FED240149
:10860400906793F0E43C906792F07E007F1412D060
:108614007474E92FF974003EFA7B0190679412D2C6
:108624008A7BFF7AC279FC12D75380349067DDE0ED
:10863400FEA3E0FF2401906793F0E43E906792F07C
:108644007C007D1412D07474E92FF974003EFA7B17
:108654000190679412D28A7BFF7AC3790812D753A8
:108664009067DFE475F00112D0BE9067DDE475F029
:108674000112D0BE02859B7B017A6779E190683054
:1086840012D28A7BFF7AC3791412096AAD07AC0649
:108694009067DFE0FEA3E0FFD3ED9FEE6480F8EC8B
:1086A40064809840057EFF7FFF22D3ED9400EC6444
:1086B4008094804029D3ED943CEC64809480501ED7
:1086C400ED25E0FFEC33FE74B42FF582EE3416F59D
:1086D40083E04410F0ED24FFFFEC34FFFE227EFF24
:0386E4007FFF22F3
:1086E7007BFF7AB07926120877E4906828F0A3F028
:1086F700906828E0FEA3E0FFC3943CEE648094807A
:1087070040030287CFE0242DF582E43417F583E098
:10871700C36480948050030287C2906776E0FDD3DC
:10872700EF9D7480F86E9840030287CFEF4E601C70
:10873700906828E0FEA3E0FF7C007D0412D088ED5E
:108747004C70097BFF7AB07926120877906777E03B
:10875700FF3395E0FE906828E0FCA3E0FDEFB50548
:108767000CEEB5040890682C742AF0800690682CEB
:108777007420F0ED2401906793F0E43C906792F049
:1087870090682CE0906794F0906829E0242DF5829A
:10879700E43417F583E0FF3395E0FE7C007D141287
:1087A700D07474E92FF974003EFA7B019067951233
:1087B700D28A7BFF7AC3791F12D753906828E47552
:1087C700F00112D0BE0286F77BFF7AB07926120835
:1087D7007790172DE0FF3395E0FE7C007D1412D0D3
:1087E7007474E92FF974003EFA7B01C003C002C01C
:1087F700017BFF7AC3792C9069DF12D28A9069E2F4
:10880700E4F0A37407F0D001D002D00312E96DEFB2
:10881700700E7BFF7AC379341208777EFF7FFF22C1
:108827007B017A68792A90683012D28A7BFF7AC3F3
:10883700791412096AEF24FFFFEE34FFFE90677682
:10884700E0FDC3EF9D7480F86E9850D4C3EE64804A
:0E8857009480500474FFFEFF906777EFF022CC
:10886500E4FF9069DCF09069DCE0FEC3943C502A9B
:10887500742D2EF582E43417F583E0FEC3648094ED
:1088850080400FAD070F742D2DF582E43417F58365
:10889500EEF09069DCE004F080CC9069DCEFF090BC
:1088A50069DCE0FFC3943C5045742D2FF582E43418
:1088B50017F58374FFF0742D2FF582E43417F583D3
:1088C500E0FF3395E0FE7C007D1412D07474E92F2F
:1088D500F974003EA801FC7D017BFF7AC379637EB4
:0F88E500007F0212CFF39069DCE004F080B12233
:1088F400E4906885F01207F5E4906881F0A3F0C372
:10890400906882E0943C906881E09400501AA3E05F
:10891400242DF582E43417F58374FFF0906881E424
:1089240075F00112D0BE80D77BFF7AC37966120836
:1089340077900020E0FFA3E0906881CFF0A3EFF0F0
:10894400C3906882E0941F906881E0944E50231293
:10895400E8E690688BEFF0906881E475F00112D03E
:10896400D4FC747E25F0F582EC3417F583EFF0B473
:108974001ACEC3906882E0941F906881E0944E40C0
:10898400097BFF7AC279B11208777BFF7AB0792626
:10899400120877900020E0FEA3E0247EF582EE34F6
:1089A40017F583E0641A703F906885F0906775E06E
:1089B400FF906885E0C39F502AE0FF242DF582E4F0
:1089C4003417F583EFF0EF25E024B6F582E434168E
:1089D400F583E04410F0906885E004F0E090677659
:1089E400F080C912886522E4906885F0900020E048
:1089F400FFA3E0906881CFF0A3EFF0E4906884F0E7
:108A0400906884E0FFC39450503B906881E475F013
:108A14000112D0D4FC747E25F0F582EC3417F58372
:108A2400E090688BF0E0FE641A601AEE640A601548
:108A3400906884E0FD04F0748C2DF582E43468F5CC
:108A440083EEF080BB90688BE0641A700302904B55
:108A5400748C2FF582E43468F583E4F090688CE03C
:108A6400FF643B6096EF64206091EF608E7BFF7A39
:108A7400C379959067C212D28A7B017A6879F090A3
:108A840067C512D28A7A6979049067C812D28A7A41
:108A94006979409067CB12D28A7A6979B89067CEA7
:108AA40012D28A7A6979C09067D112D28A7A6979A6
:108AB400C89067D412D28A7A6979D09067D712D2D3
:108AC4008A7A6979D69067DA12D28A7A68798C12AE
:108AD400DBE17B017A6879F012E9D4906886EFF0E3
:108AE400E4906883F0906775E0FF906883E0FEC3CC
:108AF4009F40030289FFEE75F014A424E9F9740081
:108B040035F0FA7B01C002C0017A6879F09069DF20
:108B140012D28A906886E0FF9069E2E4F0A3EFF055
:108B2400D001D00212E96DEF600302904290688593
:108B3400E0C3943C4003029042E4906888F07B01D7
:108B44007A69790412E9D4906887EFF07B017A6935
:108B540079047D2F12E9E9EA497003028C3CE49020
:108B64006884F0906887E0FF906884E0C39F504376
:108B7400E0FF2404F582E43469F583E0FE742C2FCD
:108B8400F582E43469F583EEF0906888E004F074CB
:108B9400042FF582E43469F583E0B42F0E742C2F8E
:108BA400F582E43469F583E4F08008906884E00495
:078BB400F080B07B017A693B
:108BBB00792C12DE81906883E025E025E02481F595
:108BCB0082E4340EF58312D1FAE4906884F0906855
:108BDB0088E0FF906887E0C39FFE906884E0FDC348
:108BEB009E5023E0FEEF2E2404F582E43469F583D6
:108BFB00E0FF742C2EF582E43469F583EFF0906876
:108C0B0084E004F080C8742C2DF582E43469F5837C
:108C1B00E4F07B017A69792C12DE81906883E02580
:108C2B00E025E0246DF582E43413F58312D1FA804C
:108C3B00337B017A69790412DE81906883E0FB252E
:108C4B00E025E02481F582E4340EF58312D1FAEBB2
:108C5B0025E025E0246DF582E43413F58312D2066A
:108C6B0000000000E4906888F07B017A697940127B
:108C7B00E9D4906887EFF0E4906889F0F090688908
:108C8B00E0C394044003028D6EE4906884F0906816
:108C9B0088E0FF906887E0C39FFE906884E0FDC387
:108CAB009E5038ED2F2440F582E43469F583E0FFC4
:108CBB0074A42DF582E43469F583EFF074A42DF5DB
:108CCB0082E43469F583E0FF642C6003EF7004E405
:108CDB00F08008906884E004F080B37B017A6979B6
:108CEB00A412DE81906883E075F010900F7112D2A0
:108CFB0037C083C082906889E0FBD082D08375F047
:108D0B000412D23712D1FA906888E0FF906884E0A1
:108D1B002F2440F582E43469F583E07033EB049043
:108D2B00688AF090688AE0FFC39404503690688399
:108D3B00E075F010900F7112D23775F004EF12D26C
:108D4B003712D2060000000090688AE004F080D34E
:108D5B00906884E004FF906888E02FF0A3E004F0B3
:108D6B00028C88E4906888F07B017A6979407D2FCA
:108D7B0012E9E9EA497003028E1DE4906884F090D1
:108D8B006887E0FF906884E0FEC39F501D90688861
:108D9B00E004F074402EF582E43469F583E0642F2F
:108DAB006008906884E004F080D5E4906884F090CB
:108DBB006888E0FF906887E0C39FFE906884E0FDC1
:108DCB00C39E5023E0FEEF2E2440F582E43469F578
:108DDB0083E0FF74A42EF582E43469F583EFF09001
:108DEB006884E004F080C874A42DF582E43469F53E
:108DFB0083E4F07B017A6979A412DE81906883E0C9
:108E0B0025E025E0245DF582E43414F58312D1FAD4
:108E1B008018906883E025E025E0245DF582E4343A
:108E2B0014F58312D206000000009069B8E04420CC
:108E3B00249D603024FD603E24F1601624097048A7
:108E4B00906883E02479F582E43416F5837401F09D
:108E5B008045906883E02479F582E43416F58374B9
:108E6B0002F08033906883E02479F582E43416F5C0
:108E7B00837403F08021906883E02479F582E434D5
:108E8B0016F5837404F0800F906883E02479F582E3
:108E9B00E43416F583E4F09069C0E04420249D602F
:108EAB003024FD603E24F1601624097048906883DD
:108EBB00E0243DF582E43416F5837401F08045908F
:108ECB006883E0243DF582E43416F5837402F08068
:108EDB0033906883E0243DF582E43416F583740304
:108EEB00F08021906883E0243DF582E43416F5830D
:108EFB007404F0800F906883E0243DF582E434160F
:108F0B00F583E4F09069C8E04420FFB463159068E2
:108F1B0083E025E024B6F582E43416F583E054FEB5
:108F2B00F08017EFB46D13906883E025E024B6F55D
:108F3B0082E43416F583E04401F09069D0E04420DC
:108F4B00B46D15906883E025E024B6F582E4341601
:108F5B00F583E04402F08013906883E025E024B6AB
:108F6B00F582E43416F583E054FDF09069D6E044C5
:108F7B0020FFB4691CA3E04420B47215906883E011
:108F8B0025E024B6F582E43416F583E04404F08042
:108F9B0013906883E025E024B6F582E43416F5835C
:108FAB00E054FBF0EFB46B1E9069D7E04420B47231
:108FBB0015906883E025E024B6F582E43416F5833A
:108FCB00E04408F08013906883E025E024B6F58236
:108FDB00E43416F583E054F7F0906883E0FF906873
:108FEB0085E0242DF582E43417F583EFF0EF25E0CF
:108FFB0024B6F582E43416F583E04410F0EF75F0F7
:10900B0014A424E9F9740035F0FA7B0190679212ED
:10901B00D28A906885E004906795F07BFF7AC379DC
:10902B00AD12D753E49069D6F0906885E004F0E078
:10903B00906776F00289FF906883E004F0028AE97A
:04904B001288652200
:10904F00E4906814F0A3F0A3F0A3F0A3F0A3F01240
:10905F0007F57BFF7AC379DD120877900020E0FFD8
:10906F00A3E0906812CFF0A3EFF0C3906813E094E1
:10907F001F906812E0944E502312E8E690681BEFA1
:10908F00F0906812E475F00112D0D4FC747E25F0D4
:10909F00F582EC3417F583EFF0B41ACE900020E090
:1090AF00FFA3E0906812CFF0A3EFF0E490681AF0FE
:1090BF0090681AE0FFC3943C503E906812E475F03C
:1090CF000112D0D4FC747E25F0F582EC3417F583B1
:1090DF00E090681BF0E0FE641A70030298C2EE6421
:1090EF000A601590681AE0FD04F0741C2DF582E4F7
:1090FF003468F583EEF080B8741C2FF582E4346881
:10910F00F583E4F090681CE0B431A07BFF7AC4795A
:10911F00119067C212D28A7B017A17796A9067C55C
:10912F0012D28A7A00790A9067C812D28A7A0079A5
:10913F000E9067CB12D28A7A0079169067CE12D230
:10914F008A7A6879949067D112D28A7A6879149062
:10915F0067D412D28A7A68791C12DBE1906895E0A5
:10916F004420FFB47209900007E04410F08007908C
:10917F000007E054EFF0EFB4610C900006E04410EC
:10918F00F0A3E0F08007900006E054EFF0906894B1
:10919F00E04420FFB47309900005E054F7F0800B12
:1091AF00EFB46E07900005E04408F07F007E007D6D
:1091BF00007C0090000E12D1DE12CBEE50197F0012
:1091CF007E007D807CBF90000E12D1DE12CA4C90C3
:1091DF00001212D1FA801790000E12D1DE7F007E9E
:1091EF00007DB47C4312C95790001212D1FA9068D7
:1091FF0014E0FEA3E08EF012D2C59221012C92282A
:10920F0004B092300960923812C092404B000000B7
:10921F009248E490002DF0802690002D7401F0808C
:10922F001E90002D7402F0801690002D7403F080B4
:10923F000E90002D7405F0800690002D7404F0E45C
:10924F0090681AF090681AE0FFC3943C503E906803
:10925F0012E475F00112D0D4FC747E25F0F582EC87
:10926F003417F583E090681BF0E0FE641A70030278
:10927F0098C2EE640A601590681AE0FD04F0741C41
:10928F002DF582E43468F583EEF080B8741C2FF569
:10929F0082E43468F583E4F090681CE0B432A07B7C
:1092AF00FF7AC479249067C212D28A7B017A6579DA
:1092BF00E69067C512D28A7A6579E89067C812D2AC
:1092CF008A7A6579EA9067CB12D28A7A6579EC90BF
:1092DF0067CE12D28A7A68796C9067D112D28A7A65
:1092EF0068791C12DBE190686CE04420B4660C9046
:1092FF000006E04440F0A3E0F08007900006E05441
:09930F00BFF01204E6E490681AB4
:10931800F090681AE0FFC3943C503E906812E475E0
:10932800F00112D0D4FC747E25F0F582EC3417F5E8
:1093380083E090681BF0E0FE641A70030298C2EEA6
:10934800640A601590681AE0FD04F0741C2DF5821B
:10935800E43468F583EEF080B8741C2FF582E434A9
:1093680068F583E4F090681CE0B433A07BFF7AC40E
:1093780079379067C212D28A7B017A6579F690674D
:10938800C512D28A7A6579FA9067C812D28A7A6544
:1093980079EE9067CB12D28A7A6579F29067CE120D
:1093A800D28A7A68791C12DBE1E490681AF0906836
:1093B8001AE0FFC3943C503E906812E475F0011225
:1093C800D0D4FC747E25F0F582EC3417F583E09058
:1093D800681BF0E0FE641A70030298C2EE640A602B
:1093E8001590681AE0FD04F0741C2DF582E43468C9
:1093F800F583EEF080B8741C2FF582E43468F583A9
:10940800E4F090681CE0B434A07BFF7AC4794790FC
:1094180067C212D28A7B017A68796C9067C512D2CA
:109428008A7A6879809067C812D28A7A6679359084
:1094380067CB12D28A7A66099067CE12D28A7A6886
:1094480079169067D112D28A7A0079009067D4127F
:10945800D28A7A68791C12DBE190686CE044202497
:1094680097700302950224F06023240E600302958E
:1094780021E4906632F0906873E04420643760031A
:10948800029521900007E04420F002952190663271
:109498007401F0906871E04420B47709900005E009
:1094A80054BFF08007900005E04440F0906872E0F7
:1094B800FFB438169066337421F0A37411F090004D
:1094C80009E04404F054FDF0804FEF4420B46F14D9
:1094D8009066337401F0A3F0900009E054FBF05457
:1094E800FDF08035906633742EF0A3741EF0900062
:1094F80009E04402F054FBF0801F9066327402F0D9
:10950800906870E04420B47309900009E04410F0BA
:109518008007900009E054EFF0906880E04420FF55
:10952800B46609900005E04480F0800BEFB4610751
:10953800900005E0547FF0906816E0FEA3E08EF0FE
:1095480012D2C5956F04B095760960955F25809510
:10955800674B000000957E90002E7403F0801D90EC
:10956800002E7404F08015E490002EF0800E900018
:109578002E7401F0800690002E7402F0C28C9000C8
:109588002EE02428F582E43400F583E0F58CD28CB3
:10959800E490681AF090681AE0FFC3943C503E903B
:1095A8006812E475F00112D0D4FC747E25F0F582BF
:1095B800EC3417F583E090681BF0E0FE641A700342
:1095C8000298C2EE640A601590681AE0FD04F0740F
:1095D8001C2DF582E43468F583EEF080B8741C2FF6
:1095E800F582E43468F583E4F090681CE0B435A0B3
:1095F8007BFF7AC4795F9067C212D28A7B017A684E
:08960800796C9067C512D28A4B
:109610007A66790A9067C812D28A7A66790E90675C
:10962000CB12D28A7A6679269067CE12D28A7A666F
:10963000792A9067D112D28A7A66792E9067D412ED
:10964000D28A7A68791C12DBE190686CE0B4310947
:10965000900005E04410F08007900005E054EFF022
:1096600090686DE09068A8F0E4A3F07B017A6879D7
:10967000A812EB13EF0490001AF090686EE0906867
:10968000A8F0E4A3F07B017A6879A812EB13EF2429
:109690000290001BF0E490681AF090681AE0FFC393
:1096A000943C503E906812E475F00112D0D4FC74E2
:1096B0007E25F0F582EC3417F583E090681BF0E02E
:1096C000FE641A70030298C2EE640A601590681A6C
:1096D000E0FD04F0741C2DF582E43468F583EEF0AF
:1096E00080B8741C2FF582E43468F583E4F0906848
:1096F0001CE0B436A07BFF7AC479759067C212D2A1
:109700008A7B017A6879949067C512D28A7A6679E1
:10971000459067C812D28A7A6679499067CB12D28F
:109720008A7A68796C9067CE12D28A7A687980904A
:1097300067D112D28A7A6779719067D412D28A7A05
:109740006779739067D712D28A7A68791C12DBE145
:10975000906894E0B4310C900006E04402F0A3E07D
:10976000F08007900006E054FDF0906895E0B43179
:1097700009900006E054F7F0800A900006E04408E3
:10978000F0A3E0F090686CE04420249D601C24FD70
:10979000602024F1600C240970209066577401F059
:1097A000801D9066577402F080159066577403F020
:1097B000800D9066577404F08005E4906657F09031
:1097C0006880E04420249D601C24FD602024F1601A
:1097D0000C240970209066587401F0801D90665822
:1097E0007402F080159066587403F0800D906658EE
:1097F0007404F08005E4906658F0E490681AF090E4
:10980000681AE0FFC3943C503E906812E475F00182
:1098100012D0D4FC747E25F0F582EC3417F583E089
:1098200090681BF0E0FE641A70030298C2EE640AAE
:10983000601590681AE0FD04F0741C2DF582E43484
:1098400068F583EEF080B8741C2FF582E43468F577
:1098500083E4F090681CE0B437A07BFF7AC4798E73
:109860009067C212D28A7B017A68796C9067C512C0
:10987000D28A7A6679129067C812D28A7A66791685
:109880009067CB12D28A7A66791A9067CE12D28A02
:0A9890007A66791E9067D112D28A21
:10989A007A68791C12DBE190686CE0B431099000B7
:1098AA0005E04420F08007900005E054DFF07BFFDC
:1098BA007AC479A1120877227BFF7AC479C3120885
:0298CA00772203
:1098CC00900004E04410FEA3E0FF900004EEF0A32F
:1098DC00EFF020E10302996C906777E0FF3395E09D
:1098EC00FE742D2FF582EE3417F583E0FF3395E0EF
:1098FC00FEEF7802C333CE33CED8F9246DF582EE69
:10990C003413F58312D1C212CCAA7BA07A867901CA
:10991C00780012D12490688112D1FA906777E0FF19
:10992C003395E0FE742D2FF582EE3417F583E0FFAE
:10993C003395E0FEEF7802C333CE33CED8F9245DF5
:10994C00F582EE3414F58312D1C212CCAA7BA07A24
:10995C00867901780012D12490688512D1FA80148E
:10996C0090688512D2060000000090688112D20621
:10997C00000000007BFF7AC479E71208777BFF7A3E
:10998C00C479FE1208777F801202A07BFF7AC5791A
:10999C003D1208957FC01202A07BFF7AC5794F1249
:1099AC0008957BFF7AC579611208777B017A677914
:1099BC00F51208F27B017A6779F512E9D49067D534
:1099CC00EFF07BFF7AC5796E9067C212D28A7B0169
:1099DC007A6879459067C512D28A7A6879639067FC
:1099EC00C812D28A7A6779F512DBE19067F5E0FF4D
:1099FC00442012D29F9E863F9CDE619A22669B98E1
:109A0C006D9A1A719E21739D9D7400009EA1900009
:109A1C0004E054EFF0229067F6E044206475600394
:109A2C00029AD09067D6F09067D6E0FFC3940950A5
:109A3C0021E0FE24F7F582E43467F583E0FD74D76A
:109A4C002EF582E43467F583EDF09067D6E004F0F0
:109A5C0080D574D72FF582E43467F583E4F07B016D
:109A6C007A6779D712EA0590688512D1DE12D1098E
:109A7C0090665D12D1FA90665D12D1C27B0A7A00B3
:109A8C007900780012D12490665D12D1FA90677734
:109A9C00E0FF3395E0FE742D2FF582EE3417F5833D
:109AAC00E0FF123CAA7FC01202A07BFF7AC579743A
:109ABC001208957FC31202A07B017A6779D712082E
:109ACC00950299AE9067F6E0442064646003029BB3
:109ADC007E9067D6F09067D6E0FFC394095021E0E2
:109AEC00FE24F7F582E43467F583E0FD74D72EF598
:109AFC0082E43467F583EDF09067D6E004F080D50E
:109B0C0074D72FF582E43467F583E4F07B017A6730
:109B1C0079D712EA0590688112D1DE12D1099066CC
:109B2C005912D1FA90665912D1C27B0A7A00790087
:109B3C00780012D12490665912D1FA906777E0FF21
:109B4C003395E0FE742D2FF582EE3417F583E0FF8C
:089B5C00123A3E7FC01202A084
:109B64007BFF7AC579861208957FC31202A07B0118
:109B74007A6779D71208950299AE7BFF7AC57998EE
:109B84001208777FC01202A07BFF7AC579C0120841
:109B9400950299AE9067F6E0442064756003029CD8
:109BA4002E7FC01202A07BFF7AC5794F1208957FE1
:109BB400C01202A07B017A6779F51208959067F7C5
:109BC400E04420249D601C24FD602024F1600C24CA
:109BD4000970209066557401F080349066557402C3
:109BE400F0802C9066557403F080249066557404BC
:109BF400F0801CE4906655F07FC01202A07BFF7ACF
:109C0400C579D11208957BFF7AC579E2120877905D
:109C14006777E0FF3395E0FE742D2FF582EE34175D
:109C2400F583E0FF123F470299AE9067F6E04420C7
:109C340064646003029CC47FC01202A07BFF7AC5E7
:109C4400794F1208957FC01202A07B017A6779F5DB
:109C54001208959067F7E04420249D601C24FD6061
:109C64002024F1600C240970209066567401F08061
:109C7400349066567402F0802C9066567403F0801B
:109C8400249066567404F0801CE4906656F07FC0FD
:109C94001202A07BFF7AC579D11208957BFF7AC6A0
:109CA4007901120877906777E0FF3395E0FE742D11
:109CB4002FF582EE3417F583E0FF123F470299AE89
:109CC4007BFF7AC679201208777FC01202A07BFF3F
:109CD4007AC679451208950299AE9067D5E0C39487
:109CE4000A501A7BFF7AC679561208777FC012028F
:109CF400A07BFF7AC6797C1208950299AEE490673E
:109D0400D6F09067D6E0FFC394035021E0FE2447C9
:109D1400F582E43468F583E0FD74D72EF582E434EB
:109D240067F583EDF09067D6E004F080D574D72F03
:109D3400F582E43467F583E4F07B017A6779D7121E
:109D4400DE8190660212D1FAE49067D6F09067D66D
:109D5400E0FFC394025021E0FE2465F582E43468F8
:109D6400F583E0FD74D72EF582E43467F583EDF0D6
:109D74009067D6E004F080D574D72FF582E4346779
:109D8400F583E4F07B017A6779D712DE8190660669
:109D940012D1FA125EEE0299AEE49067D6F09067A3
:109DA400D5E0FFA3E0FEC39F502074F62EF582E4B5
:109DB4003467F583E0FF74D72EF582E43467F583C6
:109DC400EFF09067D6E004F080D474D72EF582E4E7
:109DD4003467F583E4F07B017A6779D712EB13EFEC
:109DE40014906777F0D36480948E5018E0FF339515
:109DF400E0FE742D2FF582EE3417F583E0C3648002
:109E04009480500C7BFF7AC6798E1208770299AE43
:109E1400900005E04404F012290A0299AEE4906728
:059E2400D6F09067D5A7
:109E2900E0FFA3E0FEC39F502074F62EF582E434D0
:109E390067F583E0FF74D72EF582E43467F583EF85
:109E4900F09067D6E004F080D474D72EF582E4341C
:109E590067F583E4F07B017A6779D71208B37FC08D
:109E69001202A07BFF7AC5794F1208957FC01202B2
:109E7900A07B017A6779D71208950299AE9067F6A7
:109E8900E04420B461061261640299AE7BFF7AC690
:109E990079A01208770299AE7BFF7AC679DF12089A
:109EA900777FC01202A07BFF7AC679F0120895026B
:039EB90099AE223D
:109EBC009068B2EFF01241D3900006E0FEA3E0FFF1
:109ECC00EE30E16E30E26B7F007E247D747C499035
:109EDC00664512D1DE12CA4C12CCAA90665912D128
:109EEC00FA7F007E247D747C4990664912D1DE1283
:109EFC00CA4C12CCAA90665D12D1FA906657E090CB
:109F0C006655F0906658E0906656F09068B2E0FFA7
:109F1C00123F479068B2E0FF123CAA9068B2E0FF93
:109F2C00123A3E900006E054FBF09068B2E0FF124B
:109F3C0043C9900006E054DFF090660E12D1C29037
:109F4C00660612D1FA90660A12D1C290660212D13C
:109F5C00FA126706906771E0FEA3E0FFE4FCFDC017
:109F6C0004C005C006C00790676912D1DE90676512
:109F7C0012D1C212D116A804A905AA06AB07D007A4
:109F8C00D006D005D004D312D1975038906771E029
:109F9C00FEA3E0FFE4FCFDC004C005C006C00790B2
:109FAC00676D12D1DE90676512D1C212D116A8046A
:109FBC00A905AA06AB07D007D006D005D004D3124A
:089FCC00D19740031235F62283
:10C87900EF7E09D3C28D308DFDC28D308DFDC28D05
:10C88900308DFDC28D308DFDD3C297C28D13308D91
:10C89900FDC28D308DFDC28D308DFDC28D308DFD77
:10C8A9009297C28DDEE7308DFDC28D308DFDC28D30
:10C8B900308DFDC28D308DFDC28D308DFDC28D3024
:10C8C9008DFDC28D308DFDC28D308DFDED705E22E6
:10C8D900EF7E09D3C28D308DFDC28D308DFDC28DA5
:10C8E900308DFDC28D308DFDD3C295C28D13308D33
:10C8F900FDC28D308DFDC28D308DFDC28D308DFD17
:10C909009295C28DDEE7308DFDC28D308DFDC28DD1
:10C91900308DFDC28D308DFDC28D308DFDC28D30C3
:10C929008DFDC28D308DFDC28D308DFD227E5C0066
:10C9390000000000000000DEF6DDF2227E5C00004F
:0BC94900000000000000DEF6DFF2221C
:10C9540002CD16E86480F8E933E83360110460F02E
:10C96400ED33EC337009E8FCE9FDEAFEEBFF220449
:10C9740060DED3EB9FEA9EE99DE8C2E78CF0C2F744
:10C9840095F0400CE8CCF8E9CDF9EACEFAEBCFFB10
:10C9940012CCE185D0F05804700320D5B3E80470BC
:10C9A400075002B2D502CD2092D5EC0460F7E4CC56
:10C9B400C0E0C398F8603B94186008400DD0E0FBD9
:10C9C40002CCF8E4FBFAC9FC8028E830E406E4C9A8
:10C9D400FBE4CAFCE830E305E4C9CACBFCE854072D
:10C9E4006010F8C3E913F9EA13FAEB13FBEC13FC38
:10C9F400D8F130F52FC3E49CFCEF9BFFEE9AFEEDDB
:10CA040099FDD0E0FBEF4E4D4C701222DB0302CDBA
:10CA14001DEC2CFCEF33FFEE33FEED33FDED30E780
:10CA2400EB02CCF8EF2BFFEE3AFEED39FDD0E0FB44
:10CA340050130BBB000302CD20ED13FDEE13FEEFEC
:08CA440013FFEC13FC02CCF817
:10CA4C00EC4D6011E8497017ED33EC3304600DE4E4
:10CA5C00FCFFFEFD22E933E8330470F802CD161218
:10CA6C00CCE158046009E4CC24815006285009021A
:10CA7C00CD2028400302CD1DC0E0EB4A7044B980A4
:10CA8C0006D0E0FB02CD0CEF4E701CBD8008EBFF16
:10CA9C00EAFEE9FD80EBE98DF0A4FEE5F002CB3572
:10CAAC00E9CDF9EAFEEBFFEF89F0A4FCE5F0CE89C5
:10CABC00F0A42EFFE435F0CD89F0A42DFEE435F082
:10CACC008067EF4E7005BD80D780C3EF8BF0A4ACB0
:10CADC00F0EE8BF0A42CFCE435F0F8EF8AF0A42CEB
:10CAEC00E5F038FCE433CB8DF0A42CFCE5F03BF8FE
:10CAFC00EE8AF0A42CFCE5F038F8E433CF89F0A4EE
:10CB0C002CFCE5F038CF3400CE89F0A42FFFE5F0F3
:10CB1C003EFEE433C98DF0A42EFEE5F039CD8AF04B
:10CB2C00A42FFFE5F03EFEE43DFD33D0E0FB5007C3
:10CB3C000BBB000F02CD20EC2CFCEF33FFEE33FED1
:06CB4C00ED33FD02CCF800
:10CB520002CD20EC5D046005E85904700302CD1695
:10CB620012CCE1580460F6EC4860F2EC7004FDFE71
:10CB7200FF22C82481C85007C398500602CD1D98D1
:10CB820050CEF582E9294B4A7005AB8202CD0C7575
:10CB9200F0007C1A7880C3EF9BEE9AED99400DC3AA
:10CBA200EF9BFFEE9AFEED99FDE842F0DC23ACF03C
:10CBB200D0E0FFD0E0FED0E0FDAB8220E7101BEB1F
:10CBC20060BAEC2CFCEF33FFEE33FEED33FD02CC0A
:10CBD200F8E803F830E705C0F075F000EF2FFFEE3C
:0CCBE20033FEED33FD40B830E7C280AAFE
:10CBEE0074F8CC6480CCC86480C8F582046043C3FA
:10CBFE00EB9FF5F0EA9E42F0E99D42F0E89C45F08D
:10CC0E0060305018E5825FFFE582F42B5582FB50B1
:10CC1E00210ABA001D09B90019088016E5825BFBCE
:10CC2E00E582F42F5582FF50090EBE00050DBD00A2
:10CC3E00010CC3EB9FF5F0EA9E42F0E99D42F0E84D
:0DCC4E009C45F06007CC4820E701B3EC22C4
:10CC5B00ED33EC33600A047003BD8004ECB2E7FCE7
:01CC6B0022A6
:10CC6C0075F020800E75F010800575F0087D007E43
:10CC7C00007F003392D530D50312D173EC334010C2
:10CC8C00EF33FFEE33FEED33FDEC33FCD5F0ED224C
:0ECC9C00E5F0247EA2D513CC92E7CDCEFF2288
:10CCAA00EDD2E7CD33EC3392D524814006E4FFFE82
:10CCBA00FDFC22FCE4CFCECDCC24E0501174FF80E1
:10CCCA00EDC3CC13CCCD13CDCE13CECF13CF04707E
:07CCDA00F030D5DE02D1733A
:10D6E800E50C2492F582E43467F583E0050C22907A
:10D6F800678F300803906792E475F00112D25C02DC
:10D70800D01C2001E97F2ED2018018EF540F2490FD
:10D71800D43440D4FF30050BEF24BFB41A005003B3
:10D728002461FFE50D6002150D0510E51070020576
:10D738000F30080E90678FE475F00112D25CEF028B
:10D74800D06202E8BF7403D2088003E4C208F50C73
:10D7580090678F12D28AE4F50DF50FF510E50D608C
:10D76800077F2012D72B80F5F50EC202C201C20333
:10D77800C204C206C207C20912D6F7FF700D3008EC
:10D78800057F0012D73CAF10AE0F22B42563C2D577
:10D79800C20512D6F7FF24D0B40A00501E75F00A4D
:10D7A80020D50DC50DA4250DF50D7002D20480E01D
:10D7B800D201C50EA4250EF50E80D524CFB41A00CB
:10D7C800EF5004C2E5D20502DA25D20280C2D201A6
:10D7D80080BCD20380B8D2D580B6D20680B07F2074
:10D7E80012D72B2003077401B50D0040F112D6E8BB
:10D7F800FF12D72B02D765D209D207809112D6E83B
:10D80800FB12D6E8FA12D6E8F94A4B7006791C7A68
:10D81800DB7BFF200333E50D602FAF0EBF00011F38
:10D828007E008E8275830012D03560050EEE6F7013
:10D83800F1C2D5EBC0E0EAC0E0E9C0E0EE12DA815F
:10D84800D0E0F9D0E0FAD0E0FB12D01CFF60A5EBE5
:10D85800C0E0EAC0E0E9C0E012D72BD0E02401F92B
:10D86800D0E03400FAD0E0FBE50E60DDD50EDA80BA
:10D8780083D203809E12DA6560F7E50E12CD2AA9DD
:10D888000E600BE50E12DB09EF7003D50EF5EA30DA
:10D89800E702F404C3995079EAF4250E0430E7014D
:10D8A800E404F50E800D12DA6560C6EA050E250E51
:10D8B80012CD2AEA9067BEF030E701E4250E04D5C0
:10D8C8000E042006011412DA81E4C0E012DB09908C
:10D8D80067BEE0601320E70714F012D71380220414
:10D8E800F0D0E014C0E07F0012D713E50E600712F5
:10D8F800D70A150E800B30060312D70AD0E002D7DC
:10D9080065D0E00480C412DA65609EE50E0412CD8D
:10D918002A9067BEEAF0E50E04200602600104249E
:10D928000412DA8174FF04C0E012DB0912D713E590
:10D938000E200602600312D70AD0E0B50EE87F4534
:10D9480012D71D9067BEE07F2B30E7047F2DF404CB
:10D95800C0E012D72BD0E075F00A84C0F012D714BB
:10D96800D0E012D71402D765791080027908C2076F
:10D97800C2098008D2D5790A8004790AC2D5E4FAA6
:10D98800FDFEFF12D6E8FC7B0820021312D6E8FD44
:10D998007B1030010A12D6E8FE12D6E8FF7B20EC95
:10D9A8003382D592D55013C3E43001069FFFE49E1D
:10D9B800FEE42002039DFDE49CFCE4CBF8C202ECEB
:10D9C800700CCFCECDCCE824F8F870F38017C3EFF5
:10D9D80033FFEE33FEED33FDEC33FCEB33FB9940C4
:10D9E80002FB0FD8E9EB300205F8D0E0C448B202D8
:10D9F800C0E00AEC4D4E4F78207B0070C2EAC0E0D0
:10DA080012DA83D0F0D0E0200204C4C0E0C4B2022D
:10DA1800C0F012D714D0F0D5F0EB02D76512D29F20
:10DA2800D80553D97058D7D64CD7D242D9744FD9C4
:10DA38007C44D97C49D7EB43D98255D8AE46D90E18
:10DA480045D87D47DB3F50D7DA2DD7DE2ED8012BBE
:10DA5800D7E223D7FF20DB2A2A0000D7F9100103D9
:10DA6800750E0612D6E8FC12D6E8FD12D6E8FE12AC
:10DA7800D6E8FF9067B702CD67790AA2D5200414CB
:10DA8800300609B910020404B9080104A2D5200718
:10DA9800025001042003669203B50D005032C0E025
:10DAA8007F203004177F30A20372077206500D12D0
:10DAB800DAD8C203C207C2067F30800F300603E9F6
:10DAC800C0E012D72B300603D0E0F9D0E0B50DCE78
:10DAD8003006177F30B9100C12D72B7F5830050746
:10DAE8007F788003B9080312D72B3003057F2D02F6
:10DAF800D72B7F202009F87F2B2007F32292038061
:10DB0800CF7F00B40700500B24B7F582E43467F5E3
:10DB180083E0FF22286E756C6C29002D504349580C
:10DB2800D20212D6E83002F8C202780D30D504D2FB
:10DB380001780EF602D79612D6E82403B405004001
:10DB480001E490DB239312D71C743A12D71CD20439
:06DB5800750D0402D970F6
:10DB5E00E50C30040104F8232824C2F582E434676E
:10DB6E00F583229067BF3004039067C2E475F0011D
:10DB7E0012D25C02D01C60EAC5107002150F14C5DB
:10DB8E0010200404FF02E8FA9067BF74FFF5F0025C
:10DB9E00D273FF02E902E50D6006D50D037F002268
:10DBAE000510E5107002050F20040302E8E69067E9
:10DBBE00BF12D25312D01CFF60A89067BFE475F05D
:10DBCE000102D25C12DBAEEFC0E012DBA0D0E0406F
:10DBDE00F380A3D2048002C2049067BF12D28AE4FB
:10DBEE00F50EF50CF50FF510750D00C203C201C24E
:10DBFE0002C20512DB71FF7005AF0E7E0022B42546
:10DC0E003012DB71FF24D0B40A00500C75F00AC537
:10DC1E000DA4250DF50D80E924CFB41A00EF5002A6
:10DC2E00C2E502DE40D20280D8D20180D4D2058075
:10DC3E00D0EF12DBA0500512DBD280ACEFC0E012A9
:10DC4E00DBAED0E06F60A1EF606E12DB8480AA7451
:10DC5E0001C50D6002F50D12DBAEEF605B20050E07
:10DC6E0012DB5EE475F00112D25CEF12D062D50DBC
:10DC7E00E6200504050C050E80C012DBA4EFC0E003
:10DC8E0012DBA0D0E0500412DB84E4FF20050E125C
:10DC9E00DB5EE475F00112D25CEF12D062EF70DA47
:10DCAE00200504050C050E8091E50D6002050D1290
:10DCBE00DBD212DBA4EF70C6300404E412DB84E581
:10DCCE000E600302DC077EFF7FFF22E50D6002057A
:10DCDE000D12DBD2D207D20612DBA4EF30070260A0
:10DCEE00D7C0E012DB84D0E0AC11AD12AE13AF148E
:10DCFE0012E5518C118D128E138F14500712DBAE5C
:10DD0E00C20680D4200510200602050E12DB5E121C
:10DD1E00D253050C12D1A802DBF6EF12DB84790880
:10DD2E00803B12DBD212DBAEEF608DBF301B12DBFD
:10DD3E00AEEF6084BF78028003BF58DE7910801D7D
:10DD4E0012DBD212DBAEEF60E0790AEFB42D04D213
:10DD5E00038019B42B02801412DB84790AE50D605E
:10DD6E0002050DE9C0E012DBD2D0E0F9D206E4FCE8
:10DD7E00FDFEFFE9C0E0ECC0E0EDC0E0EEC0E0EF7C
:10DD8E00C0E012DBA4EFF8D0E0FFD0E0FED0E0FD63
:10DD9E00D0E0FCD0F0E8604DB461004007B47B00E9
:10DDAE005002C2E524D0503DFA24F6500724F95013
:10DDBE0034240AFAEAB5F000502BCFA9F0A42FFFB5
:10DDCE0092D5E9C5F0CEA4A2D53EFE92D5E9C5F016
:10DDDE00CDA4A2D53DFD92D5E9C5F0CCA4A2D53CEB
:0ADDEE00FCC206808EE8C0E02005AC
:10DDF8002A200608050E30030312D17312DB5E12C7
:10DE0800D253050C20010B20020DEE8FF012D0EA40
:10DE1800800912D1A88004EF12D062D0E012DB840E
:10DE280002DBF620051012DB5E12D253050CE50F5B
:10DE38008510F012D0EA80E812D29FDCB753DD4A91
:10DE480058DC374CDC3342DC3348DD2C4FDD4E44A4
:10DE5800DC5D43DD3049DD6955DCD946DCD945DC7C
:0CDE6800D947DC3B2ADE2B4E0000DC3FDB
:0DDE7400ED33EC3360065004EC6480FC22BA
:10DE8100D2079069DC12D28A12DEBDC0E0FF12E92E
:10DE910002D0E040F312E551400122ECC0E0EDC0B8
:10DEA100E0EEC0E0EFC0E012DEBDD0F0AFF0D0F0A8
:10DEB100AEF0D0F0ADF0D0F0ACF080D9E475F00167
:09DEC1009069DC12D25C02D01C55
:10DECA0002CD1622EDA2E7D2E7F9EC3340F260F375
:10DEDA00B4FF08ED547F70E802CD20F82481C2E037
:10DEEA00C0E0F40428FAC313FCED92E7FD9069221E
:10DEFA0012D1FAEEA2E7E9BA7F02C3133400940002
:10DF0A00FA75F091A4E5F013F494FE8AF0A433E5CF
:10DF1A00F033248CD313FDE492E7FE7F007C3F7537
:10DF2A008302ECC0E0F8EDC0E0F9EEC0E0FAEFC021
:10DF3A00E0FB8583F090692212D1C285F08312CB6F
:10DF4A0055D0E0FBD0E0FAD0E0F9D0E0F812C95B96
:10DF5A00ED6480FD30E7011CD583C7ED33CC33F87F
:0CDF6A00D0E0A2E71328C313CC13FD2263
:10DF76003A70FA83BCAAE9E43E81E0F8BF9DE9E67F
:10DF86003F80000039283C1ABB9969663DA335E3FA
:10DF9600BF255DE73FC90FDB418DDBCCC44936EEBB
:10DFA60045C9913FC5B0F83D3F800000C317F53421
:10DFB600452FFA73C60AFDDD12E07F04A2E1920145
:10DFC6001420E01590DF76740412CE6C803012E0D7
:10DFD6007F30E102B20120E0EBA883A9829069229A
:10DFE60012D1FA8982888390DF8A740412CE6C85F6
:10DFF60082F090692212D1DE85F08212CA4CED4C75
:10E006006007300104EC6480FC2212E07FC0E0A8C7
:10E0160083A98290692212D1FA8982888390DFAE21
:10E02600740312CE6C8582F090692212D1DE85F0DF
:10E036008212CA4C906922E0CCF0A3E0CDF0A3E0B6
:10E04600CEF0A3E0CFF090DF9E740312CE6CD082A8
:10E056008582F090692212D1DE85F082E58230E079
:10E066000712CB55B2018096EFCBFFEECAFEEDC983
:10E07600FDECC8FC12CB558085ED33EC547FCC33D8
:10E08600920124605007D0E0D0E002CD167B837A5F
:10E09600F97922783E12CA4CEDF933ECF833248133
:10E0A6005011EFFBEEFA12CCAA12CC6CECB2E7FCE4
:10E0B60012C95BED33EC33602F2403F8C313FCED78
:10E0C60092E7FDE82481E4501FECF8EDF9EEFAEF53
:10E0D600FB12CCAAEF04C2E0FCF58212CC76ECB2BD
:10E0E600E7FC12C95BE58203FAED33EC33600714F3
:08E0F60013FCED92E7FDEA22A4
:10E0FE00BE1249253E4CCCCDBEAAAAAB3F80000035
:10E10E003E7ADBB03EED63383F24BC7D3F490FDBEA
:10E11E00ED33ECC2E7CC339201B4FF13ED547F60C4
:10E12E000302CD167FDB7E0F7DC97C3F02E213C258
:10E13E0002C3947F401E7007EDD2E794904015EF16
:10E14E00FBEEFAEDF9ECF87F007E007D807C3F124D
:10E15E00CB55D202ED33EC33248430E705E4C0E036
:10E16E00806B04FAEDD2E754F0C333DAFD54073472
:10E17E00002323C0E0CCC0E0F8EDC0E0F9EEC0E033
:10E18E00FAEFC0E0FBE412CC76EC24FEFC906922A0
:10E19E0012D1FA12CA4C7B007A007980783F12C9EC
:10E1AE005B906922E0B2E7CCF0A3E0CDF0A3E0CE25
:10E1BE00F0A3E0CFF0D0E0FBD0E0FAD0E0F9D0E071
:10E1CE00F812C95B90692212D1DE12CB55906922EA
:10E1DE0012D1FA90E0FE740312CE6C90692212D125
:10E1EE00DE12CA4CD0E0600F240AF582E434E1F569
:10E1FE008312D1EA12C95B30020B7BDB7A0F79C92D
:10E20E0078BF12C95BED33EC336006ECA20192E7E6
:02E21E00FC22E0
:10E2200090692212D1FA7FFF7EFF7DFF7CFF90690B
:10E2300022E0F8A3E0F9A3E0FAA3E0FBC312D19730
:10E2400060387F807E967D187C4B906922E0F8A331
:10E25000E0F9A3E0FAA3E0FB12CBEE6002501B7FD3
:10E26000807E967D187CCB906922E0F8A3E0F9A32C
:10E27000E0FAA3E0FB12CBEE500F906922E0FCA382
:10E28000E0FDA3E0FEA3E0FF22906922E0FCA3E012
:10E29000FDA3E0FEA3E0FF12CCAA90692612D1FAFA
:10E2A000906926E0FCA3E0FDA3E0FEA3E0FFEC12F2
:10E2B000CC6CC8ECC8C9EDC9CAEECACBEFCB90692B
:10E2C00022E0FCA3E0FDA3E0FEA3E0FF12C9577B20
:10E2D000007A007900780012CBEE5025906926E094
:10E2E000FCA3E0FDA3E0FEA3E07A0079007800241F
:10E2F00001FFEA3EFEE93DFDE83CFC90692612D1B3
:10E30000FA906926E0FCA3E0FDA3E0FEA3E0FFECA9
:04E3100012CC6C229D
:10E3140090692212D1FA7FFF7EFF7DFF7CFF906916
:10E3240022E0F8A3E0F9A3E0FAA3E0FBC312D1973B
:10E3340060387F807E967D187C4B906922E0F8A33C
:10E34400E0F9A3E0FAA3E0FB12CBEE6002501B7FDE
:10E35400807E967D187CCB906922E0F8A3E0F9A337
:10E36400E0FAA3E0FB12CBEE500F906922E0FCA38D
:10E37400E0FDA3E0FEA3E0FF22906922E0FCA3E01D
:10E38400FDA3E0FEA3E0FF12CCAA90692612D1FA05
:10E39400906926E0FCA3E0FDA3E0FEA3E0FFEC12FD
:10E3A400CC6CC8ECC8C9EDC9CAEECACBEFCB906936
:10E3B40022E0FCA3E0FDA3E0FEA3E0FF12C9577B2B
:10E3C400007A007900780012CBEE60244022906934
:10E3D40026E0FCA3E0FDA3E0FEA3E024FFFFEE346F
:10E3E400FFFEED34FFFDEC34FFFC90692612D1FAF8
:10E3F400906926E0FCA3E0FDA3E0FEA3E0FFEC129D
:03E40400CC6C22BB
:10E4070090692212D1FA7F007E007D007C0090691E
:10E4170022E0F8A3E0F9A3E0FAA3E0FB12CBEE7049
:10E427003BFFFEFDFC906926E0F8A3E0F9A3E0FAC4
:10E43700A3E0FB12CBEE600B40097F007E007D005E
:10E447007C002290692612D206FFFFFFFF90692603
:10E45700E0FCA3E0FDA3E0FEA3E0FF22E490692A2D
:10E46700F0A3F0FFFEFDFC906922E0F8A3E0F9A31A
:10E47700E0FAA3E0FB12CBEE5065906926E0FCA31F
:10E48700E0FDA3E0FEA3E0FF12CCAA90692AEEF01C
:10E49700A3EFF0FDCCEECCE412CC71C8ECC8C9ED0B
:10E4A700C9CAEECACBEFCB906926E0FCA3E0FDA377
:10E4B700E0FEA3E0FF12C9577B007A0079007800DD
:10E4C70012CBEE600302E44A906922E0FCA3E0FD70
:10E4D700A3E0FEA3E0FF12CC5B90692212D1FA9071
:10E4E7006922E0FCA3E0FDA3E0FEA3E0FF12E6F251
:10E4F700906926E0F8A3E0F9A3E0FAA3E0FB12CACB
:10E507004C12E65C90692612D1FA90692BE030E054
:10E5170017906926E0FCA3E0FDA3E0FEA3E0FF124D
:10E52700CC5B90692612D1FA906926E0FCA3E0FD46
:07E53700A3E0FEA3E0FF22B8
:10CCE100E9D2E7C933E833F892D5EDD2E7CD33EC99
:07CCF10033FC5002B2D52212
:10CCF800EC30E7100FBF000C0EBE00080DBD00049D
:10CD08000BEB6014A2D5EB13FCED92E7FD2274FF48
:10CD1800FCFDFEFF22E480F8A2D574FF13FC7D80A1
:02CD280080F099
:10CD2A00F920E73624F950037907E4F42402FBE5F5
:10CD3A0082158270021583DBF6E024FB501BE96042
:10CD4A0014E4F0E582158270021583E004F0B40A57
:0DCD5A0008E4F0D9EE7401F00A22C2D522DF
:10CD6700ED33EC3392D5FA602AB4FF33EDC2E77B9B
:10CD7700FF60067ACD798CE4227ACD799520D504A7
:10CD87007ACD7990224E614E002B494E46002D49AF
:10CD97004E4600E47A08F0A3DAFC7B00740722C051
:10CDA70083C082ECC0E0EDC0E0EEC0E0EFC0E0EA97
:10CDB70075F010A4CAABF075F04DA42BFBE435F069
:10CDC700FCEA2410FAEB34C5FBEC34D9FCEDC2E7DE
:10CDD700FF75F056A4F42411C5F0F434C58FF0A400
:10CDE7002AE5F03BE43CF020E71412CEE3D0E0FF65
:10CDF700D0E0FED0E0FDD0E0FC12CB558014F40467
:10CE070012CEE3D0E0FFD0E0FED0E0FDD0E0FC1290
:10CE1700CA4CD082D083E0FAEDD2E7CD33EC33248D
:10CE270082FBE4C3CF33CFCE33CECD33CD33DBF369
:10CE37007B0775F00A846004F0A31B0AE5F0F0A3F2
:10CE47008FF0740AA4FFACF08EF0740AA42CFEAC29
:10CE5700F050010C8DF0740AA42CFDE435F0F0A31A
:05CE6700DBDE74072270
:10E53E00C208C209C20AC20BF9E4F515F516FCFDB4
:10E54E00FEFFE91007EA200A0CB42D04D20AD322EA
:10E55E00B42B02D32224D0504794095041240A30C0
:10E56E000B15F88516F0740AA42872E74051C5F011
:10E57E00704D85F016D322D209C0E0E4FBFA792063
:10E58E00784112CA4CECF8EDF9EEFAEFFBD0E0FC54
:10E59E00E412CC7612C95B3008B41515D322240AC6
:10E5AE00200B20B4FE0720081AD208D32224EB60D9
:10E5BE000424E0700EA20A9208D20BC20AD322C320
:10E5CE0002CD16E4300B0BE516300A02F404A20855
:10E5DE00920A3009EA251520D2E5A2E7920B5002E5
:10E5EE00F404B4260050D8CCC0E0EDC0E0EEC0E09C
:10E5FE00EFC0E0EC12CEE3D0E0FFD0E0FED0E0FDC5
:10E60E00D0E0FC200B0512CA4C800312CB55300A09
:06E61E000312CC5BC322D5
:10CE6C00C0E0EFFBEEFAEDF9ECF812CA4CD0E0F5AD
:10CE7C00F0EFFBEEFAEDF9ECF812D1CEA3E8C0E03E
:10CE8C00E9C0E0EAC0E0EBC0E0C0F012CA4C12D13D
:10CE9C00EAA312C95BD0F0D0E0FBD0E0FAD0E0F905
:07CEAC00D0E0F8D5F0D72219
:10E6240033DA929E35B16011377FE5FE3921848952
:10E634003AAEC3FF3C1D955B3D6358473E75FDF004
:10E644003F3172183F800000C2D502CD2002CD16A2
:10E65400BD80FA50F302CD1DED33EC330460F17B41
:10E664003B7AAA79B8783F12CA4CED33EC3392D591
:10E67400247B5011A2D570DB500BED448024045050
:10E6840004A2D580CEEFFBEEFAEDF9ECF812CCAA99
:10E69400EFF582F404FC12CC7612C95BC08290E6DA
:10E6A40024740912CE7BED33CC33D0F092D525F00F
:0AE6B400A2D57001C313CC13FD22A0
:10E6BE003E9248DA3ECCCCCD3F2AAAAB40000000B9
:10E6CE003F8000003F9837F03FB504F33FD744FC3E
:10E6DE003E3172173EB172173F0515913EDE5BD982
:10E6EE00D2018002C201EDD2E7F8CD33EC330470D3
:10E6FE000BBD800592D502CD2002CD1640FBD31462
:10E70E0060F2F5F07C3FEE7A00C39496C8948B408D
:10E71E00230AC89469C8941A401A0AC89468C894FF
:10E72E001F40110AC8945AC89425400805F07A0073
:10E73E00CDC2E7CDC0F090692C12D1FAEA2323C0E6
:10E74E00E024CEF582E434E6F583C083C08212D194
:10E75E00EAD082D08312C95BECC0E0EDC0E0EEC01F
:10E76E00E0EFC0E012D1CE90692C12D1DE12C95763
:10E77E00D0E0FBD0E0FAD0E0F9D0E0B2E7F812CB6F
:10E78E005590692C12D1FA90E6BE740312CE6C909D
:10E79E00692C12D1DE12CA4CD0E0600F24DAF58259
:10E7AE00E424E6F58312D1EA12C95B90692C12D1EA
:10E7BE00FAD0E0C3947FFDE49400FC12CC717B1878
:10E7CE007A727931783F12CA4C90692C12D1DE12CE
:10E7DE00C95B30010B7BD97A5B79DE783E12CA4C6D
:01E7EE002208
:10CEB3003F8000004120000042C80000447A000087
:10CEC300461C400047C35000497424004B18968009
:10CED3004CBEBC205A0E1BCA6753C21C749DC5AE00
:10CEE300FB60065407601C232312CF11EB543860F8
:10CEF3000912CEFD12CF0C12CA4CECF8EDF9EEFA82
:10CF0300EFCB22EB12CF0C80F1543803241C90CECC
:10CF1300B3FE93FC0EEE93FD0EEE930ECE93FF2223
:0300000002E7EF25
:0CE7EF00787FE4F6D8FD75814102E83621
:10CF2300E709F608DFFA8046E709F208DFFA803EF0
:10CF330088828C83E709F0A3DFFA8032E309F608DD
:10CF4300DFFA8078E309F208DFFA807088828C8345
:10CF5300E309F0A3DFFA806489828A83E0A3F608F9
:10CF6300DFFA805889828A83E0A3F208DFFA804CD3
:10CF730080D280FA80C680D4806980F280338010AA
:10CF830080A680EA809A80A880DA80E280CA803313
:10CF930089828A83ECFAE493A3C8C582C8CCC5838B
:10CFA300CCF0A3C8C582C8CCC583CCDFE9DEE7805B
:10CFB3000D89828A83E493A3F608DFF9ECFAA9F0DA
:10CFC300EDFB2289828A83ECFAE0A3C8C582C8CC30
:10CFD300C583CCF0A3C8C582C8CCC583CCDFEADE49
:10CFE300E880DB89828A83E493A3F208DFF980CCAB
:10CFF30088F0ED2402B4040050C2F582EB2402B49D
:10D00300040050B823234582F582EF4E60AEEF60F3
:09D01300010EE5822390CF737336
:10D01C00BB010689828A83E0225002E722BBFE0212
:09D02C00E32289828A83E4932245
:10D03500BB010CE58229F582E5833AF583E02250B0
:10D0450006E92582F8E622BBFE06E92582F8E222FA
:0DD05500E58229F582E5833AF583E4932214
:10D06200BB010689828A83F0225002F722BBFE01AD
:02D07200F322A7
:10D07400EFF88DF0A4FFEDC5F0CEA42EFEEC88F001
:04D08400A42EFE22B6
:10D08800C2D5EC30E709B2D5E4C39DFDE49CFCEEC3
:10D0980030E715B2D5E4C39FFFE49EFE12D5ADC3B9
:10D0A800E49DFDE49CFC800312D5AD30D507C3E4B4
:06D0B8009FFFE49EFE2232
:10D0BE00C5F0F8A3E028F0C5F0F8E58215827002FD
:06D0CE001583E038F0229A
:10D0D400A3F8E0C5F025F0F0E5821582700215830F
:06D0E400E0C838F0E8226C
:10D0EA00BB010A89828A83F0E5F0A3F0225006F791
:0FD0FA0009A7F01922BBFE06F3E5F009F319228E
:0DD10900EF2BFFEE3AFEED39FDEC38FC2275
:0ED11600C3EF9BFFEE9AFEED99FDEC98FC2214
:10D12400E88FF0A4CC8BF0A42CFCE98EF0A42CFCAA
:10D134008AF0EDA42CFCEA8EF0A4CDA8F08BF0A428
:10D144002DCC3825F0FDE98FF0A42CCD35F0FCEB87
:10D154008EF0A4FEA9F0EB8FF0A4CFC5F02ECD394C
:0FD16400FEE43CFCEAA42DCE35F0FDE43CFC22B9
:10E87B00C2D5E830E70FB2D5E4C39BFBE49AFAE4C8
:10E88B0099F9E498F8EC30E717B2D512E8B112D643
:10E89B003EE4C39BFBE49AFAE499F9E498F880030D
:10E8AB0012D63E30D50DE4C39FFFE49EFEE49DFDE2
:04E8BB00E49CFC22BB
:0ED17300C3E49FFFE49EFEE49DFDE49CFC22CD
:10D18100EB9FF5F0EA9E42F0E99D42F0EC6480C825
:06D1910064809845F022C5
:10D19700EB9FF5F0EA9E42F0E99D42F0E89C45F0EE
:01D1A7002265
:10D1A800BB010789828A8302D1FA5005E9F802D6C1
:0AD1B800D0BBFE05E9F802D6DC2228
:0CD1C200E0FCA3E0FDA3E0FEA3E0FF22E0
:10D1CE00E493FCA3E493FDA3E493FEA3E493FF2274
:0CD1DE00E0F8A3E0F9A3E0FAA3E0FB22D4
:10D1EA00E493F8A3E493F9A3E493FAA3E493FB2268
:0CD1FA00ECF0A3EDF0A3EEF0A3EFF022A8
:10D20600A8828583F0D083D08212D21D12D21D123D
:10D21600D21D12D21DE473E493A3C583C5F0C58362
:10D22600C8C582C8F0A3C583C5F0C583C8C582C872
:01D2360022D5
:0CD23700A42582F582E5F03583F5832202
:10D24300FAE6FB0808E6F925F0F618E6CA3AF622EC
:09D25300E0FBA3E0FAA3E0F922DC
:10D25C00F8E0FBA3A3E0F925F0F0E582158270025B
:07D26C001583E0FA38F022FF
:10D27300F8E0FBA3A3E025F0F9F0E5821582700244
:07D283001583E038FAF022E8
:09D28A00EBF0A3EAF0A3E9F022A5
:0CD29300E493FB740193FA740293F922F7
:10D29F00D083D082F8E4937012740193700DA3A31E
:10D2AF0093F8740193F5828883E473740293686032
:06D2BF00EFA3A3A380DF32
:10D2C500D083D082F8E4937012740193700DA3A3F8
:10D2D50093F8740193F5828883E473740293B5F02F
:0DD2E500067403936860E9A3A3A3A380D897
:10E8BF00EFB40A07740D12E8CA740A309811A899B8
:10E8CF00B8130CC2983098FDA899C298B811F630B9
:07E8DF0099FDC299F5992291
:10E8E60010000B12EBEBBF0D027F0A02E8BF906728
:04E8F600D4E0FF2249
:08E8FA009067D4EFF0D2002278
:10E90200EFC394094006EFC3940E4004EFB4200312
:05E91200D38001C322C7
:10E91700C3EE6480948040028007C3E49FFFE49EB7
:02E92700FE22CE
:10E929009068C212D1FA7F007E007D007C00906859
:10E93900C2E0F8A3E0F9A3E0FAA3E0FBC312D18196
:10E9490040109068C2E0FCA3E0FDA3E0FEA3E0FF55
:10E9590080119068C2E0FCA3E0FDA3E0FEA3E0FF04
:04E9690012D1732232
:10D2F200E3F5F009E208B5F06D606B80F3E3F5F059
:10D3020009E608B5F060605E80F387F009E608B5CB
:10D31200F054605280F487F009E208B5F0486046A4
:10D3220080F488828C8387F009E0A3B5F0386036F8
:10D3320080F488828C8387F009E493A3B5F0276098
:10D342002580F388828C83E3F5F009E0A3B5F0161B
:10D35200601480F388828C83E3F5F009E493A3B52B
:10D36200F004600280F202D41D808580E7808E8006
:10D37200D2803C8015806C807E809B80B5808B80C3
:10D38200A1804F8070803A02D43389828A83ECFA7A
:10D39200E493F5F0A3C8C582C8CCC583CCE493A3BB
:10D3A200C8C582C8CCC583CCB5F070606E80E189F7
:10D3B200828A83E493F5F0A3E208B5F05E605C80B4
:10D3C200F289828A83E0F5F0A3E608B5F04D604B5E
:10D3D20080F389828A83E0F5F0A3E208B5F03C602D
:10D3E2003A80F389828A83E493F5F0A3E608B5F0E4
:10D3F2002A602880F2805D89828A83ECFAE493F5C0
:10D40200F0A3C8C582C8CCC583CCE0A3C8C582C876
:10D41200CCC583CCB5F004600280E27F00F845F011
:10D42200600EE863F0806480D395F01F40027F01B4
:10D432002289828A83ECFAE0F5F0A3C8C582C8CCBF
:10D44200C583CCE0A3C8C582C8CCC583CCB5F0CB1C
:10D4520060C980E389828A83ECFAE0F5F0A3C8C54B
:10D4620082C8CCC583CCE493A3C8C582C8CCC5838B
:10D47200CCB5F0A760A580E288F0ED2402B40400E8
:10D482005099F582EB2402B40400508F2323458285
:05D492002390D36B7331
:10E96D009069DCEBF0A3EAF0A3E9F09069DFE0FB3E
:10E97D00A3E0FAA3E0F912D01CFE9069DCE0FBA342
:10E98D00E0FAA3E0F912D01CFD6E702AED600E9036
:10E99D0069E274FFF5F012D0BE45F070037F0022DE
:10E9AD009069DDE475F00112D0BE9069E0E475F078
:10E9BD000112D0BE80B5D3EE6480F8ED648098402E
:07E9CD00037F01227FFF22FE
:10D49700E709F60870FA8046E709F20870FA803E55
:10D4A70088828C83E709F0A370FA807EE309F60887
:10D4B70070FA8076E309F20870FA806E88828C83AE
:10D4C700E309F0A370FA806289828A83E0A3F608F1
:10D4D70070FA805689828A83E0A3F20870FA804A3C
:10D4E70080D280FA80C680D4806580F28031801037
:10D4F70080A680EA809A80A880DA80E280CA80319C
:10D5070089828A83ECFAE493A3C8C582C8CCC58311
:10D51700CCF0A3C8C582C8CCC583CC70E9800D897F
:10D52700828A83E493A3F60870F9ECFAA9F0EDFB7D
:10D537002289828A83ECFAE0A3C8C582C8CCC58356
:10D54700CCF0A3C8C582C8CCC583CC70EA80DD897E
:10D55700828A83E493A3F20870F980CE88F0ED24E1
:10D5670002B4040050C4F582EB2402B4040050BA9C
:09D57700232345822390D4E773BD
:10E9D400E4FFFE12D01C600C0FEF70010E09E97009
:05E9E400F20A80EF22A1
:10E9E900E94A4B70012212D01CFF6D700122EF70B1
:0CE9F90004FBFAF92209E970ED0A80EA3B
:10EA0500906889EBF0A3EAF0A3E9F0906889E0FB50
:10EA1500A3E0FAA3E0F912D01CFF12E902500C9012
:10EA2500688AE475F00112D0BE80E0D20190688951
:10EA3500E0FBA3E0FAA3E0F912D01CFF642B60040D
:10EA4500EFB42D1D906889E0FBA3E475F00112D0A9
:10EA5500D4A9F0FA12D01C642D6003D38001C392AF
:10EA65000190688C12D20600000000906889E0FBD6
:10EA7500A3E0FAA3E0F912D01CFF12EBF5506A7F70
:10EA85000A7E007D007C0090688CE0F8A3E0F9A385
:10EA9500E0FAA3E0FB12D124C8ECC8EDC0E0EEC05B
:10EAA500E0EFC0E0906889E0FBA3E0FAA3E0F9128B
:10EAB500D01CFF3395E0FEEF24D0FFEE34FFFEE4DB
:10EAC500FCFDD0E0FBD0E0FAD0E0F9EB2FFFEA3E09
:10EAD500FEED39FDEC38FC90688C12D1FA90688A0D
:10EAE500E475F00112D0BE808230011090688CE090
:10EAF500FCA3E0FDA3E0FEA3E0FF801190688CE09D
:0EEB0500FCA3E0FDA3E0FEA3E0FF12D173220B
:10EB13009068ADEBF0A3EAF0A3E9F09068ADE0FBF9
:10EB2300A3E0FAA3E0F912D01CFF12E902500C9003
:10EB330068AEE475F00112D0BE80E0D2019068ADFA
:10EB4300E0FBA3E0FAA3E0F912D01CFF642B6004FE
:10EB5300EFB42D1D9068ADE0FBA3E475F00112D076
:10EB6300D4A9F0FA12D01C642D6003D38001C392A0
:10EB730001E49068B0F0A3F09068ADE0FBA3E0FA85
:10EB8300A3E0F912D01CFF12EBF5503F9068ADE003
:10EB9300FBA3E0FAA3E0F912D01CFF3395E0FEEFEC
:10EBA30024D0FBEE34FFFA9068B0E0FEA3E0FF7CD4
:10EBB300007D0A12D074EF2BF0EE3A9068B0F0901B
:10EBC30068AEE475F00112D0BE80AD30010A9068E2
:10EBD300B0E0FEA3E0FF800F9068B0E0FEA3E0FF8B
:08EBE300C3E49FFFE49EFE2243
:10D58000EF4E6013EDBB011089828A83EF60010EBC
:10D59000EDF0A3DFFCDEFA2289F05007F709DFFC8B
:0DD5A000A9F022BBFE06F309DFFCA9F02272
:10E7FB00020003E493A3F8E493A34003F68001F231
:10E80B0008DFF48029E493A3F85407240CC8C3331E
:10E81B00C4540F4420C8834004F456800146F6DFED
:10E82B00E4800B010204081020408090C7CEE47EE8
:10E83B00019360BCA3FF543F30E509541FFEE493E2
:10E84B00A360010ECF54C025E060A840B8E493A3A9
:10E85B00FAE493A3F8E493A3C8C582C8CAC583CAD4
:10E86B00F0A3C8C582C8CAC583CADFE9DEE780BE8C
:01C8780000BF
:10D5AD00BC000BBE0029EF8DF084FFADF022E4CC62
:10D5BD00F875F008EF2FFFEE33FEEC33FCEE9DEC2B
:10D5CD00984005FCEE9DFE0FD5F0E9E4CEFD22ED71
:10D5DD00F8F5F0EE8420D21CFEADF075F008EF2FBB
:10D5ED00FFED33FD4007985006D5F0F222C398FDAC
:05D5FD000FD5F0EA2249
:10D6020075F008758200EF2FFFEE33FECD33CDCCDF
:10D6120033CCC58233C5829BED9AEC99E582984062
:10D622000CF582EE9BFEED9AFDEC99FC0FD5F0D63F
:10D63200E4CEFBE4CDFAE4CCF9A88222B800C1B969
:10D642000059BA002DEC8BF084CFCECDFCE5F0CBA7
:10D65200F97818EF2FFFEE33FEED33FDEC33FCEBE0
:10D6620033FB10D703994004EB99FB0FD8E5E4F99B
:10D67200FA227818EF2FFFEE33FEED33FDEC33FC88
:10D68200C933C910D7059BE99A4007EC9BFCE99A7C
:10D69200F90FD8E0E4C9FAE4CCFB2275F010EF2FC1
:10D6A200FFEE33FEED33FDCC33CCC833C810D707C1
:10D6B2009BEC9AE899400AED9BFDEC9AFCE899F8FC
:0ED6C2000FD5F0DAE4CDFBE4CCFAE4C8F9228F
:0CD6D000ECF608EDF608EEF608EFF62286
:0CD6DC00ECF208EDF208EEF208EFF2228A
:0AEBEB003098FDAF99C2987E002219
:10EBF500EFC394304009EFC3943A5003D38001C367
:01EC050022EC
:00000001FF
